:1000000000400020BD6E0000FD6E0000FF6E00008D
:1000100000000000000000000000000000000000E0
:10002000000000000000000000000000016F000060
:100030000000000000000000036F0000056F0000DA
:10004000076F00002951000039730000076F00009E
:10005000076F000000000000076F0000076F00003E
:10006000076F00000976000081300000076F000074
:10007000076F0000076F0000076F0000076F0000A8
:10008000076F0000A1770000076F0000076F0000F6
:10009000076F0000076F0000076F0000076F000088
:1000A000076F0000076F0000000000000000000064
:1000B0000000000000000000000000000000000040
:1000C00010B5064C2378002B07D1054B002B02D02E
:1000D000044800E000BF0123237010BD600200202F
:1000E00000000000A0E10000044B10B5002B03D07D
:1000F0000349044800E000BF10BDC04600000000F6
:1001000064020020A0E10000164B002B00D1144B2C
:100110009D46402292029A1A924600218B460F4633
:100120001348144A121A0BF0E3F80F4B002B00D0BF
:1001300098470E4B002B00D0984700200021040068
:100140000D000D48002802D00C4800E000BF0BF065
:100150008FF82000290007F00DF90BF063F8C04676
:100160000000080000400020000000000000000027
:1001700060020020B02F00200000000000000000FE
:1001800002000120104011D1042A0ED91368180969
:1001900080B2002809D001388000031D11180979A8
:1001A000002902D001309842F8D170470020FCE7C6
:1001B0000378002B03D05AB2002A01DB01307047CC
:1001C0003F229343C03B59424B41C01803789343AD
:1001D000802BF4D10130F9E710B500240378002B0F
:1001E00001D1200010BDFFF7E3FF0134F6E770B541
:1001F000002204000D00411C092003F05DFA0028D4
:1002000006D001236200134343600023A34200DBB6
:1002100070BD9A00A958821891600133F6E770B555
:10022000012803DC1C2001F039F870BD01230D68A2
:1002300011201D42F7D04868184206D1042804D97D
:100240000F2302681340042B01D00E20EBE703F0CC
:1002500091F86D100400002D03DDFFF7BDFFA842EB
:1002600006DA1220DFE72000FFF7A2FF0400013DBD
:10027000012DF8D120787F2809DDDF280BDCF82359
:100280003F22DB00800118406378134018430123AC
:1002900040001843C9E7EF280BDCFC226378120109
:1002A0009B0113403F220007000C0343A07810403D
:1002B000ECE7F72812DCFC22637892021B03134060
:1002C000E0228004520310403F221843E378134099
:1002D000FC220343A07812018001E8E7012040429C
:1002E000D5E7F8B54D680F00EB0706D4042D04D907
:1002F0000F232E683340092B03D00B2000F0CEFFD4
:10030000F8BD6B683609B6B25C10731EA3420FD8F5
:100310000321200008F0A8FE6421642803DC01000A
:10032000032800DA03212800891903F0F7F90500F2
:100330002B6800201B099BB2013B9C42E0D23A682B
:10034000A31C9B005A510123013464001C436C60C0
:10035000D6E7F0B585B0012803DC1C2000F09EFF35
:100360002CE001274B683A000093022806D08B68E6
:100370003B4203D05F10002F00DC17000124009BDC
:10038000234200D0AEE0042B00D8ABE00F261B6860
:100390000D6801933340042B25D1254205D1042D4E
:1003A00003D92B681E40042E01D00E20D6E70098FA
:1003B000FFF7E6FEB84203DA0120404205B0F0BD87
:1003C000009802F0D7FF0600280002F0D3FF0100DA
:1003D000781E30180BF042FB0028EDD0801B013056
:1003E00040002043EAE7092B3DD1009B5B685B108E
:1003F00001939F42E0DC25422CD1042D2AD92B68A1
:100400003340042B26D1280002F0B4FF039602905B
:100410007E1C009AB300D058854201D17800E0E7F5
:1004200020420ED104280CD90368039A1340042BF0
:1004300007D102F09FFF010002980BF0D9FA0028C3
:10044000ECD0019B37009E42E2DDB5E71F00019B27
:100450009F42B1DC7B1C00999A008A58AA42F5D1D0
:1004600078000124BDE7032B3CD12C402ED1042D74
:100470002CD931002B68194003291DD1180980B2ED
:100480005B0F80000B402E1DC01A019B019A1B09B7
:100490009BB257009B00BF0FDF1B009B3F1A04332A
:1004A0003018BC4200DD87E73200191982420FD3B1
:1004B00016D101346000D4E7042907D1280002F0E6
:1004C00059FF06002800FFF75BFEDEE70F2045E737
:1004D0000D78AC461578AC4502D101310132E5E723
:1004E0000134DEE7212039E710B502F027FF430091
:1004F0000120184310BD0000C30711D404280FD9F0
:100500000F2302681340032B0AD119400133591AF3
:10051000C0234907DB051940024B1A401143016013
:100520007047C046FFFFFF9FF7B507000E001C2075
:10053000012F06DD4C68012322001A40009203D1EE
:100540000D2000F0ABFE53E0022F02D08A681A4261
:10055000F6D0012335681D4200D0A9E0042D00D853
:10056000A6E01C41002C00DC1C000F20296808407C
:10057000092828D16B685B100093022F05D0B3685F
:10058000009A5B109A4200DD0093009B01221D1B24
:100590000135EB43DB171D40691C092003F08CF883
:1005A000071E09D001236D001D4303003268083384
:1005B00045600099A14201DA3800FEBD0134A10076
:1005C000515802C3F5E7042845D1280002F0D2FEB5
:1005D000FFF702FE0190022F04D0B3685B1098422F
:1005E00000DD0193019BA34204DA002003F0D6F85A
:1005F0000700E1E7280002F0BDFE0700009BA342D0
:1006000021DB2800009702F0B5FE05003800FFF757
:10061000CFFD019B01340700A342F7DA009BC41A07
:10062000200003F0BBF8071EC6D002F0A3FE019025
:10063000306802F09FFE2200009B591B4118019870
:100640000AF03AFEB8E73800FFF7B2FD009B07005A
:1006500001330093D2E703282AD10B099BB2490F3B
:100660009B000140591A022F04D0B26852109142E7
:1006700000DD1100A14205DA00220320110003F081
:100680001BF8B5E703200E1B331DD9170140C9180D
:100690008910002203F010F8071E00D18CE7013604
:1006A00031000334FFF728FF381D29193200C7E74E
:1006B000212046E7F8B5002805DC1C2000F0EEFDFF
:1006C00005002800F8BD01260C6826400FD06410F4
:1006D000E343DB171C40E11C89100022032002F0D9
:1006E000EBFF051EEDD02100FFF706FFE9E7042C24
:1006F00001D80025E5E70F2322681340042B1BD106
:100700002000FFF73DFDC31C07000320D91701405F
:10071000C9188910320002F0CFFF051ED1D0390070
:10072000FFF7EAFE200002F025FE2B1D01003A0033
:1007300018000AF0C1FDC4E7092BDAD10320636871
:1007400032005F10FB1CD9170140C918891002F054
:10075000B3FF051ECDD03900FFF7CEFEFF20BE420D
:10076000AFDA0122B300E3189B68134208D01341AB
:10077000FF2B00DD0300D943C917AA190B401371E1
:100780000136ECE710B57F2902DC0170013010BDA5
:100790001A4B99420CDC40238A115B4213430370CD
:1007A0003F230B4080214942194341700230EEE75C
:1007B000134B994210DC20230A135B4213433F245E
:1007C000802203708B1152422340214013430A437D
:1007D000437082700330DAE70A4B9942D7DCF0238A
:1007E0000370603B4370113B8A11FF3B1A438270D8
:1007F0003F2211401943C1700430C8E7FF070000D1
:10080000FFFF0000FF0F0100F0B50D0085B00028CC
:1008100003DC1C2000F042FD0DE009680122080005
:1008200010400AD002AC11412000FFF7ABFF011BC2
:10083000200002F0BFFF04001AE004293FD90F2373
:100840000C682340092B3AD14B685B1001930323BA
:100850009C46019B9A420EDD02F0A0FF041E07D0C9
:100860002E68012502F086FD2F00019B9D421DDDB3
:10087000200005B0F0BD01329300CC580123234085
:1008800001D10D20C6E764107F2C0DDD0D4E022333
:10089000B44209DD0C4E6346B44205DD00270B4E21
:1008A000E30FA6427B419B00C018D2E70135AB00A5
:1008B000F1583942E5D04910FFF764FFD5E7212010
:1008C000A8E7C046FF070000FFFF0000FF0F010080
:1008D00010B504000120084010D104290DD90F23C0
:1008E0000A681340042B08D1080002F043FD010000
:1008F00020000BF07DF84342584110BD0020FCE77A
:10090000F7B50F00012803DC1C2000F0C7FCFEBD7A
:1009100001264D682E4006D1042D04D90F222B68E4
:100920001A40092A01D00B20EFE76A681B099BB225
:100930005410A34200D85C1E39681E48FFF7C8FF58
:1009400001230190002813D139681B48FFF7C0FF2D
:10095000002811D0002C0DD00123621C013C9C40CA
:100960009200535123436B6004E00136B200AB5058
:10097000B442FADA0020CAE73B680D20DA07C4D592
:100980005B10002B11DD9C420FDB9B00A200291D98
:10099000EB1889180433994209D10123013C9C408A
:1009A000AA181C4353606C60E4E71220ADE7586856
:1009B0001860EFE783C9000087C90000002310B565
:1009C0000C000B70C30705D50D49421020000AF03A
:1009D000D3FF08E00B49002802D0042804D10A49BB
:1009E00020000AF0E9FF10BD0428FCD90F2302689B
:1009F0001340042BF7D102F0BDFC04490200E5E7E7
:100A000074D300008CC9000092C9000097C900008F
:100A1000F0B593B0060001911C20012E1EDD019B54
:100A200001251A6814002C4000D022E1042A00D8C5
:100A30001FE111680F221140092949D10294029B3C
:100A400001999B00CB5819002940039105D1042B33
:100A500003D918681040092806D0222000F01EFC97
:100A60000700380013B0F0BD5B685B10E418029B10
:100A7000013302939E42E2D1611C012202F01CFE6E
:100A8000071E01D10027ECE7010064002543039E07
:100A900045600831019AB300D058026843681209D2
:100AA00092B25B109A4200D8531E0022934209DC96
:100AB000DA43D21713409B00C918029B01369E42AD
:100AC000E8DBCEE794000519AD6801320D51EDE782
:100AD00004296DD127000292019ABB00D3582B4202
:100AE00031D1042B2FD9186802990140042932D141
:100AF0001800FFF745FB24180137BE42ECD1200057
:100B000002F04CFE071EBDD0019BB6009B19041DD0
:100B10000293019B1D6801231D4227D1042D25D975
:100B20000F262B681E40042E38D12800FFF728FB23
:100B30000600280002F01EFC0100200032000AF02E
:100B4000BBFBA41920E0180005A9FFF737FF05A893
:100B50000AF058FFCFE7032900D07EE7020992B2DE
:100B6000430F92000B40D31A1C19C5E705A92800B2
:100B7000FFF724FF05A80AF045FF05A905000200BC
:100B800020000AF099FB6419019B04330193019A38
:100B9000029B9342BDD10023237062E7032EF3D161
:100BA0001A0992B25B0F92001E40961B291DC4E7E2
:100BB00003295ED12F0015000294029B019A9B002D
:100BC000D3583B4200D048E7042B00D845E71868CB
:100BD0000100294003293BD1020992B2430F920040
:100BE0000B40D31A1C19029B013302939E42E4D19D
:100BF0000320E31CD9170140C9188910002202F014
:100C00005BFD071E00D13DE72100FFF775FC0025C5
:100C10003E1D019AAB00D45801231C4220D1042C64
:100C20001ED90F2123681940032919D1180980B250
:100C30005B0F80000B40C01A0023834214DBC343C8
:100C4000DB171840029B013536189D42E1DB08E7AF
:100C5000042900D001E71800FFF792FA2418C2E730
:100C60002000FFF78DFAE7E7E2181279F25401331A
:100C7000E3E7212000F012FB04E70000F0B50D00CF
:100C800095B0002806DC1C2000F008FB04002000C2
:100C900015B0F0BD0C68012123000B40009306D174
:100CA000042C04D922680F331A40092A01D00B20E2
:100CB000EAE7626852100392002A03DC009802F00F
:100CC0006DFDE3E73F4A019201280BD068680842B6
:100CD00008D1042806D902681340042B02D102F07F
:100CE00049FB019001980AF08DFE06000F27039B37
:100CF0000834013B04935E43039B02909B001B1945
:100D0000059301232068184251D104284FD9036864
:100D10003B40042B52D1FFF733FA059B04343618BD
:100D2000A342EED1300002F039FD041EAFD02B6893
:100D30000593029B002B03D0686802F01BFB019017
:100D4000200002F017FB0500009B059A9B00D318BA
:100D50009F68380002F00EFB012306001F4201D1FC
:100D6000042F04D807A93800FFF728FE07AE30008B
:100D70000AF048FE07000200310028000AF09CFA41
:100D8000029BED19002B0AD0049B009A934206DDCA
:100D90002800029A01990AF08FFA029BED18009B35
:100DA00001330093009A039B9342CDD16FE707A9CB
:100DB000FFF704FE07A80AF025FEAEE702F0DAFA14
:100DC000F9E7C046D6CD000010B50024A04207DDEB
:100DD0000B6801341C4003D05C10E343DB171C405C
:100DE000611C0122092002F067FC002803D00123C6
:100DF00064001C43446010BD0A6870B510000125F2
:100E0000284034D1042A32D90F24136849681C4081
:100E1000092C17D154681B099BB22C41A34200D85E
:100E20005C1E844205DC02200133984206DB002070
:100E30000FE085005519A9600130F2E784001151D7
:100E40000130F2E7032C12D1294203D1132000F024
:100E500025FA70BD4910FF29F8D81B099BB204324E
:100E60009B00D3189342E2D911700132FAE70B20AC
:100E700000F014FADBE700000123F7B500254E6807
:100E80000F0033400093AB420ED11D00042E0BD94E
:100E90000F2233681A40092A10D172681B099BB2CD
:100EA0005510AB4200D85D1E3968CB0717D54C10E2
:100EB000002C01DDA5421DDA122032E0042A04D103
:100EC0003000FFF75DF90500EEE7009D032AEBD146
:100ED0001D09ADB25B0FAD001340ED1AE4E72E48DB
:100EE000FFF7F6FC002814D00AF0E2FC290008F015
:100EF000A1F94C1C009B002B4CD1042E4AD932681E
:100F00000F331340092B10D10134A400A459200041
:100F1000FEBD39682148FFF7DBFC2C000028E9D131
:100F2000113000F0BBF90400F1E7042B2AD13000A6
:100F300002F020FA0500FFF74FF9A042BCDB012CBC
:100F40001ADC300002F016FA00902800FFF730F9A2
:100F5000461B300002F022FC041ED8D002F00AFA30
:100F60000190786802F006FA009B3200E91A4118F5
:100F700001980AF0A1F9CAE72800FFF719F9013C26
:100F80000500DCE7032B05D13419E478023B64004B
:100F90001C43BCE70B20C4E77CC9000087C90000E4
:100FA000F7B54D680F002A0001210A402FD1042D0A
:100FB0002DD90F242B68BE681C40092C14D16968F8
:100FC0001B099BB24C100192A34200D85C1E3968E9
:100FD0002A48FFF77DFC00282DD00F232A681340F4
:100FE000092B1DD1012317E0032C10D10E4203D190
:100FF000132000F053F9FEBD72100192FF2AF7D8BA
:101000001A0992B25B0F92001C40141BDFE70B2001
:10101000EFE701339A00AE509C42FADA0020EAE78B
:10102000032BFBD12B0001335A1BA242F6DC6A468C
:101030001279DA70F7E73968CB0706D5491000292D
:1010400001DD8C4209DA1220D3E70D48FFF740FC9E
:101050002100002801D11130CBE70F232A6813406B
:10106000092B03D1013189004E51D7E7032BD5D18C
:101070006B461B796D18EB70D0E7C04683C9000042
:1010800087C9000010B50124086820421AD104283D
:1010900018D90F2102681140092901D1406810BDFB
:1010A000032908D113099BB2500F9B000840181A5E
:1010B00040002043F3E7042904D102F05BF9FFF775
:1010C0008BF8F5E70B2000F0E9F8E8E710B5034AE4
:1010D0000B21034804F020F910BDC04624C90000CC
:1010E0001CC9000000207047002070470020704796
:1010F0000020704700207047002070470020704794
:101100000020704700207047002070470020704783
:1011100010B5034A0B21034804F0FEF810BDC04689
:101120000CCA000064CA000010B50124044002D0BB
:101130004410200010BD04280CD90F23026813406E
:10114000042B07D102F016F921000A220AF022FD31
:101150000400EEE70D22014B1A70EAE7A00200201E
:10116000012210B5024018D1042802D903681A09D7
:1011700092B201230B4012D1042902D90B681B093A
:101180009BB20024934206D104309B000431C31863
:10119000984206D30124200010BD0022E9E7002375
:1011A000EFE704780A78002C01D1002AF2D0013050
:1011B00001319442ECD00024EDE70000F0B585B099
:1011C0000393019002912C4E2C4B002A02D0022254
:1011D0003270013A00251A601B68F554019B9D424C
:1011E00001DB05B0F0BD029AAB00D058234B1C6860
:1011F000C8239B0037191C1B0123184206D0204A24
:101200004310210038000AF085FB09E01D4A002840
:1012100002D004281BD11C4A210038000AF07AFBB6
:1012200030000AF0EFFB154A039B1060002B0CD036
:10123000019B013BAB4208DD144B984205D8431C8F
:101240001360202232540022F2540135C6E70428EC
:101250000FD90F2302681340042B04D102F08AF83F
:101260000B4A0300CDE7092B04D14368094A5B1000
:10127000C7E70123084AC4E7A1020020C4050020F3
:1012800074D300008CC9000092C900001F03000045
:1012900083D90000C8CC0000D7CC0000014B1870E7
:1012A00000207047A002002070B501F0D7FD094C66
:1012B0000100251D1F2228000AF0BCFB28000AF0AF
:1012C000A1FB0423043080080001184320602000A3
:1012D00070BDC0467C020020C368F0B59D008368E5
:1012E00089B05D190300183306930369069A9F00BD
:1012F000069B0290DF19436901939B00D318039367
:10130000CD4B1B78002B26D17F222B68CB491C129A
:1013100013409B005B58043501929F46029B58780E
:1013200004F008FC0023029A137027E0C24B1B78DC
:10133000002B10D12B68019A1C121340BF4A9B004E
:101340009B580435E9E7069B3A1DD11ABA4BD829B8
:1013500028DD1A221A70029BB74C9B6821780193F2
:10136000EA1A029B92109B7812021A43029B587849
:1013700004F0E8FB0023029A23701370029B069A84
:101380009B680193ED1A029BAD10DD60069BFE1A6F
:10139000029BB6101E61039B9B1A029A9B1053611D
:1013A00009B0F0BD1B783C60002B01D01700D2E7DC
:1013B0002B6801991C120B40A0499B005B58170039
:1013C0000435AAE7069B3A1DD11A9B4BD82902DDAA
:1013D0001A221A70BFE728681B78291D3860002B75
:1013E00002D017000D00B6E76B6801991C120B4084
:1013F00092499B005B58170008358EE7069B3A1D03
:10140000D11A8D4BD82902DD1A221A70A3E7A40045
:101410001B782C193C60002B01D017009BE72B6830
:1014200001991C120B4085499B005B58170004353D
:1014300073E7069B3A1DD11A7F4BD82902DD1A2289
:101440001A7088E77E49A40061581B783960002B28
:1014500001D017007FE72B6801991C120B407749D8
:101460009B005B581700043557E7043F744B3A68FC
:10147000A400E250704B1B78002B00D06BE72B6868
:10148000019A1C1213406D4A9B009B58043544E797
:101490006B4BA400E058FFF747FE043F0600386896
:1014A000FFF742FE36180120654B76000643E650F2
:1014B000614B1B78002B00D04DE72B68019A1C1262
:1014C00013405E4A9B009B58043526E7069B3A1D55
:1014D000D11A594BD82902DD1A221A703BE7069817
:1014E000039C0121A04202D221000C3909681B781B
:1014F0003960002B01D017002DE72B6801991C12D1
:101500000B404E499B005B581700043505E7069BCE
:101510003A1DD11A484BD82902DD1A221A701AE74F
:101520000699039881420FD203000C3B1B68454982
:101530005B106418E41AA40023583B603E4B1B78F0
:10154000002B05D0170006E7182119700023F4E7D7
:101550002B6801991C120B4038499B005B581700FF
:101560000435DAE6069B039A934219D213000C3B2A
:101570001B68344A043FA4185B10E31A039A3968C5
:101580009B0099502C4B1B78002B00D0E3E62B6876
:10159000019A1C121340294A9B009B580435BCE653
:1015A0001822254B1A70EDE7069B039A93422DD221
:1015B000244B3E1FE31814000C3C04932368049A48
:1015C0005B10D31A039A9B009858FFF7ADFD079064
:1015D0003068FFF7A9FD2468049B64101C1B079B5F
:1015E000A4001F1801207F00039B0743E75037002A
:1015F000114B1B78002B00D0ADE62B68019A1C1212
:1016000013400E4A9B009B58043586E618220A4B6D
:101610001A70EDE7069B3A1DD11A074BD82902DD57
:101620001A221A7097E60399A40061581B78396052
:10163000002B09D017008EE6A0020020C8CA0000C7
:101640007C2D0020FDFFFF3F2B6801991C120B40F1
:10165000D7499B005B58170004355EE6043F039BA7
:101660003A68A400E250D34B1B78002B00D072E6FE
:101670002B68019A1C121340CD4A9B009B580435DD
:101680004BE6039BA4001C192368043F38685E10D6
:10169000FFF74AFD36180120C64B76001B7806433B
:1016A0002660002B00D056E62B68019A1C121340CE
:1016B000BF4A9B009B5804352FE6069BA4003F1BA6
:1016C000BC4CBB420CD82378002B00D043E62B68DF
:1016D000019A1C121340B64A9B009B5804351CE625
:1016E000B54801F037FE2378002B00D033E62B6895
:1016F000019A1C121340AE4A9B009B5804350CE61D
:10170000A300ED18002C00DA38E6AA4B1B78002B5A
:1017100000D020E62B68019A1C121340A44A9B00BB
:101720009B580435F9E5043F3B68042B04D1A30022
:10173000ED18002C00DA21E69E4B1B78002B00D020
:1017400009E62B68019A1C121340994A9B009B588A
:101750000435E2E5043F3B68042B06D0A200AD1837
:10176000002C02DA002B00D108E6924B1B78002BEC
:1017700000D0F0E52B68019A1C1213408C4A9B00A4
:101780009B580435C9E53A1F13685B10013B002BD9
:1017900006DD01215B00A4000B432D191360EDE56C
:1017A000844B17001B78002B00D0D4E52B68019ADE
:1017B0001C1213407E4A9B009B580435ADE53A004D
:1017C000069B0C32D31AD82B03DD1A22794B1A70E0
:1017D000C1E5FF2361005B001940FE3BFF3B19435D
:1017E0003960029906988968241204916D1A029949
:1017F000AD1089782D020D4303999D40091A891077
:1018000099401D430B43BB60029B7D609C70E4B21A
:101810006A4BE4000392E358029A9360654A127897
:10182000002A03D008331D00039F94E51D00019A90
:101830009B680C351C1213405D4A9B009B58039F0C
:101840006BE53B1F1C68039A069B93422DD10A202F
:10185000E3070CD4042C13D90F2322681340042B64
:1018600011D1200001F086FD0AF0CCF8063064307A
:1018700003F0E6FD00280FD1043D069B03937DE5B0
:101880000720042CF3D02000431E9841FA23404245
:10189000FF3318400730EAE7029B2100587804F034
:1018A00063F90023029A1370E7E7039B039A0C3B4A
:1018B0001B6802995B109B00D31A0C3B1C601F1D18
:1018C0001300083B1B685A108A70D2B23B49D20001
:1018D0005B0055589B0A029A9B009560ED18039B8C
:1018E000069A043B1B685B109B00D3180393314B93
:1018F0001B78002B00D02EE52B68019A1C12134098
:101900002B4A9B009B58043507E53B1F1868FFF7DF
:101910000BFCA40006003F1B1E2827DC00280DDC62
:10192000244B1B78002B00D015E52B68019A1C1264
:1019300013401F4A9B009B580435EEE401F07CFAEB
:10194000033E361801F078FA1D4B801B9842F9D8F7
:10195000184B1B78002B00D0FDE42B68019A1C1259
:101960001340134A9B009B580435D6E40123029A86
:10197000137001F061FA029B0A3886195E60FDE47B
:101980003B1F1868FFF7D0FBA40006003F1B002890
:1019900018DC084B1B78002B00D0DCE42B68019A84
:1019A0001C121340024A9B009B580435B5E4C04604
:1019B000C8CA0000A0020020E9CC00008425002055
:1019C0003F420F00C84B984203DD1D22C74B1A70DF
:1019D000C1E40123029A137001F02EFAFA239B004E
:1019E0005E43029B0A3E30185860C7E4A300FF1A0A
:1019F000002320001A003900FFF7E0FBBC4EBD4C6D
:101A00003168200001F0D6FEBB4B31681860200021
:101A100003F05EFF3168200004F0ADF8B34B1B7893
:101A2000002B00D097E42B68019A1C121340B34A94
:101A30009B009B58043570E4AC4BA4001B783F1B03
:101A4000002B00D087E42B68019A1C121340AB4A8C
:101A50009B009B58043560E4029803F055FDA34BAE
:101A60001B78002B00D076E42B68019A1C121340DF
:101A7000A24A9B009B5804354FE43B1F1B68002B78
:101A80003ED13B000C3B1B68DA072CD53900012204
:101A90005B105800083902430A60002B44DD012224
:101AA00059001143381F0160390008390968114194
:101AB000CB1A39000C390968114224D09B18934085
:101AC000A4001343039AA350884B1B78002B00D02B
:101AD00041E42B68019A1C121340884A9B009B58D2
:101AE0000435FFF71AFC042B06D90F211A680A40A7
:101AF000092A01D15B68C9E719227C4B1A702AE4D4
:101B00005B10013BC9E7042909D90F200A6802408C
:101B1000092A04D102339B005B58A400D2E71922A2
:101B2000724B1A70FFF717FC0435CDE7A300069A35
:101B3000FB189B1AD82B13DC0122631E002C14DC2B
:101B40006A4B1B78002B01D0FFF705FC2B68019A2C
:101B50001C121340694A9B009B580435FFF7DDFBBC
:101B60001A22624B1A70FFF7F6FB3A601C0004372A
:101B7000E3E7069A3B1D9B1A5C4ED82B03DD1A2324
:101B80003370FFF7E8FB069B039AA40093422AD226
:101B90003B1F1868FFF7C8FA011E21DD039B0C3BB1
:101BA0001A68521082421BDB9007801A544B40186F
:101BB000C018039B8000C2583B1B1A604B4B3F1B55
:101BC0001B780437002B01D0FFF7C5FB2B68019A67
:101BD0001C121340494A9B009B580435FFF79DFB9C
:101BE00020233370EAE71823FBE7434BA4001A686D
:101BF0003B1B1F001A603D4B04371B78002B01D0A4
:101C0000FFF7A9FB2B68019A1C1213403B4A9B006B
:101C10009B580435FFF781FBA3009C46FE1A002C5D
:101C200017DC1C22314B1A70002333606346FF1A05
:101C30002E4B04371B78002B01D0FFF78CFB2B6851
:101C4000019A1C1213402D4A9B009B580435FFF744
:101C500064FB002033685A108300F15801230B40C5
:101C600003D10D21214A1170DFE749108A4200DDBE
:101C70000A0001308442EFDC012352001343D4E711
:101C8000A3009C46FE1A002C17DC1C22174B1A706E
:101C9000002333606346FF1A144B04371B78002B74
:101CA00001D0FFF758FB2B68019A1C121340134A0E
:101CB0009B009B580435FFF730FB002033685A1017
:101CC0008300F15801230B4003D10D21074A117005
:101CD000DFE749108A4200DA0A0001308442EFDC73
:101CE000012352001343D4E780EE3600A002002007
:101CF000C4050020A102002008000020C8CA00007E
:101D0000FCFFFF3F3B00083B1868FFF70DFA3B1F45
:101D100006001868FFF708FA0023864200DA043349
:101D2000A4003A1B17001360E54B04371B78002B07
:101D300001D0FFF710FB2B68019A1C121340E14AF7
:101D40009B009B580435FFF7E8FA3B00083B1868F6
:101D5000FFF7EAF93B1F06001868FFF7E5F9F30FF4
:101D6000C217B0425341A4003A1B17009B001360F6
:101D7000D34B04371B78002B01D0FFF7ECFA2B680C
:101D8000019A1C121340CF4A9B009B580435FFF761
:101D9000C4FA3B00083B18683B1F1968A600BE1B2D
:101DA0000423814202D0042802D80023336018E0C3
:101DB00001239C461842F8D10F2302681A40042AD6
:101DC000F3D163461942F0D10429EED90B680B32E6
:101DD0001340042BE9D1FFF7C3F9431E984180005B
:101DE0003060B74BA4001B783F1B0437002B01D099
:101DF000FFF7B1FA2B68019A1C121340B14A9B00FD
:101E00009B580435FFF789FA3B00083B18683B1FD5
:101E10001968A600BE1B0023814202D0042802D804
:101E20000423336018E001239C461842F8D10F23A5
:101E300002681A40042AF3D163461942F0D10429FA
:101E4000EED90B680B321340042BE9D1FFF788F968
:101E50004342584180003060994BA4001B783F1BDF
:101E60000437002B01D0FFF776FA2B68019A1C1279
:101E70001340944A9B009B580435FFF74EFA3B00F1
:101E8000083B1868FFF750F93B1F06001868FFF77A
:101E90004BF9F317C20F86425341A4003A1B1700B7
:101EA0009B001360864B04371B78002B01D0FFF793
:101EB00052FA2B68019A1C121340824A9B009B58CD
:101EC0000435FFF72AFA3B00083B1868FFF72CF9A6
:101ED0003B1F06001868FFF727F90023864200DD44
:101EE0000433A4003A1B17001360754B04371B78AA
:101EF000002B01D0FFF72FFA2B68019A1C12134018
:101F0000704A9B009B580435FFF707FA3B1F1B687C
:101F1000A400043B5A1E93413A1B17009B00136018
:101F2000674B04371B78002B01D0FFF714FA2B689E
:101F3000019A1C121340634A9B009B580435FFF71B
:101F4000ECF93B00083B1868FFF7EEF83B1F060072
:101F50001868FFF7E9F832180120A4003B1B1F00A6
:101F6000520002431A60564B04371B78002B01D0F5
:101F7000FFF7F1F92B68019A1C121340514A9B009C
:101F80009B580435FFF7C9F93B00083B1868FFF779
:101F9000CBF83B1F06001868FFF7C6F8321A01207D
:101FA000A4003B1B1F00520002431A60444B04373D
:101FB0001B78002B01D0FFF7CEF92B68019A1C1279
:101FC0001340404A9B009B580435FFF7A6F93B009D
:101FD000083B1868FFF7A8F83B1F06001868FFF7D2
:101FE000A3F802000120A4003B1B1F007243520013
:101FF00002431A60324B04371B78002B01D0FFF7E5
:10200000AAF92B68019A1C1213402E4A9B009B5878
:102010000435FFF782F93B1F1868FFF785F8061EA5
:1020200017D11F23264A1370A4003B1B1F001E60FC
:10203000234B04371B78002B01D0FFF78CF92B685A
:10204000019A1C1213401F4A9B009B580435FFF74E
:1020500064F93B00083B1868FFF766F8310007F0A9
:1020600003F8012640000643DEE73B1F1868FFF730
:102070005BF8061E17D11F23114A1370A4003B1BE7
:102080001F001E600E4B04371B78002B01D0FFF79A
:1020900062F92B68019A1C1213400A4A9B009B5854
:1020A0000435FFF73AF93B00083B1868FFF73CF8A6
:1020B000310007F0BFF8012649000E43DEE7C046B5
:1020C000A0020020C8CA00003B1F1868FFF72CF8C8
:1020D000C217801850400122A4003B1B1F00400083
:1020E00010431860F14B04371B78002B01D0FFF729
:1020F00032F92B68019A1C121340ED4A9B009B5841
:102100000435FFF70AF9A300FE1A3068012C24D128
:10211000FFF70AF80494079009F0CAFB0799002911
:1021200000DC012107F086F8049BA400C9180123F4
:1021300049001943DD4B3F1B1B7831600437002BEE
:1021400001D0FFF708F92B68019A1C121340D84AF6
:102150009B009B580435FFF7E0F8FEF7E5FF04907D
:102160007068FEF7E1FF049B0130C31A0793D3E7C1
:10217000A300FE1A31002000049301F09DFC049B93
:102180003060FF1AC94B04371B78002B01D0FFF7D2
:10219000E2F82B68019A1C121340C54A9B009B5819
:1021A0000435FFF7BAF83B00083B1868FEF7BCFFA0
:1021B0003B1F06001868FEF7B7FF02000120A400CD
:1021C0003B1B1F003240520002431A60B74B0437DA
:1021D0001B78002B01D0FFF7BEF82B68019A1C1268
:1021E0001340B34A9B009B580435FFF796F83B0019
:1021F000083B1868FEF798FF06003B1F1868FEF7BB
:1022000093FF320002430120A4003B1B1F00520039
:1022100002431A60A54B04371B78002B01D0FFF74F
:102220009AF82B68019A1C121340A14A9B009B58F4
:102230000435FFF772F83B00083B1868FEF774FF9F
:1022400006003B1F1868FEF76FFF32004240012076
:10225000A4003B1B1F00520002431A60934B04373B
:102260001B78002B01D0FFF776F82B68019A1C121F
:1022700013408F4A9B009B580435FFF74EF83B1FD5
:102280001868FEF751FFC0430122A4003B1B1F004A
:10229000400010431860854B04371B78002B01D099
:1022A000FFF759F82B68019A1C121340804A9B00D3
:1022B0009B580435FFF731F83B00083B1868FEF7E0
:1022C00033FF06003B1F1868FEF72EFF32008240E6
:1022D00051000122A4003B1B1F000A431A60734BEC
:1022E00004371B78002B01D0FFF735F82B68019AD3
:1022F0001C1213406E4A9B009B580435FFF70DF8E3
:102300003B00083B1868FEF70FFF06003B1F1868EC
:10231000FEF70AFF3200024151000122A4003B1BDC
:102320001F000A431A60614B04371B78002B01D051
:10233000FFF711F82B68019A1C1213405C4A9B00AE
:102340009B580435FEF7E9FF3B000C3B1868FEF78D
:10235000EBFE3B00083B06001868FEF7E5FEF117B0
:102360000200C317300006F0B7FF3B1F0490059131
:102370001868FEF7D9FE02000498059906F060FF80
:1023800043000120A4003E1B37001843474B306038
:102390001B780437002B01D0FEF7DDFF2B68019A74
:1023A0001C121340424A9B009B580435FEF7B5FFB0
:1023B000A300FE1A310020000493FEF705FD049BE4
:1023C0003060FF1A394B04371B78002B01D0FEF721
:1023D000C2FF2B68019A1C121340354A9B009B5880
:1023E0000435FEF79AFFA300FF1A39002000FEF71C
:1023F00003FD2E4B1B78002B01D0FEF7ACFF2B68A2
:10240000019A1C1213402A4A9B009B580435FEF780
:1024100084FFA300FE1A310020000493FEF72CFD78
:10242000049B3060FF1A214B04371B78002B01D02E
:10243000FEF791FF2B68019A1C1213401C4A9B0067
:102440009B580435FEF769FFA300FF1A39002000EE
:10245000FEF7A6FD154B1B78002B01D0FEF77BFF86
:102460002B68019A1C121340114A9B009B5804359B
:10247000FEF753FFA300FE1A310020000493FEF77D
:1024800001FE049B3060FF1A084B04371B78002BB9
:1024900001D0FEF760FF2B68019A1C121340044A1A
:1024A0009B009B580435FEF738FFC046A002002071
:1024B000C8CA00003B1F186800F05CFF3A00083AE9
:1024C00012680300A400D10729D4042A0CD910688B
:1024D0000F221040013808280FD806F027FD0520EC
:1024E0000E220E0E0E0E2400F049180009F080FA9C
:1024F000434258413B1B80001860ED4B3F1B1B784B
:102500000437002B01D0FEF726FF2B68019A1C121E
:102510001340E84A9B009B580435FEF7FEFEE6494F
:10252000E3E7E649E1E7E649DFE7069B3E1DF31AEC
:10253000DF4CD82B03DD1A232370FEF70CFF00F0CD
:1025400085FC43000120184323783860002B02D01B
:102550003700FEF700FF2B68019A1C121340D54A82
:102560009B009B5837000435FEF7D7FE069B3E1DA7
:10257000F31ACF4CD82B03DD1A232370FEF7EBFEA2
:1025800000F05AFCCF4B4000184001231843237839
:102590003860002B02D03700FEF7DDFE2B68019A71
:1025A0001C121340C34A9B009B5837000435FEF7AA
:1025B000B4FE0123A600BE1B20001A003100FEF766
:1025C000FDFDC14C2068643002F03AFF002802D1C2
:1025D000043DFEF7D3FE029B21685A78BB4803F006
:1025E000D8FA0123029A3700137000F025FCB84B8B
:1025F00022681B68063253431818029B5860FEF786
:10260000BDFEA600BE1B2000012300223100FEF704
:10261000D5FDAD4C2068643002F012FF0028D7D001
:10262000AA4803F0ADF8DCE7A4003E1BFEF73CFE31
:1026300037009F4B30601B780437002B01D0FEF72A
:102640008AFE2B68019A1C1213409A4A9B009B58E1
:102650000435FEF762FEA4003E1B300000F025FCAE
:102660003700934B30601B780437002B01D0FEF706
:1026700072FE2B68019A1C1213408E4A9B009B58D5
:102680000435FEF74AFEA4003E1B300000F00FFCAC
:102690003700874B30601B780437002B01D0FEF7E2
:1026A0005AFE2B68019A1C121340824A9B009B58C9
:1026B0000435FEF732FEA300FE1A31002000049319
:1026C00000F0F8FB049B3060FF1A794B04371B784D
:1026D000002B01D0FEF73FFE2B68019A1C1213401D
:1026E000744A9B009B580435FEF717FEA4003F1B5D
:1026F000380000F011FC6E4B1B78002B01D0FEF768
:102700002AFE2B68019A1C1213406A4A9B009B58B0
:102710000435FEF702FEA300FE1A310020000493E8
:1027200000F022FC049B3060FF1A614B04371B78D9
:10273000002B01D0FEF70FFE2B68019A1C121340EC
:102740005C4A9B009B580435FEF7E7FDA4003F1B45
:10275000380000F04BFC564B1B78002B01D0FEF7E5
:10276000FAFD2B68019A1C121340524A9B009B5899
:102770000435FEF7D2FD0121200000F01FFC4C4B78
:102780001B78002B01D0FEF7E6FD2B68019A1C1286
:102790001340484A9B009B580435FEF7BEFD0021BC
:1027A000200000F00BFC424B1B78002B01D0FEF701
:1027B000D2FD2B68019A1C1213403E4A9B009B5885
:1027C0000435FEF7AAFDA4003E1B300000F030FCEB
:1027D0003700374B30601B780437002B01D0FEF7F1
:1027E000BAFD2B68019A1C121340324A9B009B5879
:1027F0000435FEF792FDA4003E1B300000F02CFCD7
:1028000037002B4B30601B780437002B01D0FEF7CC
:10281000A2FD2B68019A1C121340264A9B009B586C
:102820000435FEF77AFDA4003F1B380000F0EEFBF4
:102830001F4B1B78002B01D0FEF78DFD2B68019AF2
:102840001C1213401B4A9B009B580435FEF765FD84
:10285000A4003F1B380003F07DFC154B1B78002BB8
:1028600001D0FEF778FD2B68019A1C121340114A23
:102870009B009B580435FEF750FDA4003E1B300022
:1028800003F016FD37000A4B30601B780437002B2D
:1028900001D0FEF760FD2B68019A1C121340054A17
:1028A0009B009B580435FEF738FDC046F9CC00006C
:1028B000A0020020C8CA000001CD000008CD000021
:1028C0000FCD0000FEFFFF7FC4050020A102002005
:1028D00004000020A4003F1B380003F00BFCC24B97
:1028E0001B78002B01D0FEF736FD2B68019A1C12D5
:1028F0001340BE4A9B009B580435FEF70EFDA40012
:102900003E1B300003F00CFC3700B74B30601B78E7
:102910000437002B01D0FEF71EFD2B68019A1C1214
:102920001340B24A9B009B580435FEF7F6FCA30007
:10293000FF1A3900200001F0E9FBAB4B1B78002B9C
:1029400001D0FEF708FD2B68019A1C121340A74A1C
:102950009B009B580435FEF7E0FCA300FF1A3900EA
:10296000200001F00DFAA04B1B78002B01D0FEF7E0
:10297000F2FC2B68019A1C1213409C4A9B009B5846
:102980000435FEF7CAFCA300FF1A3900200001F04D
:10299000F5FA954B1B78002B01D0FEF7DCFC2B6879
:1029A000019A1C121340914A9B009B580435FEF774
:1029B000B4FCA300FF1A3900200001F007FB8A4B8A
:1029C0001B78002B01D0FEF7C6FC2B68019A1C1265
:1029D0001340864A9B009B580435FEF79EFCA300DB
:1029E000FE1A31002000049303F0DDFC049B3060EC
:1029F000FF1A7D4B04371B78002B01D0FEF7ABFC90
:102A00002B68019A1C121340784A9B009B5804358E
:102A1000FEF783FCA300FE1A31002000049303F0AC
:102A2000CAFC049B3060FF1A6F4B04371B78002BE5
:102A300001D0FEF790FC2B68019A1C1213406B4AE0
:102A40009B009B580435FEF768FCA300FE1A31007A
:102A50002000049303F0B7FC049B3060FF1A624B24
:102A600004371B78002B01D0FEF775FC2B68019A08
:102A70001C1213405D4A9B009B580435FEF74DFC29
:102A8000A300FE1A31002000049303F0A4FC049B71
:102A90003060FF1A544B04371B78002B01D0FEF72F
:102AA0005AFC2B68019A1C121340504A9B009B58F9
:102AB0000435FEF732FCA300FF1A3900200001F0B4
:102AC00097F9494B1B78002B01D0FEF744FC2B688B
:102AD000019A1C121340454A9B009B580435FEF78F
:102AE0001CFCA300FF1A3900200001F097FA3E4BAE
:102AF0001B78002B01D0FEF72EFC2B68019A1C12CC
:102B000013403A4A9B009B580435FEF706FCA3008D
:102B1000FE1A31002000049301F0FCF9049B3060A0
:102B2000FF1A314B04371B78002B01D0FEF713FC42
:102B30002B68019A1C1213402C4A9B009B580435A9
:102B4000FEF7EBFBA300FF1A3900200001F0AEF9FD
:102B5000254B1B78002B01D0FEF7FDFB2B68019A5B
:102B60001C121340214A9B009B580435FEF7D5FBED
:102B7000069B029AFB1A9B101361A300FF1A3900EF
:102B8000200002F0DDFB184B1B78002B01D0FEF774
:102B9000E2FB2B68019A1C121340144A9B009B58BD
:102BA0000435FEF7BAFB069B029AFB1A9B101361D1
:102BB000A300FE1A31002000049302F0C1FB049B25
:102BC0003060FF1A084B04371B78002B01D0FEF74A
:102BD000C2FB2B68019A1C121340044A9B009B58AD
:102BE0000435FEF79AFBC046A0020020C8CA0000C8
:102BF0000023F7B55A1E0192002B07DA01F09CFA68
:102C000002F0C4FE03F024F81923019300263000DB
:102C1000194B1968B14212DD184B1A6801328A4209
:102C20000FDAF0241A601D68154F6C43E35D002B2A
:102C30001FD0E419022B06D12000FEF74DFB019BAB
:102C4000D8E70022EDE7012B0DD1002801D100F0DB
:102C5000F3F8F0226A43BB185B680A49C31A8B4237
:102C600001D80223BB54F0235D43054BEB5C022BE0
:102C7000E2D00136CCE7C046C805002000000020A5
:102C8000241C00203F420F00012200210A4B0B4868
:102C90001A61195004301950A2210420C90058505B
:102CA000C121C0208900800258501A60044BFC31B9
:102CB0001960044B1A70704700A000400405000022
:102CC00000E100E0EC05002004207047F8B550C991
:102CD000012322001A40101E2DD03340181E2AD086
:102CE00064100020192C26D81D4B761035009E420A
:102CF00000DD1D001B4F3B5D012B05D00121200095
:102D000004F0CEFC01233B55174B1B78002B01D15F
:102D1000FFF7BAFF0023154A9E420DDCFF25144938
:102D20001448D65CB44202D15E007052D5540133CF
:102D3000042BF6D10420F8BDD15C8C4203D10C4A9F
:102D40005B009D52F6E70133042BF5D10023D15CE3
:102D5000FF2901D1D454F2E70133042BF7D1E9E77D
:102D600088130000D0050020EC0500201C00002086
:102D70000E000020DC050000F8B530C90126230054
:102D80003340181E1BD02B003340181E17D034417F
:102D90000020192C13D8174F3B5DB34204D03100EB
:102DA000200004F07DFC3E5569100800124A1038DE
:102DB000124B904204D9012252421A600420F8BDFD
:102DC0001C600F4806F050F90E4B18800E4B1B7814
:102DD000002B02D1FFF758FFF0E701220B4B9A645A
:102DE000A922D2009A588018A82280B2D200985006
:102DF000E4E7C046D00500209086010018000020BE
:102E000020A107000C000020EC05002000A00040DD
:102E10000420704701220020054B06491A615850D2
:102E20000431033058500831801858501A607047E8
:102E300000800040040500000122034B1A64A82210
:102E4000D20098587047C0460080004010B5FFF788
:102E5000F3FFFA21890006F07DF810BD00487047A5
:102E600054CD00001A20704770B5054E0400335C45
:102E70000D008B4202D004F013FC355570BDC046E6
:102E8000D005002070B50024064D635D012B05D1EF
:102E90000021200004F004FC0023635501341A2CA7
:102EA000F2D170BDD005002070470D20704735204D
:102EB00070470000F8B501240B6806000D0023429E
:102EC00004D10D20FEF7EAF92000F8BD5B102000C8
:102ED000052BFAD80E4A9B009C580E4F3B5D002BE9
:102EE00005D00021200004F0DBFB00233B55012E20
:102EF00006DD6B68042B03D10221200004F0D0FB17
:102F0000200004F07BFA012440002043DDE7C046A6
:102F10003CCD0000D0050020F8B5012605683542FB
:102F200002D04468344203D10D20FEF7B7F9F8BD52
:102F30006D10192DFBD80A4F7B5D012B04D0310099
:102F4000280004F0ADFB7E55064964108C4202DC7B
:102F5000E143C9172140280004F0D6FAE7E7C0464C
:102F6000D0050020FF03000070B501240D68254244
:102F700004D10D20FEF792F9200070BD6D10192DBF
:102F800017D80024012804DD4C68043C63425C41EE
:102F90006400094E735DA34204D02100280004F0B0
:102FA0007FFB7455280004F0AFFB03000420012BC5
:102FB000E3D00020E1E7C046D005002070B5040052
:102FC0000D0019280ED8084E335C012B04D00121C6
:102FD00004F066FB01233355290020004D1EA94152
:102FE00004F07CFB70BDC046D0050020036810B51E
:102FF000DA0703D40D20FEF751F910BD41685810CF
:1030000004394A425141FFF7D9FFF6E737B569461F
:103010000A00064B30CB30C203680220042B02D1D9
:1030200000F0ACFF37BD00F0D1FFFBE714CD00008E
:1030300010B5084C237D002B05D00021142004F08E
:103040002FFB00232375142004F05EFB43425841FC
:10305000800010BDD005002010B5084CA37D002BCA
:1030600005D00021162004F01BFB0023A3751620B9
:1030700004F04AFB43425841800010BDD0050020B7
:10308000F7B5304D304E6B6C002B15D0A8240023C3
:10309000E40037596B642D4B186800280CDB2C4B6F
:1030A00019784A425141C9B2197004F017FB294BF3
:1030B0001B88DF19BFB23751AB6C002B39D0002110
:1030C000254B264FF458A9643A780C340193244DCB
:1030D0008A4206D02B68032B03D8224AD05C04F026
:1030E000FDFA2B68204A0133134004D50422013B2A
:1030F0005242134301331B4900228C462B60042BA0
:1031000018D06046C05C591CFF2802D10B00012278
:10311000F5E7002A00D02B60012104F0DFFA01233B
:103120003B702B68114A5B009B5AE418019BA4B2C8
:10313000F450F7BD01235B422B6000233B700C4B26
:10314000F3E7C046FCA0004000A0004018000020AB
:10315000EB0500200C00002044050000EA050020DB
:10316000CC0500201C000020030000800E00002081
:1031700050460000084B094AFF201A805A809A8066
:10318000DA800023064A07491370074A087048701E
:103190008870C870136070470E000020DC050000C6
:1031A000EA0500201C000020CC0500200122024B73
:1031B00052421A607047C0461800002010B5034AFA
:1031C0000421034802F0A8F810BDC0461CCD000041
:1031D000A6D40000E12170B54902144803F006FFAF
:1031E000FFF718FE0A2004F003F90023FF21104A1C
:1031F000995401331A2BFBD1012200200D4B010001
:103200001A6004230C4A0D4D1468002CFCD02C6865
:103210000002013B20431160002BF5D10122084B35
:103220001A6004F09FF801F0D3F870BDAC1B0020C9
:10323000D005002000D0004000D1004008D500405B
:1032400004D00040F8B50B4E070030000D0003F02D
:1032500015FF0400A84200DD2C003D00EB1B9C4242
:1032600005DD300003F014FF28700135F6E720007B
:10327000F8BDC046AC1B002010B50100014803F0AA
:10328000BDFE10BDAC1B002010B5054C200003F0A6
:10329000C3FEE1212000490203F0A8FE10BDC04694
:1032A000AC1B0020C3070CD4064B1B68834208D814
:1032B000054B1B68984204D8031F1B68002B00D0E5
:1032C00018007047F8050020F405002000230122B3
:1032D00010B50A48990001334250642BFAD1084CCA
:1032E000084B00211A602000074A08F001F8074B3C
:1032F000074A6360074B1A6010BDC0467C2D002052
:10330000FC05002008000020D40900003027000040
:1033100000060020F005002010B5044B044A1A6096
:10332000044B054A1A60FFF7D1FF10BDF8050020D5
:10333000FC050020F4050020D00F0020044B1B6882
:103340001868000980B20238C343DB171840704781
:10335000F005002000B59BB00200054901A808F067
:103360000BFB01A802F028FA02F072FCFCE7C04651
:10337000C6CD00000B4BC20704D4042804D80A4B66
:1033800000D00A4B180070470F2203681A40031D33
:10339000042AF7D0064B092AF4D0064B032AF1D0B1
:1033A000054BEFE7A0CD000092C900008CC90000DA
:1033B000AACD0000BACD0000B1CD00000020064A21
:1033C0000649131F186013681B099BB202339B0048
:1033D000D2188A42F5D3704700060020D00F002093
:1033E000F7B50F240126314B314A1968314B324D64
:1033F000186813681F002740072F26D813681B0979
:103400009BB202339B00D218AA42F2D300242B4E67
:10341000A500AD192868FFF745FF01342860642C2A
:10342000F6D1274C2068FFF73DFF2060254C20682F
:10343000002802D0FFF736FF20600025224B1B68D2
:103440000093009B9D4214DBF7BD1B099BB29B00C0
:10345000D3189A42D2D01F68374208D1B94206D257
:10346000B84204D3043F3F68002F00D01F60043BE4
:10347000EFE7F0236B43154A9B181A78002A01D115
:103480000135DEE71F693C2300266B43DB199B00F7
:1034900001930136BB1BF3D4019BB4001C1B0B4BE7
:1034A0001C19A069FFF7FEFEA061F2E7F8050020F5
:1034B00000060020F4050020D00F00207C2D002005
:1034C00008000020D00F0020C8050020241C002088
:1034D000F7B50124204246D1234B1B689C469842F5
:1034E00041D3224B1B68019398423CD8031F1B68B1
:1034F000002B38D10200036800941B099BB2002BFB
:103500000FD10099131F196090422CD015682B1F02
:103510001B68990069180C68013B14600A602A0056
:10352000EDE79D0055192968009C214219D18C4571
:1035300017D8019C8C4214D30E1F3468002C10D174
:103540000F680F343C40072C08D92F60151F2B60E3
:103550000B680A601B099BB20A00D0E70099316032
:10356000CDE7013BCBE7F7BDF8050020F4050020CF
:103570000D4970B50A000D4D1368141F1B0926680C
:103580009BB2981C002E0BD000238A4200D00B0067
:1035900023608300C91880001218AA42ECD370BDC2
:1035A0001B011360F7E7C04600060020D00F002083
:1035B000F8B5124C27000F223B681D09ADB213422B
:1035C0000DD06E1CB600A74204D032003900200096
:1035D00007F07BFE0022A3190436A4191A600235F5
:1035E000AD00074B7F199F42E5D31B1B9B10013B8E
:1035F0001B012360034B1C60F8BDC0460006002081
:10360000D00F0020F0050020F0B59BB0FFF714FCB0
:1036100000240700214AA300D0580134FFF758FFC7
:10362000642CF7D11E4B1868FFF752FF1D4B18682A
:10363000002801D0FFF74CFF00261B4B1B689E4261
:1036400017DBFFF795FFFFF7CBFEFFF7B1FFFFF7A3
:10365000F3FB164BC21B1B6815491B6801A81B090D
:103660009BB2023B08F088F901A802F0A5F81BB054
:10367000F0BDF02575430F4BED182B78002B01D1D1
:103680000136DAE72B695C1E002CF9DBA300EB188E
:103690009869FFF71DFF013CF6E7C0467C2D00202E
:1036A00008000020D00F0020C8050020F0050020F1
:1036B00080CD0000241C0020F7B5174D4F1C2B684F
:1036C00006001B680C001B099BB201929F420BDB9A
:1036D000FFF79AFF2B681B681B099BB29F4203DB15
:1036E0000A20FDF7DBFDFEBD2868A71CBA00DB1B26
:1036F00081181B010B6029600021031F19600F2333
:103700001E4003002401264340C3083A9A189A42F7
:10371000E9D9019902C3FAE7F0050020F7B50300E3
:103720000122134004000D000193002B2BD1174BF5
:103730001B68834227D8164B1B68834223D90F236B
:10374000144F386000681840FFF7B6FF019B3C68D3
:10375000061E3B6017D0236804301B099BB29D42B4
:1037600000DD1D00AA00211D251F07F0A5FDFFF7A4
:1037700025FE2E60FFF734FE00232B602268064BE7
:103780001340236034002000FEBDC046F805002031
:10379000F4050020D00F0020F0FF0F0003230430B9
:1037A00010B5C11719400918891000220420FFF72D
:1037B00083FF10BD70B5050008000C00FFF7EEFF99
:1037C0000023002804D170BDE95CC21811710133D7
:1037D000A342F9DBE343DB171C40002304192371E8
:1037E000F1E7F0B50C009BB0022804DC1C20FDF7CB
:1037F00055FD1BB0F0BD01230868184206D104280E
:1038000004D90F2601683140042901D00E20EEE7CB
:1038100061680D001D40F9D10429F7D90A683240CA
:10382000042AF3D1A2681A4201D10D20DFE7FFF785
:10383000A1FD06006068FFF79DFDA768010001ACCF
:103840007F103000257002F07CFF390064232200D5
:1038500002F0DCFF200008F0D5F801002000FFF79F
:10386000A9FFC6E710B51C4CA544041E02D1FFF702
:1038700095FF0BE002F07EFE0138062828D805F0FF
:1038800055FB090911182904240000208023DB00BE
:103890009D4410BD200002F0E9FE011B2000FFF74F
:1038A00089FFF3E7200002F08FFE43000120184358
:1038B000ECE780226946D200200002F09CFE6846B8
:1038C00008F0A0F801006846E9E704210348E6E7AC
:1038D0000020CCE70420D9E700FCFFFF0CCE00005D
:1038E00070B50C00022803DC1C20FDF7D7FC70BD6E
:1038F00001230868184206D1042804D90F2501685D
:103900002940042901D00E20EFE761681942FAD15D
:103910000429F8D90A682A40042AF4D1A2681A4274
:1039200001D10D20E1E7FFF725FD05006068FFF7F5
:1039300021FDA46801006410280002F002FF2100AC
:1039400002F03FFFFFF78EFFD1E770B50D000128B1
:1039500003DC1C20FDF7A2FC70BD01240868204296
:1039600006D1042804D90F2102680A40042A01D094
:103970000E20EFE76A682242FAD1042AF8D91368C8
:103980000B40042BF4D1FFF7F5FC06006868FFF745
:10399000F1FC0100300002F0D4FE02F056FF4000BE
:1039A0002043D9E7F8B507000C001C20012F0BDDE0
:1039B00001250868284206D1042804D90F2102688D
:1039C0000A40042A03D00E20FDF768FCF8BD6268A7
:1039D0002A42F8D1042AF6D913680B40042BF2D1FD
:1039E000FFF7C8FC06006068FFF7C4FC0100022F67
:1039F00014D0A4682C4211D06410300002F0A1FE53
:103A0000050002F0B7FD012811D1002C02DD0135BF
:103A1000012C06D12800FFF725FFD7E701246442D7
:103A2000EBE7280002F02EFE013C0500F0E702283B
:103A3000F0D1002CEEDD0135012CEBD00022280066
:103A4000110002F051FE02F01DFE013C0500F3E7FB
:103A500010B501240868044016D04410200005F079
:103A600097FD134905F062FC07F048FB03F090FF57
:103A70000022104B06F0FCFC03F032FF07F0CEFAF8
:103A800043000120184310BD04280CD90F230268FD
:103A90001340042B07D1FFF76DFC21000A2208F028
:103AA00079F80400DAE70D20FDF7F8FBD6E7C04609
:103AB000D30237390000D040086870B501240500F2
:103AC000254006D1042804D90F2302681340042B93
:103AD00003D00E20FDF7E2FB70BDFFF74BFC03782F
:103AE0002900233B5A4253411022C01808F052F8D3
:103AF00080239B05C218044B9A4201D91420E9E7A0
:103B000040002043E8E7C046FFFFFF3F10B5034AEF
:103B10000621034801F000FC10BDC046DCCD0000CA
:103B2000D7CD00000020704710B51E20FDF7B6FB72
:103B300010BD10B51E20FDF7B1FB10BD10B51E2045
:103B4000FDF7ACFB10BD10B51E20FDF7A7FB10BDA7
:103B500010B51E20FDF7A2FB10BD10B51E20FDF70D
:103B60009DFB10BD10B51E20FDF798FB10BD10B5D4
:103B70001E20FDF793FB10BD10B51E20FDF78EFB38
:103B800010BD10B51E20FDF789FB10BD10B51E201D
:103B9000FDF784FB10BD10B51E20FDF77FFB10BDA7
:103BA00010B51E20FDF77AFB10BD000010B5034ACA
:103BB0000E21034801F0B0FB10BDC04648CE000006
:103BC000B8CE00000120034B1860034B1B688340F4
:103BD00018437047F40F0020D40F0020F0B5EFF326
:103BE00010810123194083F31088134C134AA44613
:103BF0001268134E013A9340124F134A002B17D00C
:103C0000146803420FD03D682C60C046C046C046D1
:103C1000C046C046C046C046C0460C4C1568246825
:103C200025605B08EAE765462C6014683460F8E7B5
:103C300081F31088F0BDC046080500502000002028
:103C40000C050050E00F0020E80F0020DC0F0020E2
:103C500030B585B001AD0C220649280007F02CFBD9
:103C60000024285D01210134FFF7FEF80C2CF8D167
:103C700005B030BD77CF0000F7B56A46394B01ADCE
:103C800013800F239370384B2B800A23AB70FFF700
:103C9000D3F8364B364CC0182368984201D2002323
:103CA00023602668002E3DD16B469F5D01213800C0
:103CB000FFF7DAF801360021380003F00FFD032E7C
:103CC000F2D10026AF5D01213800FFF7CDF80136B3
:103CD0000121380003F002FD032EF3D1C820013882
:103CE000C046C046C046C046C046C046C046C046A4
:103CF000C046C046C046C046F1D100212878FFF733
:103D0000B3F868780021FFF7AFF8A8780021FFF733
:103D1000ABF8FFF791F8FA2300251B01C0182060CB
:103D20002800FEBDFFF788F8236800259842F7D3E6
:103D3000032003F063FB0600042003F05FFB36184A
:103D40000A2003F05BFB0B4B9B1B181A0A4BA84283
:103D500006DB18600023094A236013600125DFE7B2
:103D60001D60F7E70D0E000003040000102700009F
:103D7000EC0F0020E3030000D40F0020F40F00201C
:103D80000022054B10B51A60044B1B68934201D00A
:103D900002F090FB002010BDF00F0020D01A002090
:103DA00010B5041E10DA1A240A4BA400E2580123AD
:103DB0009340094A09491360094A1160094A0A49AE
:103DC00011600A4A136010BDFFF74CF8A042EADD0B
:103DD000EAE7C04660DC0000E80F0020080500505C
:103DE000E00F0020DC0F00200C05005018050050EB
:103DF0002B4BF7B51B680C00002B03D10120404270
:103E0000FFF7CEFF24680126250035401AD0FF2297
:103E10006310120260121040DAB21043FF221B023C
:103E20001204134018431F4B1B68202B06D1B440CB
:103E30001D4BA40EA400E35800021843FFF7CEFE6A
:103E40000020FEBD042CFBD90F2322681340092B50
:103E5000F6D1FF2763683F025B100193019B9D42EF
:103E6000EEDAAB00E3189B68334216D05A105812B2
:103E7000D1B238400843FF21120209040A4010431E
:103E8000084A1268202A06D15B009B0E06499B0057
:103E9000020258581043FFF7A1FE0135DEE7C04685
:103EA000E80F00202000002060D100000200086818
:103EB00010B5C3070FD540101823012A03DD4A6847
:103EC000042A00D10833054A1360FEF7EDFFFFF71F
:103ED00067FF002010BD01204042EDE720000020D8
:103EE00010B50124044002D04410200010BD042865
:103EF0000CD90F2302681340042B07D1FFF73AFABD
:103F000021000A2207F046FE0400EEE70D20FDF72F
:103F1000C5F9EAE70868F8B5C3071AD5FFF7E0FF67
:103F20000300203B5E2B25D80520434301221D18AA
:103F30000020114E9D4219D005211024F75C3C420F
:103F400000D080180139520064100029F7D10133E4
:103F5000F0E704280ED90F2203681A40042A09D179
:103F60001B099BB2002B05D00379DAE7012340003F
:103F70001843F8BD0120FCE783CF000070B5086846
:103F80000D00FFF7ADFF04006868FFF7A9FF621E90
:103F90000100042A14D8451E042D11D805236B43B3
:103FA0009B18012215009D402B00064805682B43F5
:103FB0000360054B1B68002B02D0200002F07BFA47
:103FC000002070BDF00F0020D01A002070B50868E6
:103FD0000D00FFF785FF04006868FFF781FF621E90
:103FE0000100042A13D8451E042D10D805236B4365
:103FF0009B1801229A400748036893430360064BCD
:104000001B68002B03D00022200002F054FA00208D
:1040100070BDC046F00F0020D01A0020F0B505009A
:1040200089B008680C00FFF75BFF0690022D36DDB3
:104030006068FFF755FF0190A068FFF751FF04008B
:104040000127231D661E0793731C0293079B9E4244
:1040500035D0052373430593019B019D05330493DC
:10406000049BAB421ED0042E16D86B1E042B13D813
:104070000122059B2349013B5B199A409446224A41
:104080000B681068069A3A4003920DD062461A43B4
:104090000A60012200280DD17F000135E0E70124EC
:1040A0000194CDE7029ECFE7624693430B60002860
:1040B000F2D0039A0299280002F0FDF9ECE7019B87
:1040C0001E1D042E1AD8012C18D1002505273B00EF
:1040D00021006B439B1999400B000A4A0135116876
:1040E0009943094B11601B68002B05D0019B0022EE
:1040F000581D290002F0DFF9052DE8D1002009B094
:10410000F0BDC046F00F0020D01A0020086810B59E
:10411000C30703D5FFF7E4FE054B1860054B1B688A
:10412000002B03D0024B186802F0C6F9002010BD26
:10413000F00F0020D01A00207FB5A04C2368002B80
:104140000AD19F4A1268002A06D19E4B1B68002B99
:1041500001D0FFF791FD7FBD9B4D2A68002A26D133
:10416000984A1268002A1BD0FFF786FD0028F2D07B
:10417000FFF76EFD924B24681A681C60002A16D067
:10418000002C14D101AD0C229049280007F094F8BE
:10419000285D00210134FEF767FE0C2CF8D1DAE728
:1041A000874A1268002AE5D1002BE3D0E0E700211E
:1041B0000D2003F093FA00210E2003F08FFA002166
:1041C0000F2003F08BFA2E68012E5DD0022E00D155
:1041D000A2E0002E51D101363100794C0420236831
:1041E000994303F07BFA04212368052019404B42D0
:1041F000594103F073FA10212368062019404B42FD
:10420000594103F06BFA80212368090119404B42A0
:1042100059410C2003F062FA8021236809021940F9
:104220004B4259410B2003F059FA8021236849027F
:1042300019404B4259410A2003F050FA802123686B
:10424000890219404B425941092003F047FA802165
:104250002368C90219404B425941082003F03EFA35
:10426000802321681B0319404B425941072003F06A
:1042700035FA31000D2003F031FA2B680321581C68
:1042800004F0D8FF296066E702214D4C072023681F
:1042900019404B42594103F021FA0820216801409E
:1042A0004B42594103F01AFA80212368C900194092
:1042B0004B425941052003F011FA8021236849013E
:1042C00019404B425941062003F008FA8021236827
:1042D000C90119404B425941042003F0FFF98021E4
:1042E0002368890319404B4259410A2003F0F6F92B
:1042F000802321681B0419404B425941092003F0D7
:10430000EDF931000C2003F0E9F931000B2003F046
:10431000E5F931000E20AEE72021294C0720236863
:1043200019404B42594103F0D9F940212368082034
:1043300019404B42594103F0D1F9802123680920EB
:1043400019404B42594103F0C9F9802123684900C3
:1043500019404B4259410A2003F0C0F980212368DB
:10436000890019404B4259410B2003F0B7F98021D5
:104370002368890119404B4259410C2003F0AEF9E2
:1043800080212368490319404B425941062003F01C
:10439000A5F980212368C90319404B4259410420E3
:1043A00003F09CF9802321685B0419404B4259417A
:1043B000052003F093F901210F205CE7F00F0020A6
:1043C000E40F0020F40F0020D80F002077CF00006A
:1043D000012010B54042FFF7E3FC0020FFF7FEFB91
:1043E00010BD000010B5034A0921034800F094FFF6
:1043F00010BDC04660D20000A8D2000030B5022433
:104400008025094B094AED009C505C59002CFCD0DA
:10441000A124E400884202D30021995030BD8025B8
:10442000ED0018514019F5E700E0014004050000D7
:1044300010B5002806D1C020B02140028902FFF744
:10444000DDFF10BDB02080218002C902F7E7000027
:1044500043425841064B40421840B0239B02C018CB
:10446000036800201A0E532A01D11B02180A704754
:1044700000C0FEFF30B501248025054B054AED0044
:104480009C505C59002CFCD001600021995030BD3B
:1044900000E001400405000043425841074B404200
:1044A0001840B0239B02C018A62310B50902DB05F3
:1044B000090A1943FFF7DEFF10BDC04600C0FEFF2A
:1044C00070B5012480250D4B0D4EED009C515C59BB
:1044D000002CFCD0002902DC00229A5170BD5578D6
:1044E00014782D0225439478013924042543D47887
:1044F000043224062C4310C0ECE7C04600E0014023
:104500000405000070B505004B680A009C1C2100E2
:10451000A400FFF7D5FF281970BD0000134B1B68DE
:10452000002B0CD08022B023D2029B0200280BD19A
:104530001A1D5B681B0E522B00D110007047B02271
:10454000C02392025B02F1E782420DD903681B0E81
:10455000522B09D1436802339B00C018824203D911
:1045600003681B0E522BE9D00020E7E7F81000206B
:10457000F0B50020B7B00024FFF7D0FF27000500FA
:104580002600002D2ED1284D2868FFF761FF32004C
:104590003B0001900094254904A807F0EDF904A818
:1045A00001F00AF9224B64201C682B68A0215A42B2
:1045B0005341204A5B421340B02292029B18E41AF6
:1045C0006043490204F050FDA02252020300009211
:1045D0001949220004A807F0CFF904A801F0ECF86B
:1045E00037B0F0BDFF226B6829689C460233FF1884
:1045F0000B12013613409C4200DA1C00FF200A1403
:10460000024003926246014001920091039A0B49D5
:1046100004A807F0B1F904A801F0CEF82800FFF7CC
:104620007DFF0500ADE7C046F8100020B2D30000C2
:10463000FC10002000C0FEFF5CD300009ED30000F1
:1046400070B50020FFF704FF04000120FFF700FF12
:10465000844200DA04000A4B1D686A425541280072
:104660001D60FFF7E5FEA0226B4252021340054A8F
:1046700028009B18044A611C1360FFF70DFF70BDF2
:10468000F810002004800100FC100020F8B5002084
:10469000FFF7DEFE07000120FFF7DAFE3E00204DA7
:1046A0000643204C0DD18021C020C9024002FFF7F3
:1046B000A5FE01213000FFF7EFFE1B4B2E602360AB
:1046C0001DE0874209DD0023B0212B60164B8902D3
:1046D000236023680020012517E0012380212B603F
:1046E000124BC9022360F4E7120E522A08D00028A8
:1046F00000D023600E4801F05FF8FFF7A1FFF8BD7E
:1047000028005A68023292009B188B4205D21A6820
:10471000561CE9D10028F2D0D1E72160EFE7C0466E
:10472000F8100020FC1000200480010004C00200EA
:1047300077D3000070B50020FFF7F0FEFF260500DC
:10474000002801D1280070BD03681C143440FFF715
:10475000E5FEDA2CF4D10500F2E700008022F0B586
:104760005200A1B00021674806F0C2FD802200215E
:104770005200654806F0BCFD644BFF271B681A0019
:10478000049353425A4110000592FFF751FE049CD6
:104790000020631E9C415E4B64421C405D4BE4184C
:1047A000FFF7C8FF0600002E2DD10498FFF750FE3A
:1047B000411C0598FFF770FE059A574D534B2C602E
:1047C0001A60FEF761FD514B64201B68A0215A421C
:1047D00053414F4A5B421340B0222C6892029B180F
:1047E000E41A6043490204F03FFCA0225202030095
:1047F00000924A49220007A807F0BEF807A800F077
:10480000DBFF21B0F0BD3268131412123A403B4076
:1048100003921A000A3A092A49D83A4B039A995C3A
:10482000002931D110223E4806F062FD35002B6888
:1048300003991A123A40914209D11A143A400B2AAC
:1048400027D0132A2DD00A2A01D1354B1D6028000C
:10485000FFF764FE051EEAD1314B196800290FD01D
:104860002000FFF74FFE04002D4B5B19596800290B
:1048700003D02000FFF746FE040004350C2DF3D1D1
:10488000204B0121039A99543000FFF747FE0600A0
:1048900089E73B40022BDADC214A9B00D3185D609C
:1048A000D5E7102200211E4806F022FDCFE71A00AE
:1048B000153A082AE8D8144A0399525C002AE3D131
:1048C0003500152B00D01500300003681A143A404B
:1048D000152A0FD01D2A00D10025FFF71FFE002842
:1048E000F3D1002D04D020002900FFF70BFE0400B7
:1048F000054BC6E7039A1B123B409A42EDD10500D7
:10490000EBE7C046F80F002000110020F81000204F
:1049100000C0FEFF04C00200FC10002041D30000D4
:104920000C2F002010B5FFF719FF10BDF0B585B0B2
:10493000039203220333DC17294D1440E4182B683B
:10494000284F5A42534180225B42D202A4103B407E
:104950009B18A21C0291244E910000910190316895
:1049600000980A18934215D2FFF7F8FE2B685A42B6
:10497000534180225B421F40D202BF183368009A25
:104980009B189F4206D2194800F016FF0025280008
:1049900005B0F0BD029B356819066B461A7BA4234F
:1049A000DB051343FF222F00090C1943019B12045E
:1049B0001B04134019432800FFF75CFD0837281D2E
:1049C00021003760FFF756FD002C04D00A9A210021
:1049D0003800FFF775FD009B083BFF183760D6E7EE
:1049E000F810002000C0FEFFFC1000201BD30000C8
:1049F00070B59AB0FFF74AFEFF221E4CD20000218C
:104A0000200006F075FCFF25FFF794FE0026002825
:104A100014D10200C300E3580130591E8B41D21853
:104A2000FF28F7D1144901A806F0A6FF01A800F05D
:104A3000C3FE124800F0C0FE1AB070BD03681A141D
:104A40002A400A2A0AD11A122A40FF2A03D0D20089
:104A5000A1180B71A050FFF761FDD8E7132AFAD116
:104A60001B122B40FF2BF6D0DB00E2181671E6502C
:104A7000F1E7C04684250020E7D30000FBD3000007
:104A80000021094B094A59600131516059680029D8
:104A9000FCD000211961012393600222044B813173
:104AA000FF315A501A607047FC100040001000405F
:104AB00000E100E00222064B0121DA670022054BEB
:104AC0005A61054A11615A69002AFCD07047C046F4
:104AD00004E100E0FC1000400010004010B5044C60
:104AE0002378002B01D0FFF7E5FF0020207010BDD8
:104AF00001120020802301205B055B6E5B001843E0
:104B0000704700000120024B1B685B001843704790
:104B1000841200200120024B1B685B001843704781
:104B2000240000200120024B1B685B0018437047E3
:104B30008812002070B504000D001600FEF786F9FB
:104B4000802301215B055A6E267000265300617098
:104B5000E1706272010A5A0A6071A171A272010CBD
:104B60005A0C000E5B0EA6702571E1712072E27284
:104B7000237370BD10B5044C200006F043FF010004
:104B80002000FEF717FE10BD8D1200200E4B10B551
:104B90001B680E4C5A1C0FD00D4C002B0CD00D4C2A
:104BA000012B09D00C4C022B06D0094C042B03D04E
:104BB0000A4C052B00D1074C200006F023FF010012
:104BC0002000FEF7F7FD10BD280000208CD4000067
:104BD00001CD000097D4000008CD000091D4000062
:104BE00070B5214C2278002A3DD1204B01215A601A
:104BF0008022D20511605A68002AFCD000220720CA
:104C00001B4B1C4901255A500439585008315A5041
:104C100019481A4958501A491A485A501A495A50AC
:104C2000A622D2009D50082218495A5004315850EB
:104C30000220174958501749174858501748043947
:104C40005850182016495850C12189005A5005392A
:104C5000FF395858921802435A501249124A995033
:104C6000FFF70EFF257070BD01120020FC00004010
:104C7000001000400C050000746962751C050000FE
:104C800024050000200004022C050000140500008B
:104C9000340500003C050000FFFF0000211001006A
:104CA00054050000021200200405000070B50E4BF0
:104CB00006001B78002B01D1FFF792FF00200B4D5F
:104CC0002C7884420ED00A4B202219780323091B2A
:104CD0001940084B4901C918300006F0EDFA0120CF
:104CE000013C2C7070BDC046011200208C120020C7
:104CF0000012002002120020002370B588B09842F4
:104D000035DD0D6801262C0034409C422FD1230054
:104D1000042D2CD90F222B681A402300092A26D1F2
:104D20006A683F2A23DD6846FFF7C0FF230000289A
:104D30001DD06B4619783300A14203DB6B461B5D27
:104D40005B003343A200AA1801349360202CF2D1F7
:104D5000092169444A780B7812021A438B781B04A4
:104D60001A43CB781B061343024A1360042318002E
:104D700008B070BD8812002070B5454B8AB01B7812
:104D8000002B01D1FFF72CFF02AC2000FFF78EFFB4
:104D9000002802D100200AB070BD23780B2BF9D96E
:104DA0006378012BF6D1E378012BF3D10023112096
:104DB000384E394D33602B7068442379374A417837
:104DC0001360027809021143827812041143C278F9
:104DD00012060A4332490A60002B0ED1152169449C
:104DE0004A780B7812021A438B781B041A43CB784B
:104DF0001B0613433360002318E0012B1AD1152141
:104E000069444A780B7812021A438B781B041A43C0
:104E1000CB781A211B06134333600E23627C69444E
:104E2000934200DD130000229A422CD1002204207C
:104E3000EA54B0E7022B03D1627B10331621EEE770
:104E4000042B0DD1152108226944684606F034FA76
:104E50000098019902F0B4FC06F0E0F83060CAE76F
:104E6000052BC8D1152108226944684606F024FAAA
:104E70000098019902F0A4FC06F0D0F83060627D41
:104E80000A231E21CBE7885CA8540132CCE7C04638
:104E900001120020841200208D1200202800002022
:104EA0008812002010B5134B04001B78002B01D191
:104EB000FFF796FEFFF7FEFD00200F4A0F49104B4B
:104EC000545058600130106058680028FCD0002011
:104ED00018610130906018690028FCD0094B0A481D
:104EE0001B785B011B185350FFF7E4FDFFF7C8FD6B
:104EF00010BDC04601120020001000400405000053
:104F0000FC100040001200200212002010B588B0F2
:104F100000281DDD0A68012113000B4018D1042A66
:104F200016D90F2014682040092811D150683F2855
:104F30000EDD9800101880680024084201D040104F
:104F4000C4B26846C4540133202BF2D1FFF7AAFF44
:104F5000002008B010BD000010B5002813DD0C685B
:104F6000E30710D56410532C0DD8084B1B78002B89
:104F700001D1FFF735FEFFF79DFDA123044ADB00B9
:104F8000D450FFF77DFD002010BDC0460112002067
:104F90000010004010B500280EDD0C68E3070BD5AB
:104FA0006410FF2C08D8054B1B78002B01D1FFF7AC
:104FB00017FE034A034BD450002010BD01120020FD
:104FC000001000402405000013B5002814DD0C6813
:104FD000E30711D5094B64100093094B0193072C8B
:104FE0000AD8084B1B78002B01D1FFF7F9FD6B465F
:104FF000054A1957054BD150002016BDE2ECF0F4DC
:10500000F8FC000401120020001000400C05000014
:1050100070B588B0002820DD0124086804401CD148
:1050200004281AD90F2302681340042B15D1FEF768
:10503000A1F9060006F0E6FC0500122800D91225A9
:105040002A0002210D326846FFF774FD6B465D733E
:10505000A54205DC6846FFF725FF002008B070BDBB
:105060002300325D6B449A730134F1E7F0B50D0013
:105070008BB0012832DD08680122040014402DD1D4
:1050800004282BD90F2301680B40042B26D16B6811
:10509000134223D0FEF76EF96E6807007310019378
:1050A00006F0B0FC05000E2800D90E252A000121CB
:1050B000113202A8FFF73EFD6A46127902AB5A731D
:1050C00002AA73129373019B76141B0ED67313748A
:1050D0005574A54205DC02A8FFF7E4FE00200BB0E2
:1050E000F0BD3A5D02A963189A740134F1E730B556
:1050F00089B0002814DD0C68E30711D5102268463A
:105100000021FFF717FD6B466A4665105D73684620
:1051100063122D0E64149373D4731574FFF7C2FEDB
:10512000002009B030BD0000174B184A596800290B
:1051300003D00021596001319160196900291FD005
:10514000002018618023DB00D3581149012B18D1AE
:10515000A923DB00D3585B420B600E490B78032B6D
:1051600001D801330B7003200B490B780133034046
:105170000B700A495B015B18094953500123936086
:1051800070470860FAE7C046FC100040001000407D
:10519000240000208C1200200012002002120020A7
:1051A0000405000010B5034A1021034800F0B4F8CC
:1051B00010BDC0460CD4000003D40000044A0549C9
:1051C0001368C85401339B059B0D13607047C0469C
:1051D000BC160020BC12002070B5114C114A236887
:1051E000834202DC0023236016E0155C411C2E0084
:1051F000FA3E012E05D899420FDA555C013D1F2D6C
:1052000001D90800ECE70100151A565C6E54013113
:105210008B42FADC181A206070BD1570FAE7C046A0
:10522000C81A0020C816002010B5FDF705FE064B71
:105230001A68824201D900221A601B68C31A034807
:1052400098428041404210BDB8120020204E00001C
:1052500010B5094C094A23681268934200D110BD69
:10526000074AD05CFEF708F80028F8D0236801331D
:105270009B059B0D2360ECE7C0160020BC160020A8
:10528000BC12002010B50400064B074A1B681268C8
:105290009B1ADB439B059B0DA34200DB10BDFFF770
:1052A000D7FFF1E7BC160020C0160020F7B50500B7
:1052B00056680191B000441C06301700FFF7E2FF6A
:1052C000FB20FFF77BFF1C20FFF778FFE8B2FFF71A
:1052D00075FFE0B22412FFF771FFE0B2FFF76EFF37
:1052E0006B461879FFF76AFF0025AE4200DCF7BD78
:1052F000AB00FB189C680135E0B2FFF75FFF20129E
:10530000C0B2FFF75BFF2014C0B2FFF757FF200EBB
:10531000FFF754FFE9E7000070B5074E33680B2B29
:1053200008DC0C255D43054C01332851641961608C
:10533000A260336070BDC046C41600201C2F002040
:10534000F0B587B002900C00012803DC1B20FBF7AE
:10535000A5FF45E0244B08680093C30709D404283F
:1053600007D90F2302681340042B02D1FEF702F87D
:1053700000901D4B60680193C30709D4042807D926
:105380000F2302681340042B02D1FDF7F3FF0190B5
:105390000027164B1B680493049BBB42D6DD0C26EA
:1053A0007E43134B0099F618306806F021FB051E6A
:1053B00005D17368B6680593059B9D4201DB0137F3
:1053C000EAE730680199039606F012FB08360028D8
:1053D00008D121000298039B083102385B68984786
:1053E00007B0F0BD0135E7E7D6CD0000C4160020B8
:1053F0001C2F002010B5FBF769FEFEF7F3FFFBF74B
:1054000087FEFDF7DBFEFEF781FBFEF7CFFBFFF724
:10541000C9FE00F093FE01F051F801F09BFA10BDB7
:10542000962210B512010021034805F061FF002209
:10543000024B1A6010BDC046241C0020C805002085
:10544000064B074A1B6812689B1ADB439B059B0DA2
:105450000122834200DC002210007047BC160020AD
:10546000C0160020F8B505000C0016001F1E0ED156
:105470000320FFF7E5FF002808D0FA20FFF79EFE83
:10548000E8B2FFF79BFEE0B2FFF798FEF8BD501DB3
:10549000FFF7D6FF0028F9D0FB20FFF78FFEE8B218
:1054A000FFF78CFEE0B2FFF789FEF0B2FFF786FE51
:1054B0003012C0B2FFF782FE3C00E31B9E42E5DDE6
:1054C0002078FFF77BFE0134F7E7000070B5002479
:1054D000F0250B4B1B68A34202DCFFF7A1FF70BD58
:1054E0002B006343074A9B181A78002A05D0597885
:1054F000002311201A00FFF7B5FF0134E9E7C04689
:10550000C8050020241C0020F8B507000024F02561
:105510002B0063430C4A01349E18B74211D03178F6
:1055200000290BD00133D15C002311201A00FFF7B2
:1055300099FF2A000021300005F0DAFE0A2CE7D19D
:10554000F8BD024B1C60F9E7241C0020C8050020B0
:10555000F0B5150001222F00754C1740A5440190AD
:105560000291002F11D005AB1A706A105A70120EFA
:105570001A710522691299706D140299DD70FFF796
:1055800071FFCF239B009D44F0BD042D1ED90F2039
:105590002A681040042826D1022304AA2800137187
:1055A000FDF7E8FE040006F02DFA624B984200D9A0
:1055B0001800B84204DC421C05AB02990198DEE7F2
:1055C00001377B1EE35C05AAD355F2E7042D00D01A
:1055D000A9E0032304AA043D13716B425D4105ABAE
:1055E00055710222E9E709287ED1042205AB1A7021
:1055F0006A68511000916946521209789A70009AAF
:1056000059701F2A01DD202200926A46127806ACEA
:10561000DA70009BBB4202DC05ABE21ACDE7012643
:10562000BB00EB189868064006D1042837D90F2133
:105630000368194002290CD10123237043106370C1
:1056400042121B0E4014A270E07023710534013722
:10565000DFE7042921D102232370FDF78BFE03909D
:1056600006F0D0F9A31C0C2809D86070864201D13D
:105670009C19ECE7039A925D9A550136F6E70C22E5
:105680006270039A925D9A550136092EF9D12E2344
:10569000E372237363730E34D9E7012907D103231F
:1056A000043823704342584160700234CFE709291F
:1056B00009D10423237043685A1062705B12A370EF
:1056C000E6700434C3E703290BD105232370006877
:1056D000020992B2430F92000B40D31A63701B125F
:1056E000EDE726700134B2E7032800D049E7052131
:1056F00005AB1970110989B2520F890002408A1A4C
:10570000111299705A701100642A00DD642104207E
:10571000D970C9B2041FA14201DC04324DE72C5CF0
:105720001C540130F6E7002D00D02AE751E7C046AF
:10573000C4FCFFFF2303000070B502000024F02129
:105740000D4E0800604380194578954203D001341E
:105750000A2CF6D170BDF022002105F0C9FD074AE0
:105760001368013BA34200D11460002329001A00F2
:105770001120FFF777FEEDE7241C0020C80500206C
:1057800010B5B2B002236A460400137006F03AF96D
:10579000C72800D9C7200023984207DC421C6B466B
:1057A000FE211420FFF75EFE32B010BD69460133C2
:1057B0005A1EA25CCA54EFE730B5B3B002236A4662
:1057C0000500137006F01EF90400C72800D9C7248D
:1057D00000239C420BDC20003230FFF753FD621C9B
:1057E0006B46FF211420FFF73DFE33B030BD694604
:1057F00001335A1EAA5CCA54EBE70000F7B5234BED
:1058000006001B68F02100930023009A9A4211DCE5
:105810000024F0231A006243019201991C4A551892
:105820002F78002F12D001340A2CF3D11948FFF73A
:10583000C3FF29E00A005A43154882185078B04245
:1058400002D11278002A1FD10133DEE7F02239009D
:10585000280005F04DFD02230D4A0199EB605354D9
:105860000D4AF1008A58009B6E70AE70AA602F61DD
:105870006F61A34202DC054B01341C600023310040
:105880001A001020FFF7EEFDF7BDC046C805002046
:10589000241C002095D900008425002010B5FFF7B6
:1058A00015FEFF24084AE3005B429B18074AD35CBD
:1058B000043B012B03D8E043C0B2FFF79FFF013C3C
:1058C000002CEFD110BDC046FC070000842500204D
:1058D000F7B50F00FF247F2501901E4AE300D31A7D
:1058E0001D4A9A181278062A01D0032A20D1FF22D5
:1058F000D2009B18186883682B401C2B18D1C368F2
:105900001A002A40042A13D102692A40192A0FD109
:105910001B0A01339B000C30C018FDF72BFD0378E8
:105920000600002B10D006F06DF80023B84209D015
:10593000013C002CD1D1F7BD019AF15CD25C9142BF
:10594000F6D101339F42F7DCE043C0B2FFF756FFC8
:10595000EEE7C04684250020FC07000070B5050076
:10596000FF24084AE3005B429B18074AD35CAB4222
:1059700003D1E043C0B2FFF741FF013C002CF0D15E
:1059800070BDC046FC07000084250020F7B5FDF778
:1059900053FA514B1A68824201D900221A601A68E0
:1059A0004E49821A8A4200D883E01860FDF74EFA09
:1059B000071E00D101370020FDF73AFB01900020BF
:1059C000FDF74AFB019B0090454C464D002B14D03F
:1059D0002368002B00D07AE02B682760002B00D1D1
:1059E00071E0414B01261B78002B63D10920FFF7A2
:1059F000B5FF3E4B1E703C4B1E70009B002B12D01F
:105A00002B68002B0FD123682F60002B1ED0374B43
:105A100001261B78002B52D10920FFF79FFF334B43
:105A20001E70314B1E702368002B0FD02F4E327822
:105A3000002A0BD19F4200D227602368FB1A312B2A
:105A400004D90720FFF78AFF012333702B68002B4E
:105A50000FD0254E3278002A0BD1BB4200D92F60DF
:105A60002B68FF1A312F04D90820FFF777FF012395
:105A700033702368002B0CD0019B002B09D11B4EE7
:105A80003378002B02D10720FFF768FF0023236043
:105A900033702B68002B0CD0009B002B09D1124CCB
:105AA0002378002B02D10820FFF758FF00232B603A
:105AB0002370F7BD0720FFF751FF0C4B9CE7082030
:105AC000FFF74CFFADE7009B002B9CD1ABE7009AA2
:105AD000002A95D1AAE7C046B41200200F27000083
:105AE000A4120020AC120020B0120020A812002046
:105AF00037B500240500FFF7E9FC01A80194FDF784
:105B000085FA21002000FEF73BF9FEF715FBFDF7B3
:105B100031FBFDF74BFBFEF75BFCFDF7B3F9A5424C
:105B200004D0FDF7D3FB0248FFF746FE37BDC04661
:105B300086D90000002310B501001A001120FFF7DC
:105B400091FC10BD07B56B46197069465A70131267
:105B50008B701314120ECB700A716B460100052274
:105B60001320FFF77FFC07BD10B50A0001001220CB
:105B7000FFF7EEFC10BD70B5050008000C003230D8
:105B8000FFF780FB2B00220000211B20FFF76AFC9F
:105B900070BD10B50C000300110014202200FFF7A7
:105BA00061FC10BD012370B5FF24084A41185B4217
:105BB000884201D3D84370BD06781D0A2340734044
:105BC0009B009B5801306B40F2E7C04668D500004F
:105BD000002313B501930B4BC2000400D0580028DA
:105BE00005D0436808309900FFF7DCFF01900920D9
:105BF000FFF748FB01AB042221001720FFF732FC1E
:105C000013BDC04684250020F7B50190FEF792FD34
:105C100001250400FF276D42002C01D12800FEBDA4
:105C2000266833143B40152B0DD121000198083113
:105C300005F0DEFE002801D135123D402000FEF7C0
:105C40006DFC0400E8E71D2BF8D101256D42F5E756
:105C5000F0B580279DB0FFF7FBFAA54CA54D206855
:105C6000FF00391A4019FDF7EDFA23680600C31842
:105C70002360002B0ED11DB0F0BD2068391A281802
:105C8000FDF7E0FA236806001B182360FDF7D4F83F
:105C9000994B1860002EF0DC2B78FA2B00D037E1FE
:105CA0002368022B07DCFFF7BFFA0028E3D00120AE
:105CB000FFF792FADFE76878AC78023818282BD81B
:105CC00003F03EF919002C0030003400370040008A
:105CD0002A004A007C0086008A00A000F100020130
:105CE0002A002A002A002A002A002A002A002A0064
:105CF0002A002A001001FF2C0ED02000FFF71CFD07
:105D000000227E4BE100CA505B181A7121000092FC
:105D100013001320FEF70AFE0320C9E72000FFF757
:105D20006DFDF9E72000FFF707FDF5E7FFF7B6FD8A
:105D3000F2E7FFF7CBFB0020FFF7DAFE7048FFF732
:105D40003BFDE9E7632CE7D86E4BA200D258210057
:105D50001520FFF7FDFBDFE7FEF7ECFCFF27040053
:105D6000002CD9D025682B143B40152B04D02000E3
:105D7000FEF7D4FB0400F3E72000083005F042FEF4
:105D800006000530FFF77EFAFB20FFF717FA2D1209
:105D90001D20FFF713FAE8B2FFF710FAF0B2FFF791
:105DA0000DFA3012C0B2FFF709FA25002B1B9E42F4
:105DB000DDDD287AFFF702FA0135F7E700211D2023
:105DC00000910B000A00FEF7B1FDFDF77FFAA3E793
:105DD0002000FFF7FDFE9FE7FDF740F803AC4A4ABD
:105DE00064210090494B200005F094FD022320001F
:105DF000237005F007FE2300020000211620FFF7A4
:105E000031FB89E700243D4AE300D558002D27D017
:105E10006B689E00701DFFF735FA2B0000253200DD
:105E2000083321000120FFF71DFB2F00FEF782FC45
:105E30002E00002818D1002F04D03A0001212000A4
:105E4000FFF734FA002D04D02A0002212000FFF7CA
:105E50002DFA002E04D0320000212000FFF726FA90
:105E60000134FF2CCFD157E7FF2103681A120A40F3
:105E7000A24209D11A140A400B2A08D10B400CD0B7
:105E8000012B0CD0022B0CD0FEF748FBD1E7132AD4
:105E9000FAD100252F002E00F6E70600F4E70700F0
:105EA000F2E70500F0E70024FFF710FB22002100D5
:105EB00000942300DA20FEF739FDFF222100D200F2
:105EC0000E4805F015FA80E7012C02D1FEF750FBD1
:105ED00022E7022C02D1FEF725FD1DE70120FFF786
:105EE00007FE19E7002321001A001A2087E7C046A1
:105EF000C81A0020C8160020B812002084250020EF
:105F000068D900007C2D00207FD900007AD90000DC
:105F1000FB2B00D0CBE62268042A00DCC3E62E79F6
:105F2000E878574B360206439E4200DDBFE6331D3C
:105F30009A4200DCB7E6EB5CFE2B00D0B7E66B784C
:105F4000AC78771E1B2B61D019D8072B47D0082BB4
:105F50001CD0012B18D1FF2C16D02000FFF7ECFB32
:105F60006D79484AB31E009221002A000A20FEF7EC
:105F7000DDFC454BE400E0501B191D7104E01D2BB6
:105F800056D048D31E2B6AD0701D91E6632CFBD8E7
:105F90006A79022A13D0032A1BD0012AF4D1E979A5
:105FA000AB79090219432B7AA4001B0419436B7ABD
:105FB0001B060B435B001343344AA350E4E7002F56
:105FC000E2DDB11E2F48FDF7F5FB304BA400E05099
:105FD000DAE7AB79A4005A1E93419B00ECE7632FEC
:105FE000D2DC03AD3A002A49280005F065F9002308
:105FF0002800EB55FFF708FE0028C5DB234B800087
:10600000C25821001520FFF7A3FABDE73900204848
:10601000FFF75EFCB8E7FF2CB6D06A79022AB3D846
:1060200018490B2000912100B31EFEF77FFCABE75F
:10603000632F00DD6327002303A99F420ADCFB4393
:106040000022DB173B40CB181A70152000917B1CF7
:106050002100EAE7EA185279CA540133EDE7012C2E
:1060600092D1002F90DD6B79002B03D01C00322BD6
:1060700000DD322464235C43064B1C6084E7C04689
:10608000F6030000CE160020842500207C2D002081
:10609000CD160020040000200120704710B5064CEA
:1060A000200000F08DFD0549200000F0B1FD012227
:1060B000034B1A6010BDC046F41A0020801A060077
:1060C000CC1A002010B501210D20FCF7CDFE0121D6
:1060D0000E20FCF7C9FE00210F20FCF7C5FE044C82
:1060E000200000F0A9FC1021200000F0C1FC10BD30
:1060F000D41A002010B504680D20E30703D56410FE
:10610000FF2C03D91720FBF7C9F810BDFFF7DAFF02
:10611000E1B2024800F0CEFC0020F6E7D41A0020DD
:1061200010B5FFF7CFFF0021034800F0C3FC430088
:106130000120184310BDC046D41A002010B5034AF0
:1061400008210348FFF7E8F810BDC046ACD90000AD
:10615000ECD90000F8B5012306681E4205D0456859
:106160001D4202D084681C4203D10D20FBF796F833
:10617000F8BD76101520802EF8D86D101620FF2D52
:10618000F4D86410FF2C01D91720EFE70B4B1B68E4
:10619000002B01D1FFF782FF094FF1B2380000F068
:1061A000CEFDE9B2380000F0D1FCE1B2380000F0D9
:1061B000CDFC380000F02EFE0020D9E7CC1A0020DC
:1061C000F41A0020F7B501221400904222DD0D6878
:1061D0002A421FD01D4B15411B684C68002B01D172
:1061E000FFF75CFFE9B201272500194E3D40300062
:1061F00000F0A5FD002D0FD03C413000E1B200F0D1
:10620000A5FC300000F006FE0024A04202D02320AE
:10621000FBF744F82000FEBD042CF2D90F232268BE
:106220001340092BEDD163685B100193019BAB42D6
:10623000E7DDAB00E3189968394204D04910C9B2D0
:10624000300000F083FC0135F0E7C046CC1A002096
:10625000F41A0020144B70B51B6805000E00002BCB
:1062600001D1FFF71BFF114CEDB22900200000F017
:1062700066FDF1B2200000F069FC0021200000F072
:1062800069FD002801D0404270BD01222900200094
:1062900000F050FD200000F04AFC0028FAD0200059
:1062A00000F04AFCF0E7C046CC1A0020F41A0020A7
:1062B00010B501240368234202D04168214203D172
:1062C0000D20FAF7EBFF10BD5810802801D91520DA
:1062D000F7E74910FF2901D91620F2E7FFF7BAFFC7
:1062E00040002043EFE710B50400012814D1052138
:1062F0001820FFF7AFFF7F282BDC03007F3301DA84
:106300007F20404264235B4258437F2102F0ACFE71
:10631000052C00D1404210BD032811D101001820E6
:10632000FFF798FF7F2814DC03007F3301DA7F201A
:10633000404264235B4258437F2102F095FEEAE726
:106340000020052CF5D107211830FFF783FF7F28A7
:1063500002DD0138FF38D0E703007F3301DA7F2008
:10636000404264235B4258437F2102F07DFED1E727
:1063700070B50120FFF7B7FF04000320FFF7B3FF5C
:1063800005000520FFF7AFFF6D43644340436419E8
:10639000201804F079FE01F043FB04F03FFE4300B7
:1063A0000120184370BD10B50120FFF79CFF43008A
:1063B0000120184310BD10B50320FFF794FF4300E0
:1063C0000120184310BD10B50520FFF78CFF4300D6
:1063D0000120184310BD10B508211820FFF73AFF1F
:1063E0000300C00FC01801234010153040001843AF
:1063F00010BD0000F8B501231C00984229DD0F688C
:106400003B4226D04E6835001D4022D1042E20D9B3
:106410000F2231680A40092A1BD173685C10202CB6
:1064200000DD2024134B1B68002B01D1FFF736FE43
:106430007F10F9B2104F2200380000F07BFCA5421B
:1064400014DA380000F073FB002804D101246D0039
:106450002C432000F8BD380000F06EFB0122AB0099
:106460004000F31810439860AD18E8E76400012578
:10647000EEE7C046CC1A0020F41A00200020704736
:1064800001207047002070470020704701207047AE
:1064900000207047002070470020704700207047A0
:1064A0000020704700207047002070470020704790
:1064B00000207047704770477047000010B5034ACE
:1064C0000E210348FEF728FF10BDC0463CDA00004D
:1064D000ACDA00000378013B1F2B00D97047013074
:1064E000F8E710B5FFF7F6FF0378002B0BD001306B
:1064F000222B11D10378002B03D0421C222B03D175
:106500001000FFF7E7FF10BD5C2B03D14378002B91
:1065100000D0821C1000EDE73A2BF2D02C2BF0D0EB
:106520007B2B0BD1FFF7D6FF0378002BE9D07D2B17
:1065300001D10130E5E7FFF7D4FFF5E720225B2B1F
:1065400014D1FFF7C7FF0378002BDAD05D2BF0D012
:10655000FFF7C7FFF7E7202BD3DD2C2BD3D0190093
:1065600091435D29CFD0222BCDD001300378002B71
:10657000F1D1C6E7002210B5904216D0FFF7AAFF6E
:1065800003780422222B10D0023A7B2B0DD0013A43
:106590005B2B0AD0190030390232092905D92D2B7D
:1065A00005D14178303909290AD8100010BD0522DB
:1065B000742BFAD00132662BF7D001326E2BF4D057
:1065C000581E83415A42F0E770B5FFF783FF037806
:1065D00001222D2B01D18018023A00230A2502E066
:1065E0006B430130CB1801783039CCB2092CF7D984
:1065F0005A43100070BDF8B50C001500FFF76AFF94
:106600000378222B02D000232370F8BD0D236A1ECD
:10661000210008250C260A279C4601300378222BEE
:1066200002D100230B70F0E7002BFAD0441C5C2B46
:106630000BD14378841C622B0ED0662B0ED06E2BB0
:106640000ED0722B0ED0742B0ED0002AE9DD0B7009
:10665000013A01312000E1E72B00F6E73300F4E7CF
:106660003B00F2E76346F0E70923EEE710B50400CC
:10667000FFF737FFA04202D90378202B00D910BDC5
:106680000138F7E710B5002815D00378002B13D098
:10669000FFF720FF2021037802008B4300205D2BB1
:1066A00009D01000FFF71DFF03782C3B5A425341DD
:1066B000C018FFF70FFF10BD1800FCE70300002013
:1066C00070B50C0081420EDD1A785B2A0BD1581C84
:1066D000FFF700FF0125AC4205D0FFF7D3FF0028EC
:1066E00001D00135F7E770BD70B50C001500002929
:1066F00001D000230B70002820D00378002B1ED07F
:10670000FFF7E8FE037806002C2B03D10130FFF7DA
:10671000E1FE0600337800207D2B0FD0844204D0A8
:106720002A0021003000FFF766FF3000FFF7D9FE96
:1067300003783A2B02D10130FFF7CCFE70BD180070
:10674000FCE7F0B50D0004009DB02E78002E35D08A
:106750002E21280005F03EF9071E14D0431B01939B
:10676000303E092E14D82800FFF72EFF010020002C
:10677000FFF7A4FF0400002C20D0002F1ED0019BA7
:106780000133ED18E1E7280005F03CF90190E7E757
:1067900023787B2B11D1601C642203A9FFF7A4FF8F
:1067A000041E0BD0019A290003A805F032F9002835
:1067B000E1D02000FFF795FEEEE7002420001DB099
:1067C000F0BD70B5050000200C0081421DDD2800E1
:1067D000FFF7D0FE0300681C012B14D00020022B11
:1067E00013D10022681C1100FFF77EFF012C0CD092
:1067F000FFF748FF00221100FFF776FF013CF5E7A5
:10680000FFF740FF013C012CFAD170BDF8B505003F
:1068100000200C0016001F0081420DDD2800FFF74C
:10682000A9FE03000020022B06D1681C3A003100AB
:10683000FFF75AFF012C00D1F8BDFFF723FF3A0004
:106840003100FFF751FF013CF4E710B50024A042EE
:1068500018D0FFF73FFE03787B2B0AD101300022CE
:106860001100FFF741FF00280CD0FFF73AFE01347A
:10687000F5E75B2B06D10130FFF704FF002801D0BC
:106880000134F9E7200010BDF8B5002816DD0D68C9
:10689000EB0713D56D10013D0124FDF74BFF0026DA
:1068A000FF27644200280CD1002E21D0300005F0D3
:1068B000A9F801003000FCF77DFFF8BD01256D420D
:1068C000EAE703681A143A40152A0BD11B123B4021
:1068D0009C4200DA1C009D4201D106000836FDF7FB
:1068E0001DFEDFE71D2AFAD1012400266442F6E7E7
:1068F0000120013464002043DFE7000010B5086880
:106900000C00FCF737FDFFF77FF9002803DB626816
:10691000024B8000C250002010BDC0467C2D0020DC
:1069200010B50868FCF726FDFFF76EF90123002873
:1069300002DB024B8000C358180010BD7C2D0020E4
:1069400010B50868FCF716FDFFF75EF9C043C00FED
:10695000800010BD10B5034A04210348FEF7DCFC9B
:1069600010BDC0463CDB000035DB000010B5FCF775
:1069700031FCFCF7D1FCFEF73DFD0448FEF71CFF9F
:10698000FEF736F8FEF78AFF10BDC0468BDB00002D
:1069900010B5FCF72DF910BD70B5002504AC2478B6
:1069A0000573A94205D10A4B0A4A23210A4804F07B
:1069B00015FC01600949920052589B0002715B5816
:1069C000A40083716358856043710223C37170BD55
:1069D000A3DB000002DC0000B1DB000060DC000093
:1069E000037B002B04D1437383730361013303736F
:1069F000704700001FB50191A02100240068C90064
:106A0000D2B24450012A10D0A24209D0032A0AD09F
:106A1000074A8350074B019AC250012343501FBDC0
:106A200002221343F4E70422FBE70622F9E7C046FB
:106A3000540500002405000010B50400FFF7D0FF46
:106A4000A1222368A179D20099506179064A2000D9
:106A50009950217904329950044B19685A689B68FF
:106A6000FFF7C8FF10BDC0460C050000E81A002063
:106A70004BB2002B0FDB80233F290FD81F290FD8E3
:106A80000F290FD807290FD803290FD81B06016833
:106A9000074A8B50704780239B04F8E7DB04F6E736
:106AA0001B05F4E75B05F2E79B05F0E7DB05EEE786
:106AB000240500000368074A99501A00FC32D16887
:106AC0000029FCD0A321C90058580023C0B2D360CC
:106AD0007047C0461C05000007B58022074BD20551
:106AE0001A6000229A6002321A7111230E3200934A
:106AF000034905330348FFF74FFF07BDE81A00209D
:106B000000300040D41A0020F8B505000E00170030
:106B10000024BC4208D02B68315D1B6828009847D0
:106B2000002801D00134F4E72000F8BD704710B50B
:106B30001C3000F0A9F910BD10B51C3000F096F91A
:106B400010BD10B51C3000F0A5F910BD70B5437E26
:106B50000D00002B01D1002070BD6430040000F056
:106B6000A2F90028F7D12000290000F070F90120D7
:106B7000F2E70000F7B50193FA23002504009B001B
:106B800083600D4B4560083303601C300F00160016
:106B900000F052F92000643000F04EF9074A2761F6
:106BA000B600B35820006375019B9B009B58657627
:106BB000A576A375FEBDC04640DC000060DC000089
:106BC0000123A022C375837D0E49C133FF33D20553
:106BD0009B009950437DC133FF339B009950CC22D9
:106BE0000169094B5204CA5005220169243BCA506D
:106BF000827D01690833CA500269417D034BD1503F
:106C00007047C0460C060000240500000C0500007B
:106C1000A022002310B50469D200A3500A4CA1425F
:106C20000FD90A4C8C425B4109495B420B40CD2194
:106C3000C9045B1804690749635005210369995029
:106C400010BDCC235B04F5E7A086010090D00300C3
:106C5000000098FD24050000F7B5040000200D0099
:106C60000193824265D01600402A00D940262700B1
:106C70001C37380000F0F6F8B1232269DB00D5504C
:106C800080220123216992008B50A27E002A03D129
:106C900022691362226913600025731EAB4207D17B
:106CA000019B002B04D0802202212369920099507D
:106CB000012223691A622369FC33DA68002A02D1AF
:106CC0009A6A002AF9D09A6A002A0BD1DA60A323C3
:106CD0002269DB00D1583800C9B2013500F0B7F89D
:106CE000B542DAD3019B2269002B0FD11300FC338C
:106CF0009B6A002B0AD10133A376D3612369FC334D
:106D0000DA6C002AFCD00022DA640AE000230121B8
:106D1000A37651611A002369FC3399680029FCD0DD
:106D20009A602369FC339A6A002A01D000229A6291
:106D3000E8B2FEBD10B50123FFF78EFF10BD0300C2
:106D4000AC3310B504001970643000F08BF80123E7
:106D5000637610BD0023020070B5AC3243760D009F
:106D60001178B12204000069D2008150802221698B
:106D700092008B50226901331362226993602600CE
:106D80006436300000F080F8002812D0300000F0A7
:106D90006DF81E4B2269D0502369FC331A6A002A11
:106DA00002D19A6A002AF9D09A6A002A01D11A629D
:106DB000E5E723690122002D0DD11900FC31896A14
:106DC000002908D1DA612369FC33DA6C002AFCD08F
:106DD0000022DA6407E05A612369FC339A68002ACA
:106DE000FCD000229A6000202369FC339A6A824218
:106DF0000BD098622169064A8B588B501800022BE1
:106E000003D0181F431E9841033070BD1C050000BD
:106E1000C404000010B50121FFF79CFF10BD000065
:106E200010B51323122202490248FFF7A3FE10BD3A
:106E300000400040F41A002010B540220021040058
:106E400004F056FA002320002364636410BD10B5DB
:106E50003F24026C531C2340446C9C4201D081545B
:106E6000036410BD0023036443647047436C026CE9
:106E7000934206D03F21C25C01330B4043641000B3
:106E8000704701204042FBE7036C406C181A00D5A4
:106E900040307047436C026C934201D0C05C704735
:106EA00001204042FBE73F22036C406C013313405A
:106EB000181A43425841C0B27047000003210A48E3
:106EC00002680A430260094802680A4302600849EE
:106ED000084A094B9B1A03DD043BC858D050FBDC21
:106EE00000F012F8F9F710F92405004054050040AD
:106EF000ACE100000000002060020020FEE7FEE799
:106F0000FEE7FEE7FEE7FEE72D4B10B51A68D2B2AA
:106F1000012A0FD12B4A126812070BD12A4AE0240A
:106F20001168F0220800104021422DD1274909683C
:106F300011422CD01A68D2B2012A12D12149096813
:106F400009070ED1F020204909680140402908D1E5
:106F50001E490968014204D18020C121C005C90031
:106F600042501B68DBB2012B0DD1164B1B681B076F
:106F700009D1154B1A68F0231A40A02A0FD1134AE1
:106F800012681A420ED010BD3028CFD0D2E7104A76
:106F9000104911608021104A09021160CAE7D02A05
:106FA000F1D1ECE70D4B1A68012A04D00C4A1A60A3
:106FB0001A68012AFCD1C0220A4B1A60E3E7C046D6
:106FC000E00F00F0E40F00F0E80F00F0EC0F00F02D
:106FD00004050040DFFF07C0186C004000EC0640CD
:106FE0007593000014EC06400120704710B503684B
:106FF0001322DB69984710BD70470000054B0269FA
:10700000D1500369FC331A6A002AFCD00022012007
:107010001A6270471C050000030010B55C331A7833
:107020001F231A401E3B19009140114AD167C2220A
:10703000042104699200A150026953600269D3607F
:10704000A02300220169DB00CA5001230169094A1B
:107050005B428B500169084A8B5001690C3A8B5096
:10706000016908328B501430FFF7FCFE10BDC0469A
:1070700004E100E00C0500001405000010B5143018
:10708000FFF702FF10BD10B51430FFF703FF10BD6E
:1070900010B51430FFF7EAFE10BD0000030070B514
:1070A0005E331A780469724BE25003005D331A783C
:1070B0000469704BE250030061331C7802696E4B27
:1070C000012C00D09EE005005F352E78A225ED0052
:1070D0005651020060321578A1220669D200B550DF
:1070E0000269D4509623DB00994200D88CE09623A5
:1070F0001B01994200D88AE096235B01994200D88F
:1071000088E096239B01994200D885E0E1239B010A
:10711000994200D882E09623DB01994200D880E0B2
:10712000E123DB01994200D87DE096231B029942BE
:1071300000D87AE0E1231B02994200D877E0962339
:107140005B02994200D874E0E1235B02994200D8C7
:1071500071E0E1239B02994200D86EE0474B9942CF
:1071600000D86CE0E123DB02994200D86AE0E1221A
:10717000002312038A425B41414A5B421340802252
:1071800052059B1801693F4A8B50A02304220169D4
:10719000DB00CA5000210369FC33D9600369FC336A
:1071A0001962012301690B6001698B60C1210469C7
:1071B000890062501F215C3002780A40934062319E
:1071C000314AFF3153500021415600293CDA0F2348
:1071D0000B40083B2D4C9B089B001B1903242140AE
:1071E000A140FC348C40DD69A5432C00C0258D40B6
:1071F00029002143D9611F23017819401E3B8B4090
:10720000136070BD00246CE79E23DB02BAE79D2368
:107210001B03B7E71E4BB5E71E4BB3E7EC239B03FD
:10722000B0E71D4BAEE71D4BACE71D4BAAE71D4B6E
:10723000A8E71D4BA6E71D4BA4E71D4BA2E7802343
:10724000DB049FE71B4B9DE78C080F4BA400E41861
:1072500003230B40FF21C025DB009940AD00665998
:107260008E433100C0269E4033000B436351C2E77A
:107270000C050000140500006C05000090D0030010
:1072800000D0BEFE2405000000E100E000ED00E0BB
:1072900000B013000050270000A04E0000F0750061
:1072A00000509D0000F0EB0000903A0100E0D70193
:1072B00000B0AF0300705F07F7B5009308AB1B7811
:1072C00000250193FA2304009B0083600E4B456068
:1072D0000833036014300F001600FFF7ADFD2300E4
:1072E0005C3327611E70009B084A9B00995823005D
:1072F0005D331970019B20009B009A5823005E3378
:10730000DD701A70FEBDC046DCDC000060DC0000F1
:10731000036910B51A00FC32D2680400002A0AD0B2
:10732000A322D20099581430C9B2FFF790FD002271
:107330002369FC33DA6010BD10B50248FFF7E8FF9F
:1073400010BDC046AC1B00201D2307B502220093D0
:10735000024901330248FFF7AFFF07BD002000409C
:10736000AC1B002010B5002801D004F07DFA10BD40
:107370007047000010B500F011F8FFF7F9FF012089
:1073800000F000FAFFF7F2FAFFF702FB024B002BC6
:10739000FAD000E000BFF7E700000000C420114B66
:1073A00080001A5810491140C02212020A431A5094
:1073B000C0218022490092025A501A608023A322E1
:1073C0000021DB05D20099500122F9309A60074B69
:1073D000FF301950C120023180001950403019503F
:1073E0001A60704700E100E0FF00FFFF001001405D
:1073F000014B18607047C04674000020F7B50023A9
:107400001E285AD8384B8000C258042A5BD007D8AF
:10741000022A54D055D80423012A09D000234CE075
:10742000062A54D051D31A2A53D002231B2AF5D14D
:107430002E4A116808294ED909294FD00A2402265C
:10744000A02001252A4AC00015502A482A4D076865
:107450001C20BF0007402948019700685759009039
:1074600027481B0207401F43C02300989B0203408C
:10747000FF2057515759000207401F43019B1F43EC
:10748000009B58016023184007433E435651012595
:107490001C4B156058680028FCD000205860A123C0
:1074A0000125DB00D3585560A025ED0050511BB2DB
:1074B000A14202D015D2611ACB401800FEBD0823AC
:1074C000B6E71023B4E72023B2E74023B0E78023D8
:1074D000AEE70123ACE708240026B1E70C00012643
:1074E000AEE7091B8B40E8E760DC0000700000207D
:1074F000007000402C000020040500003000002037
:10750000FF00FFFFFC700040F0B51E285BD8364B33
:107510008000C258354B1E68002E30D1C227344B34
:10752000BF00D859334C03250440C020000220433B
:10753000D851C02480206400800018512E4F18605C
:107540002E4B803CD859FF3CA043D8510437D85922
:10755000A8432043D8510837D8590C35A84384464E
:10756000072065462843D851A820C0001E50C120DE
:107570008026800076021E501C601C4B1C60142567
:1075800000202B001E4C2E0046433659771C1BD181
:107590004343E250A0230325C132FF329200DB05B2
:1075A000D550184B1A68082A14D114234343E31802
:1075B0009A6812485132FF32920059601150DA68CD
:1075C000C1239B00C250F0BD9642E1D00130032898
:1075D000D9D1F8E7082A02D9083AD140E5E70823CB
:1075E0009A1A9140E1E7C04660DC0000101C0020C0
:1075F00000E100E0FF00FFFF0405000000900040F4
:1076000034000020740000202149F0B54A6C214864
:10761000002A14D0A025A12600230124ED05F600A0
:10762000C258571C06D0C7187F68002F02D0270009
:107630009740AF5114333C2BF2D100234B64A0236D
:107640000121DB0500260F009C4614234B43C31881
:107650001A1F1268104C0E4D920014195219526CD8
:10766000002A10D01A00143A1268551C09D0103B99
:107670001B68FF2B05D03B00934065461A00074B63
:10768000EA50FC34666401310429DED1F0BDC04605
:10769000FC90004034000020009000400C050000E9
:1076A00000B51E2810D80C4A8000835803290BD837
:1076B000A0220800C133FF33D2059B0001F036FC45
:1076C000020905070021D15000BD0C21FBE7042170
:1076D000F9E70321F7E7C04660DC00001E280AD85E
:1076E000074B8000C25801239340A022D2050029F5
:1076F00002D1044953507047A121C900FAE7C0469E
:1077000060DC00000C050000030000201E2B0AD8DE
:10771000A021A222C905D2008858034A9B009B5889
:10772000D84001231840704760DC0000F7B5060020
:107730000D000C008B180193019B671B9C4207D026
:10774000336821781B683000984701340028F3D152
:107750003800FEBD0849094A094B10B51B68885816
:10776000FA22190A1B0618439200002301F0B4FD07
:107770004904C00B084310BD00100140040500007F
:10778000141C002070B5041E09D0FFF7E3FF0500AC
:1077900000F014F8FFF7DEFF401BA042F8D370BDE5
:1077A0000022044B9A60044A13680133DBB2136071
:1077B0007047C046FC100140141C002070470000B8
:1077C000F0B5C64600B5CB0F9846404A4B005B0D5E
:1077D0009A1882B00D000400132A2FDC002A49DB1E
:1077E0003B4F17413E000E40064323D07F0839002F
:1077F00029400C430AD03749BD438C4663445C4260
:107800005C418023DB021341E4071D434146CE0067
:1078100031492B008E192200346875682000290038
:1078200001F000FF009001910098019922002B00C7
:1078300003F090F802B004BC9046F0BD332A08DD96
:107840008023DB009A42F5D102000B0001F0EAFE32
:10785000F0E7224A9446012263445242DA4002424F
:10786000E8D052080242D1D094438022D2051A4176
:107870001443CBE74B005B080343DBD00B031B0B2C
:107880001C436342234380244D0C24031B0B2340E1
:107890006D042B4319004346DA000F4B9B181C68FC
:1078A0005D6802000B002000290001F0BBFE009083
:1078B00001910098019922002B0003F04BF84246F9
:1078C0004B005B08D60733431900B3E701FCFFFF09
:1078D000FFFF0F00EEFBFFFF10DD0000EDFBFFFFE1
:1078E000F8B5274A4B005B0D9A180C000700132AC5
:1078F00010DC002A36DB234B13410B423AD08024A4
:1079000024031441002064189C4306002500300025
:107910002900F8BD332A0EDD80230600DB000D00B0
:107920009A42F4D102000B003800210001F07AFEE7
:1079300006000D00EBE7144D0600AC46012563443C
:107940006D42DD40AC4663460D000342DFD0332379
:107950009A1A323B93401818874200D94C1C634650
:107960009843D2E7C90FCC070020531CCDD1074B59
:107970001C43CAE706000D000028C0D1C7E7C04677
:1079800001FCFFFFFFFF0F00EDFBFFFF0000F03FDA
:1079900030B5214A4B0087B05B0893421EDD1F4A79
:1079A000934205DD02000B0002F0D4FF07B030BDAA
:1079B00002AA00F095F803231840049A059B0128B9
:1079C00013D002281DD0002814D00298039900F08B
:1079D0006FFB80231B069C466144E7E700230022DF
:1079E0000093002301F0DEF8E0E70298039900F02D
:1079F0005FFBDBE7012402980399009401F0D2F8C1
:107A0000D4E7012402980399009401F0CBF8802375
:107A10001B069C466144C9E7FB21E93FFFFFEF7F5E
:107A2000F0B54746CE4680B58DB004000D0000F09D
:107A300067FA294B06001B780F005BB298460133AA
:107A400010D022002B002000290003F0CBFA814641
:107A5000002807D1002200232000290001F014FC97
:107A6000002806D1300039000DB00CBC9046994674
:107A7000F0BD01230293194B0694079503934B46DF
:107A80000A93434604940595002B15D00023002249
:107A90001900100002F0E2F8434608900991022B09
:107AA0000ED103F0B9FB212303600A9B0193002B45
:107AB0000CD1089E099FD5E7002300240893099460
:107AC00002A801F0C1F90028EFD1EAE703F0A4FB16
:107AD0000A9B01930360ECE77800002020DD0000A2
:107AE000F0B54E464546DE465746E0B5E14B4C0004
:107AF0008FB09046894664089C4200DC87E0DE4BEC
:107B00009C4222DCDD4A002900DC92E0DC4B02F0E2
:107B100021FFDB4B06000F009C4200D17EE1D94AD9
:107B2000D94B02F017FF02000B00414630000A60FB
:107B30004B60390002F00EFFD34BD24A02F00AFF2D
:107B4000434601259860D9606BE0D04B9C4200DC35
:107B50008FE0CF4B9C4200DD55E1CE4A2315924683
:107B60009A4451460905631A19001D00040003F0E8
:107B700055FA03F089FA02000B0020002900089250
:107B8000099302F0E7FE0022C34B02F071FC0F00E4
:107B9000060003F043FA03F077FA04000D00020038
:107BA0000B00300039000A940B9502F0D3FE00223E
:107BB000B94B02F05DFC002200230C900D9101F006
:107BC0005DFB002800D192E1002300222000290063
:107BD00001F054FB434243410133B04A4146019214
:107BE000022208A80092524600F07CFB4B4605009A
:107BF000002B16DA802243461206944642465B6802
:107C0000454263445360D3686344D36009E00B008A
:107C1000020041460A604B600022002300258A6072
:107C2000CB6028000FB03CBC90469946A246AB46BC
:107C3000F0BD934B01F0F6FC914B06000F009C4207
:107C400000D13DE18F4A904B01F0ECFC02000B00AB
:107C5000414630000A604B60390002F07BFE894AE1
:107C6000894B01F0DFFC012543466D429860D960E5
:107C7000D7E701F049F88A4A8A4B06000F0002F064
:107C8000F7FB0022884B01F0CDFC03F0C7F905009B
:107C900003F0FAF9794A7A4B0490059102F0E8FB77
:107CA00002000B003000390002F054FE754A060055
:107CB0000F0004980599744B02F0DAFB02900391CF
:107CC0001F2D00DCC7E0029A039B3000390002F050
:107CD00041FE83468A4653465B0024155B0DE31A3A
:107CE000102B6CDD04980599D322674B520502F0E6
:107CF000BFFB02000B00300039000292039302F038
:107D000029FE0A00010013000691079202003900C3
:107D1000300002F01FFE029A039B02F01BFE0600D9
:107D20000F0004980599614A614B02F0A1FB3200F3
:107D30003B0002F00FFE069E079F0B000200390079
:107D400030000292039302F005FE4B005B0D834668
:107D50008A46E41A312C32DD04980599B822544B36
:107D6000920502F085FB03000C00020002930394CD
:107D70000B000698079902F0EDFD02000B000600CB
:107D80000F000698079902F0E5FD029A039B02F0A6
:107D9000E1FD484A0290039104980599464B02F090
:107DA00067FB029A039B02F0D5FD02000B00300036
:107DB00039000292039302F0CDFD83468A465A466B
:107DC0005346414630000A604B60390002F0C2FD64
:107DD000029A039B02F0BEFD44460B000200A26023
:107DE000E3604B46002B00DB1BE75B4623608023F0
:107DF0001B065344636080231B069C466144A060BD
:107E0000E1606D420DE70B00020002F0A3FD434666
:107E100000259860D9601860596002E7D3221A4B98
:107E2000520502F097FD214A214B0D00040002F09B
:107E300091FD02000B00414620000A604B602900C2
:107E400002F088FD1A4B194A02F084FD43460125D1
:107E50009860D960E5E602000B003000390002F0BE
:107E600079FD6B1E154A9B009B5883468A46A342A8
:107E7000A5D130E7FB21E93F7BD902400000405407
:107E8000FB21F93F3163621A61B4D03DFB213941D6
:107E9000FFFFEF7FEAFBFFFF00007041A8DD00005D
:107EA00083C8C96D305FE43F0000E03F7370032E6C
:107EB0008A19A33BC14920259A837B3928DD00001C
:107EC000D3220C4B520501F0ADFB0B4A0B4B0400C7
:107ED0000D0001F0A7FB02000B00414620000A60E4
:107EE0004B60290002F036FD034A044BB9E6032338
:107EF00073E6C04661B4D03D7370032E8A19A33B6C
:107F0000F8B54746CE46674B80B50A000F0019000A
:107F100005003940994200D19BE004000100002F88
:107F200069DD3F1500D1B4E05F4B12039C4680230E
:107F3000120B5B0313435B00CA0F67449B184A0094
:107F4000F80703D5D20F5B009B188A0079108C4686
:107F5000002180201624894680030D189D4202DCF2
:107F600029185B1B8144D50F5B00013C5B19520053
:107F70004008002CF1D100208046802020250027D9
:107F8000000609E08B425CD0D40F5B00013DE31892
:107F900052004008002D16D0C4198B42F2DD27187C
:107FA0000E00002C49DB5B1AA242894149425B1A50
:107FB000121BD40F5B00013D80443100E3185200D6
:107FC0004008002DE8D113434ED143465B083749A2
:107FD0004A468846494652104244C90702D5802184
:107FE00009060B4361460F05BD18180029000CBC9B
:107FF00090469946F8BD7B005B0803433900002B8F
:10800000F5D0002F3CD1E30A153A6405002BFAD0D5
:108010008020400303423FD1002700E00F005B00B7
:10802000791C0342FAD0250020208D40401A2900F7
:10803000D71B2200C2401A4376E7FE43F60F8E1983
:10804000B1E79442A0D82718002CF6DB1E000023CD
:10805000AEE702003B002800390002F009FA2A00CE
:108060003B0001F0DFFAC2E74346013303D0434649
:1080700001335B08ABE7012398460023C144A6E720
:108080003B00020002F066FC02000B0001F0E6FD7E
:10809000ADE713000022BBE70127210020207F422B
:1080A000C6E7C0460000F07F01FCFFFF0000E03F94
:1080B000F0B54746CE4680B587B000920193754B28
:1080C0004F00814688467F089F4263DC02F0A6FF8E
:1080D000002800D1D4E04A4643464846414602F0D3
:1080E000C7F904000D006C4A6C4B02F0C1F96C4AF0
:1080F0006C4B01F097FA22002B0002F0B9F96A4AA2
:108100006A4B02F027FC22002B0002F0B1F9684A0A
:10811000684B01F087FA22002B0002F0A9F9664AA9
:10812000664B02F017FC22002B0002F0A1F9644A12
:10813000644B01F077FA22002B0002F099F90290CB
:1081400003910022604B2000290002F091F9029A6D
:10815000039B06000F002000290002F089F9009A15
:10816000019B04000D004846414602F081F90200DF
:108170000B002000290002F0EDFB02000B00300094
:10818000390002F0E7FB02000B0000204F4902F02B
:10819000E1FB70E002000B0002F06AF904000D0040
:1081A0003D4A3E4B02F064F93D4A3E4B01F03AFA3B
:1081B00022002B0002F05CF93B4A3C4B02F0CAFB68
:1081C00022002B0002F054F9394A3A4B01F02AFA06
:1081D00022002B0002F04CF9374A384B02F0BAFB70
:1081E00022002B0002F044F9354A364B01F01AFA0E
:1081F0002B00220002F03CF9354B029003919F4284
:108200009FDD344B00229F423DDC334900207B1828
:108210002E4916001F0002F09DFB049005910022DC
:10822000294B2000290002F023F932003B0002F024
:1082300091FB029A039B06000F002000290002F028
:1082400017F9009A019B04000D004846414602F0D0
:108250000FF902000B002000290002F07BFB020056
:108260000B003000390002F075FB02000B0004988F
:10827000059902F06FFB07B00CBC90469946F0BD23
:1082800000201249F7E7154B002604920593144F7E
:10829000C5E7C046FFFF3F3ED43888BEE9FAA8BD17
:1082A000C4B1B4BD9EEE213EAD529C804F7E923E45
:1082B0009015CB19A001FA3E7751C1166CC1563FFB
:1082C0004C5555555555A53F0000E03F0000F03F87
:1082D0003233D33F0000E93F0000E0FF0000E73FFA
:1082E0000000D23FF0B5DE464E4645465746E0B563
:1082F000DC4CA5440D9114001900A49A0993DA4BA3
:108300009200D6584D1E03901821E01E0696029545
:1083100000F0AAFEC3430100DB1719404B1C9A0072
:108320009B1ADB001B190B9105934C1B771918D472
:10833000A59BA5009C463F1922AE6544013707E086
:10834000286802F0A1FE013403C60435BC4208D0FF
:10835000002CF5DA00200021013403C60435BC42AC
:10836000F6D1069B002B01DA00F0FDFB069B03997A
:108370000133DB009A46099BDA0094460092002202
:10838000914672AA0492B94A6144934688469AABD0
:1083900063449B44029B002B00DABCE15D4600264F
:1083A0000027039C4D442A686B6803CC02F060F8F8
:1083B00002000B003000390001F034F9083D0600DE
:1083C0000F004445EFD1049B4B441E605F600823BF
:1083D0009C46E144D145DDD10EA8042184464942A2
:1083E00061448C46069A93009C44614684460A91F7
:1083F0000399083B63448C460C93009B00926344B2
:108400009B46009A0498D10003008C46634408916F
:108410001E685F68002A33DD954980468C466244B9
:10842000D300984470AB9A460EAB99460022914B0C
:108430003000390002F01CF802F0F0FD02F024FEDA
:1084400000228D4B04000D0002F012F802000B0018
:108450003000390002F07EFA02F0E0FD4B4601C325
:108460009946434620001A685B68290001F0DAF853
:1084700008235B429C46E04406000F00D045D5D15E
:10848000059B30001A003900984600F0DFFCFF23FE
:1084900000229B0504000D0001F0EAFF00F038FC0B
:1084A0000022764B01F0E4FF02000B0020002900BF
:1084B00002F050FA0D00040002F0B0FD814602F017
:1084C000E3FD02000B002000290002F043FA060041
:1084D00040460F00002800DCEEE0009B18215A1EE9
:1084E00092000EAB9B58091A1D000D41A9448D4006
:1084F0005D1B0EAB9D5017231B1A1D41002D2DDD5A
:1085000001239C46009BE144002B00DC1CE20E9CF6
:108510000123002C00D0B5E0009A012A09D099006F
:108520000EAA54580133002C00D0ACE0009A9A42B5
:10853000F5D1059B002B0EDD012B00D1A8E1022B0C
:1085400009D1009B0EA95A1E92000EAB9B580793AF
:108550009B029B0A8B50022D00D1C1E00023002218
:108560003000390000F08AFE009B002800D194E220
:10857000069A591E8A4210DC414A0A9894460EAA6D
:108580006344944600229B0063441C68043B2243DE
:108590008342FAD1002A00D0C0E0069B0EAA013B1C
:1085A0009B00D358002B00D0B3E001220C9B043B6E
:1085B000596801320029FAD0009B9C4662441100A0
:1085C00007921A0001338B4246DC0B9863468046C3
:1085D000A59C4344A046099C9B00A1464A4498445C
:1085E000D30022AA9146049A99449446089BA59ADE
:1085F00063448446614494469A468B0063440093E6
:108600004346586802F040FD4B4618605960029B93
:10861000002B24DB4D46039C0026002701E0286840
:1086200069680CCC01F024FF02000B003000390017
:1086300000F0F8FF083D06000F005C45EFD15346FF
:108640009E60DF6004239C460433E0449C46009B0C
:10865000E144E2449845D3D1079B0093D1E600263C
:108660000027ECE794FDFFFFF0DE000018FEFFFF9F
:10867000FFFFFF1F0000703E00007041000020401F
:10868000FFFFFF3F002180225204141B0EAA54500A
:10869000009999420EDD0EA884469B000EAA89001F
:1086A000D25861446344CF4800E01A68821A04C378
:1086B0008B42FAD101243CE7059B002B06D1009B9D
:1086C0000EAA013B9B00D558ED1517E70022C64BBB
:1086D000300000F0F7FD002800D024E100253DE740
:1086E00032003B000020C14902F034F906000F00BF
:1086F000002C00D132E7059A0020BC4900F0A6FB0F
:1087000002000B003000390002F024F906000F00CF
:1087100024E7012250E70026002754E64B46059A3D
:10872000079388468B000EA9CB58183A08950592F6
:10873000002B0DD18C464146AD4B43449B00634416
:10874000043B58680139183A0028F9D08846059248
:10875000059A0020A54900F079FB434604000D006E
:10876000002B00DA05E29E000EAB9C464346DB0080
:1087700066449C46059370AB9946049F67440097F6
:10878000306802F081FC22002B0001F071FE002213
:1087900038607960974B2000290001F069FE083F9E
:1087A00004000D00043EB945EAD14AAB03939B4651
:1087B00000239A46069B424699464346013202925E
:1087C00004934B46002B00DAAAE080208A4B009DE0
:1087D0009846C005894900260027002408E00823A0
:1087E0009C460835E044544511DC434618685968F6
:1087F0002A686B6801F03CFE02000B003000390073
:1088000000F010FF013406000F00A145E7DA5B46D7
:10881000C0C39B4601239C46009BE244083B009357
:10882000029B9A45CDD1049B9846A49B022B00DD68
:108830008EE0002B37DC1FD1059B00271D00039B1A
:1088400000249C461E006544083E2A686B68380078
:10885000210000F0E7FE083D07000C00AE42F4D115
:10886000089B002B03D080231B069C4664443A00DF
:1088700023000D990A604B600720079B18409B233B
:108880009B009D443CBC90469946A246AB46F0BD39
:10889000009B0EA95A1E92000EAB9B5807935B02D9
:1088A0005B0A8B5057E64346002B00DA70E100204C
:1088B0000021DB004AAAD61848AF32687368083E28
:1088C00000F0B0FEB742F8D1089B002B00D025E1A4
:1088D0000B0002004A984B990D9C2260636002F0E5
:1088E00039F8434607000C00002B13DD01254CAE80
:1088F000B14638002E0021004C4601360CCC00F069
:1089000091FEA146B045F7DA089B07000C00002B4A
:1089100000D015E13A0023000D998A60CB60ABE7E7
:108920000026002773E701239C46009BE1440225B3
:10893000002B00DDEBE532003B0000202B4902F06C
:1089400009F806000F0009E60024F2E54AAB03939C
:10895000A49B032B00D08FE74346002B00DC14E1DF
:10896000039ADB009B46130091465B441E685F68D8
:10897000234B43440293DB00994448AB9A464B4651
:108980005C681B681800210032003B0000900191D8
:1089900000F048FE04000D0002000B000098019951
:1089A00001F0D8FF3B00320000F03CFE4B469860DF
:1089B000D9601C605D6008235B429C46E144260050
:1089C0002F00CA45DBD14346012B00DCE3E0039ACC
:1089D00013005B441E685F68029BDB0099464A44B3
:1089E000904610E0FFFFFF000000E03F0000F03F76
:1089F000FFFFFF3F0000703EB0DE0000FB21F93FAB
:108A0000FFFFFF1F984643465C681B681800210063
:108A100032003B000090019100F004FE04000D00C4
:108A200002000B000098019901F094FF32003B0016
:108A300000F0F8FD4346039A9860D9601C605D60C1
:108A4000083B26002F009A42DCD14D469446002672
:108A500000244746083565442A686B6830002100C9
:108A600000F0E0FD083D06000C00AF42F4D1039B8E
:108A70004A9F5D689968D868089B002B65D0802262
:108A8000120694460D9B6544604464441F605D601B
:108A90009960D8601E615C61EEE69A464B4607938A
:108AA000059B30005A423900089500F0CFF90022AA
:108AB0003A4B06000F0000F005FC002824D0384B8C
:108AC00000223000390001F0D3FC02F0A7FA524630
:108AD0000400950002F0D8FA0022304B01F0C8FCE7
:108AE00002000B003000390001F034FF02F096FA6A
:108AF0000EAA50510122059B52441833904605930B
:108B000093000EAAD45023E65346300039009C004F
:108B100002F084FA0EAB1851D04619E680230D9A64
:108B20001B06CB18106053600B0002004A984B994B
:108B300001F010FF434607000C00002B00DDD5E6D6
:108B400080231B069C466444E4E62B003A000D9DFE
:108B50002A606B600A000300AA60EB603200230009
:108B60002A616B6188E6099BDB00009372AB04937A
:108B700032E4A49B022B00DDE8E6002B00DD92E648
:108B800000D079E6002700246AE6002600246EE77C
:108B90000020002198E60026340068E700007041BC
:108BA0000000703EF0B5CE46474680B587B00092D3
:108BB0000193474A4B00814688465B08934207DC95
:108BC0004146484602F02AFA4146031E484666D00E
:108BD0004A4643464846414601F04AFC04000D001F
:108BE00002000B004846414601F042FC394A3A4B2C
:108BF00006000F002000290001F03AFC374A384BEC
:108C000001F0A8FE22002B0001F032FC354A364B61
:108C100000F008FD22002B0001F02AFC334A344BFF
:108C200001F098FE22002B0001F022FC314B324A69
:108C300000F0F8FC0E9B02900391002B34D00098BA
:108C4000019900222D4B01F013FC029A039B049022
:108C500005913000390001F00BFC02000B00049874
:108C6000059901F077FE22002B0001F001FC009A2B
:108C7000019B01F06FFE224A04000D00214B3000E1
:108C8000390001F0F5FB02000B002000290000F084
:108C9000C9FC02000B004846414601F05BFE07B0EC
:108CA0000CBC90469946F0BD02000B002000290044
:108CB00001F0DEFB124A134B01F04CFE32003B0088
:108CC00001F0D6FB4A46434600F0ACFCE7E7C0465D
:108CD000FFFF3F3E7CD5CF5A3AD9E53DEB9C2B8A2E
:108CE000E6E55A3E7DFEB157E31DC73ED561C11989
:108CF000A0012A3F1111813FA6F810110000E03FAA
:108D0000495555555555C53F49004B081900704701
:108D1000474AF0B54F4691464B005B0D9944464695
:108D2000D6464A46C0B505000C000E00884607002E
:108D3000132A27DC002A4BDB3E4B13419A460B00DB
:108D400052461340034318D03B4A3C4B28002100B5
:108D500000F068FC0022002300F0AAFA002847D0A7
:108D6000002C04DA80234A465B03134198444646AC
:108D7000534600279E43380031001CBC904699465C
:108D8000A246F0BD332A08DD8023DB009945F4D1EB
:108D900002000B0000F046FCEFE7294A944601224E
:108DA00063445242DA4092460242E6D0224A234BC2
:108DB0002800210000F036FC0022002300F078FAA1
:108DC000002815D0002C1EDB534646469F430FE07B
:108DD000194A1A4B2800210000F024FC002200232D
:108DE00000F066FA002803D0002C04DB00270026E0
:108DF00038003100C1E76400640825430027002DD6
:108E0000F6D0104EF4E74B46142B0BD03422D21A76
:108E1000012393405D19BD4208D201239C462F00D7
:108E2000E044D1E7133B9C46E044CDE72F00CBE77D
:108E300001FCFFFFFFFF0F009C7500883CE4377EBC
:108E4000EDFBFFFF0000F0BF002070474B0070B546
:108E50005B0D14000A00002B1AD14B005B08034382
:108E600015D0234B002201F003FB224B9C422DDB4B
:108E70000A004B005B0D363B1F4DE318AB422ADC6A
:108E8000002B0DDD1D4C1B0522401A43110070BD47
:108E90001B4DAB42F0D102000B0000F0C3FBF6E724
:108EA0001D00353519DA174B02009C4209DD0B0015
:108EB0001548164900F032F8134A144B01F0D8FA5D
:108EC000E5E70B001248134900F028F8104A114B4F
:108ED00001F0CEFADBE70200E9E7084C3633224026
:108EE0001B051343190000220B4B01F0C1FACEE71A
:108EF00000005043B03CFFFFFE070000FFFF0F8063
:108F0000FF07000050C300009C7500883CE4377EDA
:108F100059F3F8C21F6EA5010000903C30B54A001D
:108F2000DB0FDB0752081A43110030BD02B4714653
:108F300049084900095C49008E4402BC7047C0469C
:108F400003B47146490840004900095A49008E445B
:108F500003BC7047002243088B4274D303098B4241
:108F60005FD3030A8B4244D3030B8B4228D3030CF9
:108F70008B420DD3FF22090212BA030C8B4202D39B
:108F80001212090265D0030B8B4219D300E0090AC3
:108F9000C30B8B4201D3CB03C01A5241830B8B42CC
:108FA00001D38B03C01A5241430B8B4201D34B03B5
:108FB000C01A5241030B8B4201D30B03C01A52411A
:108FC000C30A8B4201D3CB02C01A5241830A8B429F
:108FD00001D38B02C01A5241430A8B4201D34B0288
:108FE000C01A5241030A8B4201D30B02C01A5241EC
:108FF000CDD2C3098B4201D3CB01C01A52418309A0
:109000008B4201D38B01C01A524143098B4201D3D9
:109010004B01C01A524103098B4201D30B01C01A04
:109020005241C3088B4201D3CB00C01A524183087E
:109030008B4201D38B00C01A524143088B4201D3AB
:109040004B00C01A5241411A00D20146524110460B
:109050007047FFE701B5002000F0F0F802BDC04600
:109060000029F7D076E7704703460B437FD40022F0
:1090700043088B4274D303098B425FD3030A8B42AC
:1090800044D3030B8B4228D3030C8B420DD3FF2216
:10909000090212BA030C8B4202D31212090265D0E4
:1090A000030B8B4219D300E0090AC30B8B4201D397
:1090B000CB03C01A5241830B8B4201D38B03C01ADE
:1090C0005241430B8B4201D34B03C01A5241030B55
:1090D0008B4201D30B03C01A5241C30A8B4201D306
:1090E000CB02C01A5241830A8B4201D38B02C01AB1
:1090F0005241430A8B4201D34B02C01A5241030A28
:109100008B4201D30B02C01A5241CDD2C3098B420C
:1091100001D3CB01C01A524183098B4201D38B0189
:10912000C01A524143098B4201D34B01C01A52412C
:1091300003098B4201D30B01C01A5241C3088B4271
:1091400001D3CB00C01A524183088B4201D38B005C
:10915000C01A524143088B4201D34B00C01A5241FE
:10916000411A00D201465241104670475DE0CA0FD5
:1091700000D04942031000D34042534000229C4695
:1091800003098B422DD3030A8B4212D3FC2289019F
:1091900012BA030A8B420CD3890192118B4208D375
:1091A000890192118B4204D389013AD0921100E0D7
:1091B0008909C3098B4201D3CB01C01A52418309EB
:1091C0008B4201D38B01C01A524143098B4201D318
:1091D0004B01C01A524103098B4201D30B01C01A43
:1091E0005241C3088B4201D3CB00C01A52418308BD
:1091F0008B4201D38B00C01A5241D9D243088B4213
:1092000001D34B00C01A5241411A00D201466346B5
:1092100052415B10104601D34042002B00D5494219
:10922000704763465B1000D3404201B5002000F058
:1092300005F802BD0029F8D016E770477047C04610
:10924000D0400B1C1141203A03D49C4613411843D3
:1092500063465242934018437047C0468446101CF0
:1092600062468C46191C634600E0C0461FB501F0FB
:1092700097F8002801D40021C8421FBD10B500F0A6
:10928000EFFF4042013010BD10B501F089F8002811
:1092900001DB002010BD012010BDC04610B501F05B
:1092A0007FF8002801DD002010BD012010BDC04660
:1092B00010B501F011F8002801DC002010BD0120DC
:1092C00010BDC04610B501F007F8002801DA0020F3
:1092D00010BD012010BDC046F0B5CE46474615046E
:1092E0002D0C2E0080B50704140C3F0C9946030C7E
:1092F0007E435D43674363437F19340CE4199C4606
:10930000A54203D980235B029846C4444B4643439D
:109310005143250C36046544360C2404A4195B190A
:10932000591820000CBC90469946F0BDF0B54E4649
:1093300057464546DE46E0B543025B0A450083B02A
:109340000F1C99462D0EC60F002D57D0FF2D24D08F
:109350008020DB00C0041843002381469A469B46C8
:109360007F3D7C027A00FB0F640A120E984623D0E0
:10937000FF2A4BD0E30080240020E4047F3A1C4302
:10938000AD186B1C47460193534677403A000F2BAC
:1093900048D87D499B00CB589F46002B00D085E0E4
:1093A00008339A46063B9B467C027A00FB0FFF255A
:1093B000640A120E9846DBD1002C00D090E0524691
:1093C00001231A4392460120DBE74C46584617001A
:1093D000022824D0032800D1CFE000220023012856
:1093E0004DD15802D205400AFF071043384303B05D
:1093F0003CBC90469946A246AB46F0BD002B5BD1E3
:1094000004239A46033B00259B46AAE7FF35002C20
:1094100060D1524602231A4392460220B1E7FF224E
:109420000023DEE74B461B0C9C464B462604360CBD
:10943000180461463300220C6446000C43434E433B
:109440005043544380191A0C1218964203D98021B4
:1094500049028C4664441B041B0C1004C018830191
:109460005E1EB341800E1843130C1B199B0103436E
:109470001C00230179D5012362081C401443019A82
:109480007F32002A4DDD630704D00F232340042BD5
:1094900000D00434230103D53C4B019A1C40803298
:1094A000FE2ABCDCA3015B0AD2B29AE70C239A46DF
:1094B000093BFF259B4654E7180001F071FE4A4620
:1094C000431F76259A4000236D4291462D1A9A46F5
:1094D0009B4646E7524603231A439246032050E731
:1094E000200001F05DFE431F2D1A9C40763D0020B8
:1094F00047E780230027DB03FF2272E7424666E747
:109500004C463200584662E780234A46DB031A4243
:1095100022D01C4220D123435B025B0A4746FF2234
:109520005FE701239A1A1B2A21DC23000199D3400B
:109530009E318C401A0023005C1EA34113435A073E
:1095400004D00F221A40042A00D004335A0111D447
:109550009B015B0A002244E780234A46DB03134356
:109560005B025B0A3700FF223BE7019587E7002299
:10957000002336E70122002333E78023DB03234364
:109580005B025B0AFF222CE700DF0000FFFFFFF712
:1095900070B500283DD0C317C5185D40C40F280022
:1095A00001F0FEFD9E22121A962A07DCD2B208288C
:1095B00033DD083885406802400A23E0992A0BDD34
:1095C000052329001B1AD94003001B339D402B00A3
:1095D0005D1EAB4119430D00052801DD431F9D4071
:1095E0002B000F490B406E0709D00F263540042D84
:1095F00005D004335D0102D59F220B40121A9B0156
:10960000580AD2B24002D205400AE4071043204370
:1096100070BD002400220020F4E76802400AF1E750
:10962000FFFFFFFBF0B54F464646D6460C00090348
:10963000C0B5490A470F5E0039431F03DB0F9C4644
:1096400065007B0A570F1F436D0DE40F760DA14691
:10965000C000B846D200AB1B64457BD0002B5FDD59
:10966000002E00D0A4E03E00164300D112E15E1EA1
:10967000002E00D09EE1871A4346B8428041012562
:10968000C91A4042091A0B0200D431E149024E0ABC
:10969000002E00D16EE1300001F082FD0300083B96
:1096A0001F2B00DD61E120223900D21A9E40D140FB
:1096B0009F400E439D4200DD51E15D1B6B1C1F2B43
:1096C00000DD7CE12021C91A3D0030008F40884038
:1096D000DD40791E8F41310007222843D940002503
:1096E00007433A40002A09D00F233B40042B05D002
:1096F0003B1DBB42BF417F42C9191F000B0200D472
:1097000026E26A1CC64B55056D0D9A4200D106E152
:10971000C44AFF080A40530752023B43120B8EE033
:10972000002B00D0B8E06B1C5B055B0D012B00DC4F
:1097300030E1871A4346B842B641CB1A76429E1BA7
:10974000330200D54CE13B003343A1D10022002479
:10975000002570E0002B00DCE5E0002E00D183E066
:10976000AF4EB54260D0802636043743B846382B1A
:1097700000DC3EE1434613431F007A1E97413F1829
:1097800087428041404209180B0200D4B0E0A44B4C
:1097900001359D4200D1C3E0A24A7B080A40012165
:1097A0000F401F435108D30707221F433A4099E750
:1097B0009B4EB54238D0802636043743B846382B06
:1097C00000DDDCE01F2B00DC30E11E004746203EC0
:1097D000F740BC46202B04D04026F31A46469E4054
:1097E0003243170063467A1E97411F43CCE0002B9B
:1097F00000D104E24346134300D159E14B07C008AE
:1098000018438023C9081B03194208D04546ED08B8
:109810001D4204D14346D008590708432900420F8E
:10982000C9007F4D1143C0004B07CA087C49C008DE
:1098300003438D4268D012036D05120B6D0D00219C
:1098400012031800130B0A0D12051A43764B2D054F
:1098500013402B435B00E4075B08234319001CBC47
:1098600090469946A246F0BD3E00164312D05E1EB9
:10987000002E00D000E187188742804141444042D9
:10988000091801250B0233D5022585E7644633000C
:10989000414610001D00C7E7002D00D0DAE00C00A3
:1098A0000443F3D05C1C00D19FE15D4CA64200D183
:1098B0002FE1DB43382B00DD66E11F2B00DD83E168
:1098C00020240500E41A0F00DD40D940A0404346A3
:1098D000A7405B1A441EA04198462F433843171AED
:1098E000BA42924143465242991A64463500CAE64A
:1098F00007223A40002A00D0F6E64B07CA0848493A
:10990000FF083B438D4296D11900114300D19EE1DF
:10991000802109030A431203120B414D8FE7150002
:10992000002200238BE7002B00D0C7E06B1C5F05F3
:109930007F0D012F00DCF1E0394DAB4200D1B9E0E1
:1099400085180A008542894142444942511807223C
:10995000CF076D082F4349083A401D00C2E6072291
:109960003049ED1A31403A40BCE63E002838864086
:1099700000279FE6380001F013FC20308EE64346B6
:1099800013431F007A1E9741C71BB84280414042D3
:10999000091A78E60E003B0006431343002D61D1FF
:1099A000002E00D0F4E0002B00D11BE1644639000A
:1099B000100039E71A4FBB427AD03300FFE630007F
:1099C0001F3DE840202B03D04021CB1A9E40374357
:1099D0007B1E9F41072207433A400021002589E76B
:1099E000171A4346BA42B641591A76428E1B64464C
:1099F0004EE61F2B00DDADE020264746F61AB740A5
:109A0000B9461700B246DF404E463E433700564641
:109A1000B240561EB24117434246DA408918AEE6BC
:109A2000FF070000FFFF7FFFFFFF0F802026474654
:109A3000F61AB740B9461700B246DF404E463E43DD
:109A400037005646B240561EB24117434246DA40EE
:109A5000891A99E77F4CA6425BD0802424045B429C
:109A6000214327E7002E0CD1002B00D1CBE0644628
:109A700039001000774DD7E6764FBB4218D033003F
:109A800075E6002B14D04B07C00818438023C90883
:109A90001B03194207D0FC081C4204D17907D008E7
:109AA0000843E14621004C46420FC9001143C00063
:109AB000684DB9E61D0000220023C0E6002D5BD1F1
:109AC0000D00054300D1E2E65D1C00D1B0E0614D20
:109AD000AE421FD0DB43382B71DC1F2B00DD96E03C
:109AE00020250F00ED1AAF40B9460700AA46DF4017
:109AF0004D463D432F005546A840D940451EA8413C
:109B000088440743BF18974292415142414435006F
:109B10003AE6644635004146100085E60B000343F3
:109B2000002D00D063E6002BF5D04346134300D14F
:109B30007AE687188742804107224144404209184B
:109B40003A400B0200D4D5E6434B01351940C9E534
:109B5000380069E61E004746203EF740BC46202BF1
:109B600004D04026F31A46469E403243170063460F
:109B70007A1E97411F4302E6364DAE42CAD0802579
:109B80002D045B422943A6E70843411E8841A6E60F
:109B9000002B00D148E6871A4346B842B641CB1A9B
:109BA00076429E1B33024BD5171A4346BA42924166
:109BB000591A5242891A072264463A4092E50143F3
:109BC0000F00791E8F419DE71C000F00203CE740ED
:109BD000202B03D04024E31A99400843411E8841BA
:109BE00038437CE60022002425E6171A4346BA4291
:109BF0009241591A5242891A6446350043E541465A
:109C00001000144D10E680220024120380E61D008F
:109C10000F00203DEF40BC46202B03D04025EB1A1F
:109C20009940084307006346781E87411F4369E750
:109C3000871897429B4141445B42C9183500A3E510
:109C40003B003343CED0072231003A4052E6002396
:109C50001A00F4E5FF070000FFFF7FFFF0B557464D
:109C6000DE464E464546E0B5834607000E034800F3
:109C700085B092461C00360B400DCD0F002800D158
:109C80009DE0954B984239D08023F6001B041E437B
:109C9000924A7B0F334399469446030063440093F2
:109CA00000230026FF00029323031B0B984663004A
:109CB000E40F52465B0D019400D1B3E086498B421C
:109CC00000D19EE04246D100802212040A43514650
:109CD000490F11438B46814952468C460099634493
:109CE000CB1A0021D20000932B0063409A460F2E1E
:109CF00000D905E17A4BB6009B599F465B4633433A
:109D0000994600D0B8E0022308260027009002936D
:109D1000CAE7CB463A0002990195019B9A4602296F
:109D200027D0032900D180E2012944D06D49009B4E
:109D30008C4663441C00002C38DD530700D013E22E
:109D4000D2085B46DB0109D55946674B19408B4663
:109D50008021C9008C46009B63441C00634B9C42DD
:109D600007DC5B4664055F075B0217431B0B620D54
:109D700002E000230027584A00211B031C0B0B0D97
:109D80001B05234314055A4A380013401C4353460D
:109D90006400DB0764081C43210005B03CBC90460E
:109DA0009946A246AB46F0BD0122524201231B1B3D
:109DB000382B00DCADE1002200230027DCE75B4606
:109DC000334399465ED0002E00D18AE1300001F085
:109DD000E7F903000B3B1C2B00DD7BE11D22D31AAE
:109DE0005A460100DA4008398E4013005F4633437B
:109DF00099468F403F4B00261B1A00930023029385
:109E000052E7414653460B433B499B468C46009BD9
:109E1000634400935B46002B3BD1022300221E4388
:109E2000022161E7434613439B4637D04346002B4C
:109E300000D162E1404601F0B3F903000B3B1C2B5B
:109E400000DD53E102004146083A914088461D2159
:109E5000CB1A5146D9400B0041460B439B46534613
:109E600093401A00009B25499C46604403008C46A1
:109E700063440093002137E70323B14600900C268A
:109E8000029311E700230093013304260027029375
:109E90000AE70323C3461E43032125E701331E437C
:109EA0000022012120E700239A46802300271B037C
:109EB000094A61E7802349461B03194200D1E2E0C9
:109EC0005946194200D0DEE00B431B0317001B0B61
:109ED000A246014A50E7C046FF07000001FCFFFF11
:109EE00040DF0000FF030000FFFFFFFEFE07000051
:109EF000FFFF0F800DFCFFFF01F8FFFFF3030000E1
:109F0000D94500D9CBE000D1C6E03C004846002747
:109F1000009B013B00935B46160E1B021E4313027F
:109F2000984633041B0C9946310C0191FFF798F8C1
:109F30004A4642430B04210C050019438A4207D9C3
:109F40008919013D8E4203D88A4201D9851E89199B
:109F5000881A0199FFF784F809048C464A462104BF
:109F600064464243090C030021438A4204D98919FB
:109F7000013B8E4200D8F1E02D041D43AB46434621
:109F8000891A4246280C12041D0C5B46140C220050
:109F90001B041B0C5A4303946B43444302956843D0
:109FA0001B19150CEB189C4203D980246402A446AB
:109FB00060441C0C15041B042D0C20185D198142F3
:109FC00077D373D00C1AA24A7D1BAF42BF4194468F
:109FD000009B7F426344E01B1C00864200D1DBE013
:109FE0000199FFF73DF84A4642430B04290C07004C
:109FF00019438A4207D98919013F8E4203D88A4200
:10A0000001D9871E8919881A0199FFF729F80904CF
:10A010004A46894629044D464243090C0300294318
:10A020008A4207D98919013B8E4203D88A4201D955
:10A03000831E89193F04891A3A00039F1A43380086
:10A0400013041B0C584381460298150C6F4343437D
:10A0500045434846000C8446DB1963449F4203D9BC
:10A06000802040028446654448461F0C00041B04BF
:10A07000000C7D191818A94200D284E000D17FE0BD
:10A0800001231A4357E680234A461B0313431B034D
:10A090001B0BAA466F4A6FE6BA4200D935E74B461A
:10A0A000DC0758087B081C43FF0734E70024AF4255
:10A0B00089D247444745A4415B466442A4196418C9
:10A0C000013BA6421ED2A0426DD800D1B6E0241AB0
:10A0D0009B4678E703005A46283B9A400027914662
:10A0E00088E6584601F05CF8203072E603005246DC
:10A0F000283B9A4093460022B4E6504601F050F8BF
:10A1000020309AE6A642E2D1B845DCD9341A9B4603
:10A1100059E71F2B65DC504C0099A4465C4661440E
:10A1200008008C4011008240D940501E82410C43EF
:10A1300014435A46DA401300620709D00F22224026
:10A14000042A05D02200141D9442894149425B181B
:10A150001A0262D50122002300270DE68A4200D8A8
:10A160000AE7831E891907E70F231340042B00D148
:10A17000E6E5171D9742924153429B44FA08E0E5F9
:10A18000002800D1D7E57118531EB14227D3A94248
:10A1900015D358D01A0073E7002B00DC04E6012326
:10A1A00000229B44CDE502234744474589415B4259
:10A1B0009C46494289190C19E344241A03E7434693
:10A1C0005F0047459B41B8465B429E19023A891998
:10A1D000A94200D054E7404500D051E7ABE51A0052
:10A1E000F6E71F215F4649420C1BE740202B07D0B2
:10A1F0001A49009B8C46634418005B4683401A430F
:10A20000501E82413A4307270023174009D00F21EF
:10A21000002311401400042995D122005F075B023E
:10A220001B0BD20817430022A6E5802359461B03C7
:10A230000B431B0317001B0B064A9DE5BD42B2D81A
:10A240009B460024BFE68045B9D31A00C3E7C04649
:10A25000FF030000FF0700001E0400003E04000092
:10A26000F0B54F464646D6468446C0B58046194EA0
:10A2700018030F034D00000B5C0082463F0B6D0D71
:10A28000C90F9146640DDB0F0120B5420AD0B442DC
:10A2900003D0A54201D157450CD01CBC904699462D
:10A2A000A246F0BD66463E43F7D1AC42F5D15446D6
:10A2B0001443F2D10120C845EFD1994207D0002DB7
:10A2C000EBD163461F433800471EB841E5E7002045
:10A2D000E3E7C046FF070000F0B54F464646D646C6
:10A2E0004D00C0B50E03C90F8A462C491F035C0000
:10A2F0008046360B6D0D91463F0B640DDB0F8D4292
:10A300001ED08C4216D0002D1ED130438446002C26
:10A3100001D13A4323D06246002A1AD09A4529D067
:10A32000514602200139084001381CBC904699462C
:10A33000A246F0BD39001143E5D002204042F4E7C7
:10A340003043FAD1AC420FD0002C0FD13A43E7D0C2
:10A350000CE00122013B934318000130E5E763461E
:10A360000020002BE1D0DBE73A43E6D19A45D7D174
:10A37000A542D5DCA54205DBBE42D1D808D00020DD
:10A38000BE42D2D250460123013898430130CCE777
:10A39000C845C5D80020C845F4D3C6E7FF0700006C
:10A3A000F0B54F464646D6464D00C0B50E03C90F20
:10A3B0008A462E491F035C008046360B6D0D914680
:10A3C0003F0B640DDB0F8D4218D08C4211D0002D55
:10A3D00018D130438446002C1ED13A431CD1634629
:10A3E0000020002B30D051460220013908400138AE
:10A3F0002AE039001143EAD0022025E03043FBD1A6
:10A40000AC4226D0002C26D13A4324D1514602201A
:10A4100001390840013817E06246002A0FD09A45FA
:10A42000E1D1A54205DBBE42DDD819D00020BE42F5
:10A430000AD25046012301389843013004E001223A
:10A44000013B9343180001301CBC90469946A2463C
:10A45000F0BD3A43D0D19A45C5D1A542C3DCE0E76F
:10A46000C845C0D80020C845E3D3EDE7FF0700008A
:10A47000F0B55746DE464E464546E0B583460600F3
:10A480000F03480087B092461D003F0B400DCC0FD4
:10A49000002800D16FE0DE4B984238D08023FF00C7
:10A4A0001B041F43730F3B430193DA4B002799466C
:10A4B00000239B46F60081442B0369001B0B524688
:10A4C0009846490DED0F002900D185E0D04B994207
:10A4D00000D173E04346DA0080231B041343524645
:10A4E000CC48520F84461343524600206144D200A8
:10A4F00089442100694000918C46012149448A46E3
:10A500000F2F00D990E0C449BF00CF59BF465B462A
:10A510003B43019300D06AE10223082700268146CD
:10A520009B46C9E732005846019B614600910228CC
:10A5300000D175E0032800D1FEE1012800D02CE114
:10A5400000230027002600253F032A0D3F0BB348B8
:10A5500012053A4302401B051343009A5B00D107E2
:10A560005B080B433000190007B03CBC904699468D
:10A57000A246AB46F0BD5B463B43019300D12FE1C1
:10A58000002F00D1A5E1380000F00AFE03000B3BCC
:10A590001C2B00DD96E11D22D31A5A460100DA4039
:10A5A0005E4608398F4013008E403B4301939C4B1D
:10A5B00000271B1A994600239B467DE741465346D8
:10A5C0000B4393498C46E144002B00D01AE1022250
:10A5D0000220174300228CE7134300D10DE14346CC
:10A5E000002B00D181E1404600F0DAFD02000B3A79
:10A5F0001C2A00DD72E10100434608398B40984671
:10A600001D239A1A5346D3401A0043461343524619
:10A610008A404946081A824989468144002068E7F1
:10A620007B4B002700268EE7140C1204120C11003D
:10A63000370C3604350C794328008C462E006043D5
:10A640006044834656432100300C80465846794387
:10A6500040440291844506D98846802149028C46AF
:10A66000E044414602913604010C360C00048B464E
:10A6700081191E0C1B041B0C0391190079438C4695
:10A68000280075436544A8465843050C4544774364
:10A69000A94203D9802149028C466744290C8C4683
:10A6A00039000004000C2D042D186144AB440591C1
:10A6B0005946049101990F043F0C080C390051438D
:10A6C0004243904602008C46090C8B4662437C4311
:10A6D00044445C44A04503D9802149028846424451
:10A6E000210C884661460904090C8C4639005943FF
:10A6F000434370437E430F0CF6182404BE19644490
:10A7000042448C46B34203D980235B0298464044BE
:10A71000029B61469846049B370443449B46AB45E5
:10A72000AD416B420D0405992D0C8C467F19674491
:10A73000FD18A8465D462D19A542A44193466442E2
:10A74000A446C344DC448F42BF4198459B41934596
:10A750009241A445A4415B427F421F43360C5242C2
:10A760006442BF192243BF18624638184302D20D13
:10A77000039913436A020A43501E82416146ED0D5C
:10A780002A434E023243D90100D4B3E001265008D7
:10A7900032400243DE0732435B08224C5444002C13
:10A7A00062DD510709D00F201040042805D0101D8C
:10A7B0009042924152429B180200D90104D5802454
:10A7C0001948E400034054441848844200DD27E758
:10A7D0005E075B02D2081F0B630516435B0DB2E6F2
:10A7E000002399460133042700269B4664E6032391
:10A7F000019781460C279B465EE601220120174304
:10A80000002276E6032303201F43434671E6C04639
:10A81000FF07000001FCFFFF80DF0000FFFF0F804B
:10A820000DFCFFFFFF030000FFFFFFFEFE0700001F
:10A830000023802700933F030026434B83E6019BC0
:10A840003200A446584670E6AC466EE68027019971
:10A850003F0339422DD03B422BD11F433F033F0BD7
:10A8600000951600384B6EE601252D1B382D00DDB6
:10A8700066E61F2D40DC35481C005044160082401F
:10A880008440EE40501E824134431443EB40620743
:10A8900009D00F222240042A05D02200141D944220
:10A8A000804140421B181A023ED501230027002692
:10A8B00049E68027019B3F031F433F033F0B009462
:10A8C000214B40E603005A46283B9A40002601925D
:10A8D0006DE6584600F064FC203057E6030052460F
:10A8E000283B9A401300002293E6504600F058FCA3
:10A8F00020307BE6CA4650E71F201E004042041B62
:10A90000E640202D03D0124C5444A3401A43501E5D
:10A910008241324307260027164009D00F2000232A
:10A92000104014000428B9D122005E075B021F0BFF
:10A93000D2081643002306E680273F031F433F0348
:10A940003F0B1600004BFEE5FF0700001E04000051
:10A950003E040000F8B557464E464546DE460C001C
:10A960000903E0B5490A460F5F0031431E03DB0FC0
:10A97000760A9B46530F3343C84E6500C000E40F70
:10A98000D2006D0DA24681467F0D9C469046B7428F
:10A9900000D1B9E05B46012673409B46EE1BA34500
:10A9A00000D183E0002E63DD002F00D0B1E06346CC
:10A9B000134300D123E1731E002B00D0BAE1861AA5
:10A9C0006346B04280410125C91A4042091A0B0270
:10A9D00000D447E149024B0A98464346002B00D178
:10A9E00089E1404600F0DCFB0300083B1F2B00DD43
:10A9F0007CE120223000D21A4146D040994002002A
:10AA00009E400A439D4200DD6AE15D1B6B1C1F2BCB
:10AA100000DD94E1202110003500C91A8E40DA4093
:10AA20008840DD40711E8E41110007222843002519
:10AA300006433240002A09D00F233340042B05D0AF
:10AA4000331DB342B641764289191E000B0200D471
:10AA50003DE26A1C914B55056D0D9A4200D119E1FA
:10AA60008F4AF6080A40570752023743120B9BE001
:10AA7000002E00D0C5E06E1C7605760D012E00DCA0
:10AA800048E16746861ACB1BB042BF417F42B846B9
:10AA90001F004346FF1A3B00B8461B0200D55FE18A
:10AAA00037439AD100220024002579E0002E00DCF3
:10AAB000FAE0002F00D18DE0784B9D4267D08023D3
:10AAC00067461B041F43BC46382E00DC52E1634638
:10AAD00013435A1E93411E18864280414042091872
:10AAE0000B0200D4BEE06D4B01359D4200D1D2E097
:10AAF0006B4A73080A4001210E401E435108D307D8
:10AB000007221E43324095E71E00164300D045E75A
:10AB100040E7624B9D423AD0802367461B041F43A7
:10AB2000BC46382E00DDEBE01F2E00DC3AE133009E
:10AB30006746203BDF403B00202E05D04027BF1B4F
:10AB40006646BE40324390464646721E96413343A7
:10AB5000DAE0002B00D114E26346134300D168E130
:10AB600080234E07C008C9081B030643194208D0BA
:10AB70006046C008184204D163460100D2085E074F
:10AB80001643F3009946C900720F444D11434B46DA
:10AB9000DE08424B4F073743CA089D4200D16EE0A2
:10ABA00012036D05120B6D0D00211203130B0A0D1C
:10ABB00012051A433B4B2D0513402B435B00E40762
:10ABC0005B082343380019003CBC90469946A246D6
:10ABD000AB46F8BD6346134311D0731E002B00D063
:10ABE00007E18618864280416144404209180125E8
:10ABF0000B0237D502257BE73E00614691463500C2
:10AC0000C5E75C46002D00D0E1E00B000343F3D024
:10AC1000731C00D1ACE1214B9F4200D13AE1F343D8
:10AC2000382B00DD6FE11F2B00DD8CE120250E00AD
:10AC3000ED1AAE40B0460600AA46DE404546354312
:10AC40002E005546D940A8406346451EA8415B1AD0
:10AC50009C463043161AB242924163465242991AB8
:10AC60003D00B4E607223240002A00D0E4E60B4B58
:10AC7000F6084F073743CA089D4200D090E73B00D3
:10AC8000134300D1A6E180231B031A431203120BC6
:10AC9000024D89E715000022002785E7FF07000025
:10ACA000FFFF7FFFFFFF0F80002E00D0C7E06B1C6F
:10ACB0005E05760D012E00DCF0E0C84DAB4200D100
:10ACC000B9E085180A008542894162444942511819
:10ACD0000722CE076D082E43490832401D00A9E621
:10ACE000BF49ED1A114007223240A3E6320028384E
:10ACF0008240002686E6300000F052FA203073E6EB
:10AD0000634613435A1E9341C61AB04280414042E3
:10AD1000091A5CE60E00674606431743002D5ED114
:10AD2000002E00D0F3E0002F00D11EE15C4661460A
:10AD300091462CE7A94FBE427BD01E00F1E61000E1
:10AD40001F3DE840202B03D04021CB1A9A401643E8
:10AD5000731E9E410722064332400021002583E7EF
:10AD6000161A6346B2428041591A40420B1A98465D
:10AD70005C4632E61F2E00DDABE02027BB1B9A4667
:10AD800063465746BB40994613004F46F3401F4366
:10AD90003B005746BA40571EBA4113436246F24041
:10ADA000891898E62027BB1B9A4663465746BB4046
:10ADB000994613004F46F3401F433B005746BA40A5
:10ADC000571EBA4113436246F240891A9CE7834BEF
:10ADD0009F425FD080252D047342294320E7002E37
:10ADE0000CD1002F00D1D0E05C46614691467B4DEE
:10ADF000CDE67A4FBE421CD01E0065E6002F18D06B
:10AE0000C0084E0706438020C9080003014208D04D
:10AE10006346DC08044204D12100DA46D2085E070A
:10AE20001643F300994601245346C900720F11439B
:10AE30001C406A4DABE61D0000220027B4E6002D41
:10AE400059D10B00034300D1D6E6731C00D1B2E008
:10AE5000624B9F421ED0F343382B6FDC1F2B00DD6B
:10AE600097E020250E00ED1AAE40B0460600AA4637
:10AE7000DE40454635432E005546A840D940451E84
:10AE8000A8418C440643B61896429241514261440F
:10AE90003D0025E63D006146914678E60B00034300
:10AEA000002D00D055E6002BF5D06346134300D1AA
:10AEB0006DE68618864280416144404209180022AE
:10AEC0000B0200D4D0E6464B01351940B2E5B1463D
:10AED0005DE633006746203BDF403B00202E05D077
:10AEE0004027BF1B6646BE40324390464646721E10
:10AEF00096413343EFE5394B9F42CBD080252D045B
:10AF000073422943A8E70843411E8841A2E6002F67
:10AF100000D13CE66346861ACF1AB0429B415B42A1
:10AF2000FB1A98461B024ED5161A6346B24292414E
:10AF3000591A5242891A5C4600227BE501430E00F1
:10AF4000711E8E419FE71D000E00203DEE40B04671
:10AF5000202B04D04025EB1A9940084381464846EF
:10AF60004346411E8841184374E60022002417E638
:10AF7000161A6346B2429241591A5242891A3D004A
:10AF800025E561469146154D01E680220024120315
:10AF900079E61D000E00203DEE40B046202B04D087
:10AFA0004025EB1A9940084381464E464346711EA0
:10AFB0008E411E4367E7861896429B4161445B427F
:10AFC000C9183D008CE547463743CED0072241469D
:10AFD000324049E600273A00E6E5C046FF07000098
:10AFE000FFFF7FFF70B50C4E0D031C0349005B0093
:10AFF0002D0B490D240B5B0DB14208D006490020F2
:10B000008B4203D114432000441EA04170BD054370
:10B010000120002DFAD1F1E7FF07000030B5144DF3
:10B020000A034B00120B5B0DC90F0024AB4211DD6C
:10B03000104CA34210DC8024640322430E4CE41A1B
:10B040001F2C0CDD0D48C31ADA4013005C420029A6
:10B0500000D11C00200030BD094BCC18FAE7094D87
:10B06000E040AC4663449A4013000343EEE7C04619
:10B07000FE0300001D040000330400001304000060
:10B08000FFFFFF7FEDFBFFFF70B500282DD0C3173A
:10B09000C5185D40C40F280000F082F8154B1B1A3C
:10B0A0005B055B0D0A2815DD0B38854000222D035A
:10B0B0002D0B002110002D030A0D2D0B12052A4324
:10B0C0000D4D1B052A4013435B00E4075B08234337
:10B0D000190070BD02002900153291400A000B21B1
:10B0E000081AC5402D032D0BE3E70024002300259B
:10B0F0000022DEE71E040000FFFF0F804100090E62
:10B100004B1C70B5DBB24602750AC40F012B14DD6F
:10B11000E0239B006D07360BCB1800210A0D280099
:10B1200012051C4D32435B052A405B0813435B004C
:10B13000E4075B082343190070BD002914D1002DDA
:10B140001ED0280000F02CF80A281CDC0B232A0053
:10B150001B1ADA40030015339D400F4B12031B1AD4
:10B160005B05160B5B0DD8E7002D06D0320B802651
:10B1700036036D071643094BCFE7084B0026CCE793
:10B1800000230026C9E703002A000B3B9A40002554
:10B19000E3E7C046FFFF0F8089030000FF070000C0
:10B1A0001C2101231B04984201D3000C10391B0AF7
:10B1B000984201D3000A08391B09984201D30009BB
:10B1C000043902A2105C40187047C0460403020212
:10B1D00001010101000000000000000030B51C006A
:10B1E000094B05001B6885B0D868084B002A01D1BF
:10B1F000074B1A000292019300912B00220005498F
:10B2000000F026F800F0A6FD7C000020C0DF000062
:10B21000D6CD0000CDDF0000014B18687047C04656
:10B220007C000020084B10B50400002B02D0002148
:10B2300000E000BF054B1868836A002B00D09847D8
:10B24000200001F05DFBC04600000000FCDF0000B4
:10B250000EB403B5010003AB044804CB00680193AE
:10B2600000F076F802B008BC03B018477C0000205C
:10B2700070B500260C4D0D4C641BA410A64209D1DC
:10B28000002601F03FFB0A4D0A4C641BA410A642A5
:10B2900005D170BDB300EB5898470136EEE7B30017
:10B2A000EB5898470136F2E74C0200204C02002090
:10B2B0004C0200205C020020002310B59A4200D10D
:10B2C00010BDCC5CC4540133F8E710B5884202D9F4
:10B2D0008B18984203D3002307E08B5C8354013A18
:10B2E000FBD210BDCC5CC45401339A42FAD1F8E7CA
:10B2F00003001218934200D1704719700133F9E727
:10B30000936810B5013B9360002B04DA9469A34263
:10B3100007DB0A2905D01368581C10601970080053
:10B3200010BD00F04BFC0100F9E7F8B506000F0076
:10B330001400D518AC4201D1002007E021783A0072
:10B340003000FFF7DDFF0134431CF3D1F8BD0000EE
:10B35000F0B59FB002900F0016000593002805D0AD
:10B3600083690493002B01D100F0F4FD7B4B9F42D5
:10B370005BD1029B5F68BB891B0762D53B69002BD1
:10B380005FD0002306AC6361203363761033A3766D
:10B3900035002B78002B01D0252B5CD1AB1B0493FF
:10B3A0000CD0320039000298FFF7BFFF431C00D1D8
:10B3B000C4E06269049B9446634463612B78002B6C
:10B3C00000D1BBE0012200235242626002A9543244
:10B3D00052186E1C2360E360A3601370A36531787C
:10B3E00005225F4800F0D4FE751C002835D1226884
:10B3F000D30604D5532302A95B1820211970130723
:10B4000004D5532302A95B182B21197033782A2BFA
:10B410002CD0350000210A20E3682A786E1C303ACF
:10B42000092A64D900292ED026E04E4B9F4202D132
:10B43000029B9F689FE74C4B9F429CD1029BDF6819
:10B4400099E73900029800F00FFC002899D00120FC
:10B4500040421FB0F0BD01359BE7414B2268C01A46
:10B4600001238340134323602E00B8E7059B191D79
:10B470001B680591002B01DB099304E05B42E3604C
:10B480000223134323602B782E2B0AD16B782A2BAF
:10B4900035D1059B02351A1D1B680592002B2BDB4D
:10B4A0000793324E29780322300000F071FE002805
:10B4B00006D04023801B834022680135134323605C
:10B4C000297806222A486E1C217600F061FE0028A9
:10B4D0003AD0284B002B25D10722059B07339343F5
:10B4E000083305936369039A9B18636150E74343EC
:10B4F00001219B18350090E701235B42D0E7002330
:10B500000A201A000135636029786E1C3039092938
:10B5100003D9002BC5D00792C3E742430123521839
:10B520003500F1E705AB00933A00134B2100029878
:10B5300000E000BF0390039B0133D3D1BB895B06BE
:10B5400000D584E70B9884E705AB00933A000A4BDB
:10B550002100029800F080F8ECE7C04654E00000BB
:10B5600000E0000074E0000034E0000006E00000AD
:10B570000AE00000000000002BB30000F7B5150042
:10B5800001938A680B6900900C00934200DA130063
:10B5900022002B6043321278002A01D001332B6045
:10B5A00023689B0602D52B6802332B60062723688D
:10B5B0001F4027D0230043331B785A1E9341226833
:10B5C000920630D42200019943320098089EB04779
:10B5D000431C25D0062320682A68E1680340002523
:10B5E000042B03D18D1AEB43DB171D40A36822699E
:10B5F000934201DD9B1AED180027BD4220D10020A7
:10B6000010E00137E3682A689B1ABB42D2DD2200B2
:10B610000123193201990098089EB047431CF0D1CC
:10B6200001204042FEBD3020E11843310870210066
:10B630005A1C45310978A218433202331170C1E710
:10B64000220001231A3201990098089EB047431C3A
:10B65000E6D00137D1E70000F0B589B004920A00C6
:10B6600043320593039002920A7E0C000E9B6E2AD1
:10B6700000D186E01FD8632A33D008D8002A00D131
:10B680008CE0582A4DD0250042352A7030E0642ADB
:10B6900001D0692AF7D1196825680A1D280629D51D
:10B6A00008681A60002803DA2D23029A40421370BA
:10B6B0006B4E0A274FE0732A74D008D86F2A1FD028
:10B6C000702AE0D1202209680A43226003E0752A2B
:10B6D00016D0782AD7D12200782145321170614ED8
:10B6E00022E025001A684235111D196013682B707D
:10B6F000012365E008681A606906D3D500B2D1E776
:10B7000019682568081D186008682E0605D5544E6E
:10B7100008276F2A1BD00A2719E06D06F7D580B2DB
:10B72000F5E745314E4E0A7018682268011D006821
:10B730001960150621D5D30702D520231A432260AC
:10B740001027002803D1202322689A432260230077
:10B75000002243331A706368A360002B58DB042275
:10B76000216891432160002854D1029D002B5AD0BA
:10B770002500337842352B7055E05506DBD580B275
:10B78000D9E71A680D68101D4969186013682E06FC
:10B7900001D5196002E06D06FBD519800023029DDA
:10B7A00023614FE01A68111D196015680021626855
:10B7B000280000F0EDFC002801D0401B60606368A9
:10B7C00023610023029A13703CE023692A00049944
:10B7D0000398059DA847431C3ED023689B0715D4BA
:10B7E000079BE068984239DA180037E0220001230D
:10B7F000193204990398059EB047431C2CD001359B
:10B80000E368079A9B1AAB42F0DCE9E70025F7E70B
:10B810000028ADD0029D3900FDF722FC735C013D8C
:10B820002B700028F7D1082F09D12368DB0706D534
:10B8300063682269934202DC3023013D2B70029B36
:10B840005B1B2361059B07AA00932100049B0398BF
:10B85000FFF794FE431CB8D10120404209B0F0BD6F
:10B8600011E0000022E000000D4B70B51C680500DF
:10B87000A36B002B0FD1182000F06EFC094BA063C6
:10B880000360094B01224360084B83600B238381D3
:10B890000023026143610022A36B1D615A6170BDE8
:10B8A0007C0000200E33CDAB34126DE6ECDE0500DB
:10B8B000124B10B51C68A36B002B0FD1182000F0A1
:10B8C0004BFC0F4BA06303600E4B012243600E4BF9
:10B8D00083600B238381002302614361A46B0B4AC5
:10B8E000206961690A4BFDF7F7FC012200238018EB
:10B8F0005941206161614800400810BD7C00002072
:10B900000E33CDAB34126DE6ECDE05002D7F954C89
:10B910002DF451580CB430B5164B9DB00C1E1D685B
:10B9200008DA8B2301202B6040421DB030BC08BCDC
:10B9300002B01847822302A99B008B81002302904A
:10B9400008619C4200D0631E8B604B6101235B4207
:10B95000CB81209A21AB2800019300F055FD431CB8
:10B9600001DA8B232B60002CDFD00023029A1370A6
:10B97000DBE7C0467C0000200EB400B50B499CB04C
:10B980001DAB02900690079104910948094904CB28
:10B990000591006802A9019300F036FD0023029A88
:10B9A00013701CB008BC03B01847C046FFFFFF7FF0
:10B9B0007C0000200802FFFF020010B51378541C21
:10B9C000002B05D1CC5CD4540133002CFAD110BD2E
:10B9D0002200F3E7C9B20378002B04D08B4200D1D8
:10B9E00070470130F7E74B42594149420840F7E7B9
:10B9F00002780B78002A03D0013001319A42F7D047
:10BA0000D01A70470023C25C0133002AFBD1581EB4
:10BA10007047002330B59A420AD0013AC45CCD5C2D
:10BA2000AC4204D1934202D00133002CF6D1631B07
:10BA3000180030BD30B50500002A00D130BD0C78AB
:10BA4000013A6B1C2C700131002C05D19A189A42D6
:10BA5000F4D01C700133FAE71D00EDE710B5037850
:10BA6000002B0FD10B785A4253415B42184010BD56
:10BA70000023CA5C002AFAD0C45C944201D101338D
:10BA8000F7E701300378002BF2D11800EFE7000050
:10BA9000F0B51F000E0087B00590019102920C983E
:10BAA000347800F0EAFA082200194378751C134034
:10BAB00036D12D2C36D1B51C74780126002F62D0DA
:10BAC000102F09D1302C07D120222B789343582BEB
:10BAD00054D110276C7802352D4B3900F31818001B
:10BAE0000393FDF7BDFA04910121002349420200AE
:10BAF0008C4618002100303909291AD80C00A742B9
:10BB000023DD591C09D06346824206D302D1049931
:10BB1000A14202DB0123784320182C780135E9E7A4
:10BB20002E00BCE72B2C01D01E00C7E7B51C747893
:10BB3000FAE721004139192901D8373CDFE7210014
:10BB40006139192901D8573CD9E75A1C08D1059AFF
:10BB500023331360029B0398002B09D107B0F0BD7B
:10BB6000002E00D04042029A002AF7D0002B01D0CC
:10BB70006B1E0193029B019A1A60EFE73024002F9D
:10BB8000AAD10827A8E7302C9ED00A27A4E7C046F0
:10BB9000FFFFFF7F37B51300064A05001068046AEF
:10BBA000002C00D1044C0A0000942900FFF770FF1C
:10BBB0003EBDC0467C000020E0000020F8B5050036
:10BBC0000E001400002804D08369002B01D100F07E
:10BBD000C1F9224B9C422DD16C68A369A360A38953
:10BBE0001B0731D52369002B2ED023682269F7B2B9
:10BBF000981A6369F6B2834205DC2100280000F040
:10BC00003BF9002826D1A3680130013BA3602368DB
:10BC10005A1C22601F706369834204D0A389DB072A
:10BC20001AD50A2E18D12100280000F025F9002885
:10BC300012D00FE00A4B9C4201D1AC68CDE7094B12
:10BC40009C42CAD1EC68C8E72100280000F00CF83B
:10BC50000028CAD0012676423000F8BD54E000002A
:10BC600074E0000034E00000364B70B51D6806003B
:10BC70000C00002D05D0AB69002B02D1280000F08C
:10BC800069F9314B9C420FD16C680C23E25E93B290
:10BC900019072DD4D90611D4092301203360373375
:10BCA0001343A381404270BD284B9C4201D1AC6834
:10BCB000EBE7274B9C42E8D1EC68E6E75B0713D53E
:10BCC000616B002908D023004433994202D0300030
:10BCD00000F06AFA002363632422A3899343A381BB
:10BCE00000236360236923600823A2891343A3818F
:10BCF0002369002B0BD1A0218022A3898900920007
:10BD00000B40934203D02100300000F0E1F9012301
:10BD1000A289134011D00023A36063695B42A36131
:10BD2000002023698342BED10C23E25E1306BAD5FC
:10BD300040231343A3810138B5E7920700D4636918
:10BD4000A360EDE77C00002054E0000074E00000F8
:10BD500034E0000010B5062000F090FC012000F057
:10BD6000CFFD0000F7B58A8905000C00130760D4E9
:10BD70004B68002B04DC0B6C002B01DC0020FEBDAB
:10BD8000E76A002FFAD000232E682B6080235B0126
:10BD9000216A1A4034D0606DA3895B0706D56368B9
:10BDA000C01A636B002B01D0236CC01A0200216AF9
:10BDB00000232800E76AB847A189431C06D12B68F5
:10BDC0001D2B30D82B4ADA40D3072CD500236360D3
:10BDD00023692360CB0405D5431C02D12B68002BBB
:10BDE00000D16065616B2E600029C7D02300443309
:10BDF000994202D0280000F0D7F900206063BEE726
:10BE000001232800B847431CC6D12B68002BC3D0A0
:10BE10001D2B01D0162B01D12E60AFE74023A28944
:10BE20001343A381ABE740230B430120A38140428E
:10BE3000A5E70F69002FA1D00B680F60DB1B0193F2
:10BE40000023920700D14B69A360019B002B00DC0B
:10BE500094E7019B3A00216A2800A66AB0470028AF
:10BE600003DC4023A2891343DFE7019B3F181B1A21
:10BE70000193EAE7010040200B6970B505000C0052
:10BE8000002B01D1002070BD002804D08369002B55
:10BE900001D100F05FF80B4B9C4209D16C680C2279
:10BEA000A35E002BEED021002800FFF75BFFEAE73E
:10BEB000054B9C4201D1AC68F1E7044B9C42EED1AA
:10BEC000EC68ECE754E0000074E0000034E00000AF
:10BED000002310B5040003604360836081814366E2
:10BEE000C281036143618361190008225C30FFF75E
:10BEF000FFF9054B24626362044BA362044BE362C7
:10BF0000044B236310BDC046BDC60000E5C600005B
:10BF10001DC7000049C7000010B5024900F08CF8A9
:10BF200010BDC04679BE000070B568254A1E554355
:10BF30000E002900743100F081F9041E08D00021A0
:10BF40002A00016046600C30A0606832FFF7D0F92B
:10BF5000200070BD836913B50400002B28D18364D1
:10BF6000C3640365134B144A1B68826201939842B1
:10BF700001D101238361200000F020F860602000DF
:10BF800000F01CF8A060200000F018F80022E0602B
:10BF900004216068FFF79CFF01220921A068FFF7D8
:10BFA00097FF02221221E068FFF792FF0123A361AD
:10BFB00013BDC046FCDF000019BF0000F8B51C4BE4
:10BFC00007001E68B369002B02D13000FFF7C2FFE3
:10BFD0004836B4687368013B04D53368002B07D03A
:10BFE0003668F6E70C22A55E002D0DD06834F2E726
:10BFF00004213800FFF798FF30600028F0D10C23AF
:10C0000004003B602000F8BD20000A4B65662560F7
:10C010006560A560E36025616561A561082229006E
:10C020005C30FFF765F96563A563A564E564E9E73E
:10C03000FCDF00000100FFFFF7B504000700002649
:10C0400001914834002C01D13000FEBD6368A56821
:10C050000093009B013B009301D52468F2E7AB8974
:10C06000012B08D90E22AB5E013304D02900380021
:10C07000019B984706436835EBE7EC300068704752
:10C0800070B50E001D000E23C95E96B01400002985
:10C0900007DA00232B60B3891B0611D48023DB0051
:10C0A0000FE06A4600F088FB0028F2DBF022019BDB
:10C0B00012021340054A9B185A4253412B60EDE788
:10C0C00040230020236016B070BDC04600E0FFFF93
:10C0D000F7B502268B8905000C00334206D02300F9
:10C0E00047332360236101236361F7BD01AB6A46D7
:10C0F000FFF7C6FF00990700280000F09FF800280E
:10C1000008D10C22A35E9A05EFD4032293431E4369
:10C11000A681E4E70F4BAB628023A2892060134322
:10C12000A381009B20616361019B002B0DD00E2336
:10C13000E15E280000F052FB002806D00322A3890C
:10C1400093431A0001231343A381A0893843A0819C
:10C15000CBE7C04619BF000010B5034B01001868BB
:10C1600000F06CF810BDC0467C00002082B00029B1
:10C1700000D101A9101E06D0002B06D013780B6049
:10C180001078431E984102B0704702204042FAE7FF
:10C19000C9B28218904201D10020704703788B42C7
:10C1A000FBD00130F6E7000070B50500002910D083
:10C1B0000C1F2368002B00DAE418280000F034FB81
:10C1C0001D4A1368002B05D163601460280000F03D
:10C1D0002CFB70BDA34209D9216860188342F3D1BA
:10C1E00018685B6841182160EEE713005A68002A5E
:10C1F00001D0A242F9D919685818A0420BD1206881
:10C200000918581819608242E0D110685268411824
:10C2100019605A60DAE7A04202D90C232B60D5E7F7
:10C2200021686018824203D1106852684118216069
:10C2300062605C60CAE7C046181C0020032370B52A
:10C24000CD1C9D43083506000C2D1ED20C25A9429D
:10C250001DD8300000F0E8FA254A146821000029B2
:10C2600019D1244C2368002B03D1300000F0CAF907
:10C2700020602900300000F0C5F9431C2BD10C23AD
:10C280003000336000F0D1FA03E0002DDFDA0C2338
:10C290003360002070BD0B685B1B19D40B2B03D9D6
:10C2A0000B60CC18256003E04B688C420DD1136005
:10C2B000300000F0BAFA200007220B30231D904313
:10C2C000C31AE7D05A42E250E4E763600C00EFE79C
:10C2D0000C004968C3E70323C41C9C43A042E1D07F
:10C2E000211A300000F08EF9431CDBD1C7E7C046AD
:10C2F000181C00201C1C0020F8B507000D001600BB
:10C30000002905D11100FFF799FF04002000F8BDB6
:10C31000002A03D1FFF748FF3400F7E700F086FA60
:10C320002C00B042F2D231003800FFF787FF041E24
:10C33000ECD029003200FEF7BFFF29003800FFF7DC
:10C3400033FFE3E7F0B58E6885B007000C00039279
:10C3500001939E423CD890238A89DB001A4234D054
:10C360000325096923685B1A0293636902985D4398
:10C37000EB0F5D19019B6D1001331B18AB4200D907
:10C380001D00530532D529003800FFF757FF061E60
:10C3900009D10C233B6040230120A2894042134372
:10C3A000A38105B0F0BD029A2169FEF785FFA3893C
:10C3B000144A1A4080231343A381029B2661F61876
:10C3C00026606561019EED1AA560019B9E4200D921
:10C3D000019E320003992068FEF777FFA3680020D2
:10C3E0009B1BA36023689E192660DAE72A003800A9
:10C3F000FFF782FF061EE0D121693800FFF7D4FE67
:10C40000C7E7C0467FFBFFFFF0B59FB002900593E2
:10C410008B890F0016001B0611D50B69002B0ED15E
:10C420004021FFF70BFF38603861002805D10C234D
:10C43000029A013813601FB0F0BD40237B610023D6
:10C4400006AC6361203363761033A37635002B7816
:10C45000002B01D0252B46D1AB1B04930CD032000E
:10C4600039000298FFF76EFF431C00D1AEE062690D
:10C47000049B9446634463612B78002B00D1A5E0B4
:10C48000012200235242626002A9543252186E1CEB
:10C490002360E360A3601370A365317805225448DC
:10C4A000FFF776FE751C00281FD12268D30604D53D
:10C4B000532302A95B1820211970130704D55323B5
:10C4C00002A95B182B21197033782A2B16D035005E
:10C4D00000210A20E3682A786E1C303A092A4ED9D6
:10C4E000002918D010E00135B1E7414B2268C01A8D
:10C4F00001238340134323602E00CEE7059B191DC3
:10C500001B680591002B01DB099304E05B42E360AB
:10C510000223134323602B782E2B0AD16B782A2B0E
:10C5200035D1059B02351A1D1B680592002B2BDBAC
:10C530000793304E297803223000FFF729FE0028A8
:10C5400006D04023801B83402268013513432360BB
:10C550002978062228486E1C2176FFF719FE00284C
:10C560003CD0264B002B25D10722059B0733934354
:10C57000083305936369039A9B18636166E7434335
:10C5800001219B183500A6E701235B42D0E7002379
:10C590000A201A000135636029786E1C3039092998
:10C5A00003D9002BC5D00792C3E742430123521899
:10C5B0003500F1E705AB00933A00114B21000298DA
:10C5C00000E000BF0390039B0133D3D1BB890B98DC
:10C5D0005B0600D42FE7012040422CE705AB009317
:10C5E0003A00074B21000298FFF736F8EAE7C04609
:10C5F00000E0000006E000000AE00000000000008B
:10C6000045C30000002370B5064C050008002360F8
:10C6100000F060F9431C03D12368002B00D02B608D
:10C6200070BDC046AC2F002070B504000D001F295E
:10C6300004D9162303600120404270BD436C002BD7
:10C6400004D08A009B181A68002A08D1200000F044
:10C6500031F82A000100200000F01AF8EDE7002070
:10C66000012AEAD0511C03D1162301302360E4E7EC
:10C67000002428001C6090472000DEE710B5034B23
:10C6800001001868FFF7D0FF10BDC0467C000020F5
:10C69000002370B5064C050008001100236000F06F
:10C6A00001F9431C03D12368002B00D02B6070BD1F
:10C6B000AC2F002010B500F0E5F810BD70B50C00EF
:10C6C0000E25495F00F0BAF8002803DB636D1B18E4
:10C6D000636570BDA389024A1340A381F9E7C04690
:10C6E000FFEFFFFFF8B51F008B8905000C00160057
:10C6F000DB0505D50E23C95E0022022300F080F879
:10C70000A389054A28001340A38132000E23E15E6D
:10C710003B0000F02BF8F8BDFFEFFFFF70B50C00F9
:10C720000E25495F00F06CF8A389421C03D1054A2D
:10C730001340A38170BD802252011343A381606521
:10C74000F8E7C046FFEFFFFF10B50E23C95E00F00B
:10C7500021F810BD0B1E04D0FF2A04D98A230360E0
:10C760008B3B180070470A700123FAE770B505008B
:10C77000080011000022064C22601A0000F0B8F8F0
:10C78000431C03D12368002B00D02B6070BDC04632
:10C79000AC2F0020002370B5064C05000800236074
:10C7A00000F060F8431C03D12368002B00D02B60FD
:10C7B00070BDC046AC2F0020002370B5064C0500AC
:10C7C00008001100236000F055F8431C03D12368D2
:10C7D000002B00D02B6070BDAC2F0020002370B563
:10C7E000064C05000800236000F054F8431C03D1F8
:10C7F0002368002B00D02B6070BDC046AC2F0020FA
:10C8000070B50500080011000022064C22601A00D5
:10C8100000F050F8431C03D12368002B00D02B609C
:10C8200070BDC046AC2F0020704770470B1F1B68BF
:10C83000181F002B01DA0B58C018704770B505009F
:10C84000080011000022064C22601A0000F03AF89D
:10C85000431C03D12368002B00D02B6070BDC04661
:10C86000AC2F002058220120014B40421A60704733
:10C87000AC2F002058220120014B40421A60704723
:10C88000AC2F002058220120014B40421A60704713
:10C89000AC2F00205822024B00201A607047C0467F
:10C8A000AC2F002058220120014B40421A607047F3
:10C8B000AC2F002058220120014B40421A607047E3
:10C8C000AC2F002058220120014B40421A607047D3
:10C8D000AC2F0020044A1368002B00D1034B18181A
:10C8E000106018007047C046201C0020B02F0020A8
:10C8F00058220120014B40421A607047AC2F0020A3
:10C90000FEE7C046F8B5C046F8BC08BC9E46704776
:10C91000F8B5C046F8BC08BC9E46704764617461B7
:10C9200000000000A0C90000EF010000A9C900003C
:10C93000E3020000B1C9000001090000B8C900000D
:10C94000110A0000BDC9000029050000C8C9000087
:10C9500053030000CDC900007D0C0000D9C90000C0
:10C960001F020000E3C9000009080000F1C900002F
:10C97000B5060000FEC90000E904000072616E64A3
:10C980006F6D00616C6C006C6173740066616C7338
:10C9900065007472756500252E3135732E2E2E00BC
:10C9A0006D616B654C697374006164644C61737490
:10C9B0000064656C657465006A6F696E00636F7012
:10C9C0007946726F6D546F0066696E64006A6F69B4
:10C9D0006E537472696E677300756E69636F646518
:10C9E000417400756E69636F6465537472696E6734
:10C9F000006E657742797465417272617900667282
:10CA000065654D656D6F72790000000069CA0000B0
:10CA1000E51000006ECA0000F1100000B1C900006E
:10CA2000F510000074CA0000F91000007ECA000072
:10CA3000FD10000087CA00000111000091CA00002B
:10CA4000051100009CCA000009110000A8CA0000DE
:10CA50000D110000B2CA0000E9100000BDCA0000BC
:10CA6000ED10000066696C65006F70656E00636CA8
:10CA70006F736500656E644F6646696C650072652C
:10CA800061644C696E6500726561644279746573B6
:10CA900000617070656E644C696E650061707065F0
:10CAA0006E6442797465730073746172744C697357
:10CAB00074006E657874496E4C6973740073797391
:10CAC00074656D496E666F001C1300002C13000026
:10CAD00046130000C4130000FC13000032140000D1
:10CAE0006A14000090140000CC1400000E15000021
:10CAF00064150000A8150000141600005C16000064
:10CB000082160000BA160000001700002617000069
:10CB10005417000086170000BE17000042180000DE
:10CB20000A19000080190000EC190000381A0000F2
:10CB3000581A00007A1A00002C1B0000721B00001B
:10CB4000EA1B00001C1300001C130000181C00004E
:10CB5000801C0000041D00004A1D0000921D000002
:10CB6000081E00007E1E0000C61E00000C1F0000F4
:10CB7000421F0000881F0000CE1F0000162000008A
:10CB80006A200000C820000006210000702100007B
:10CB9000A6210000EE210000362200007E220000C7
:10CBA000B82200000023000048230000B424000045
:10CBB0001C1300001C130000B02300001C13000015
:10CBC000E623000012240000482400007424000022
:10CBD0001C1300001C1300001C1300001C13000099
:10CBE0002A2500006C2500001C1300001C13000007
:10CBF000B225000002260000282600001C130000B9
:10CC00001C1300001C13000056260000862600009E
:10CC1000B6260000EC260000162700004C27000076
:10CC2000762700009E270000C6270000F627000098
:10CC300026280000502800007A280000D428000090
:10CC4000FE2800001C1300001C1300001C13000031
:10CC50001C1300001C1300002E2900005A2900009C
:10CC600086290000B2290000DE290000142A0000F5
:10CC70004A2A0000802A0000B62A0000E22A0000AA
:10CC80000E2B0000442B00001C1300001C1300009E
:10CC90001C1300001C1300001C1300001C130000D8
:10CCA0001C1300001C1300001C1300001C130000C8
:10CCB0001C1300001C1300001C1300001C130000B8
:10CCC000702B0000A62B0000282564206974656D78
:10CCD000206C6973742900286F626A65637420741C
:10CCE0007970653A2025642900537461636B20755F
:10CCF0006E646572666C6F7700626F6F6C65616EF3
:10CD0000006E756D62657200737472696E67006C97
:10CD10006973740007000000030000005DCD00008F
:10CD2000C92C000065CD0000792D00006ECD0000FB
:10CD3000112E000077CD0000CD2C00001500000062
:10CD400001000000020000000400000005000000D7
:10CD50000600000043616C6C696F70650068617368
:10CD6000546F6E6500706C6179546F6E6500686118
:10CD700073536572766F00736574536572766F00D6
:10CD8000474320746F6F6B20256420757365637350
:10CD90003B206672656520256420776F726473009E
:10CDA0003C496E74656765723E003C4C6973743E25
:10CDB000003C4F626A6563743E003C427974654191
:10CDC000727261793E000D0A564D2050616E6963A2
:10CDD0003A2025730D0A006D6973630011CE0000BF
:10CDE000B93A00001ACE0000513A00001ECE0000F1
:10CDF000A539000026CE00004B39000030CE0000DF
:10CE0000E13800003CCE0000E33700006E756C6C2A
:10CE100000686578546F496E740073696E006A73B8
:10CE20006F6E476574006A736F6E436F756E740042
:10CE30006A736F6E56616C75654174006A736F6ECC
:10CE40004B65794174000000BCCE0000253B00001A
:10CE5000C4CE0000293B0000CECE0000473B0000BE
:10CE6000D7CE0000513B0000E2CE00005B3B00004B
:10CE7000EECE0000653B0000FECE00006F3B0000E0
:10CE80000ECF0000793B000023CF0000833B000061
:10CE900038CF00008D3B000044CF0000973B0000DE
:10CEA00054CF0000A13B000060CF0000333B0000E6
:10CEB0006DCF00003D3B00006E65740068617357E4
:10CEC00069466900737461727457694669007374C6
:10CED0006F70576946690077696669537461747544
:10CEE00073006D79495041646472657373007374A3
:10CEF00061727448747470536572766572007374ED
:10CF00006F707448747470536572766572006874DB
:10CF10007470536572766572476574526571756594
:10CF2000737400726573706F6E64546F48747470BC
:10CF3000526571756573740068747470436F6E6EBA
:10CF400065637400687474704973436F6E6E6563D3
:10CF500074656400687474705265717565737400EB
:10CF600068747470526573706F6E73650068747462
:10CF700070436C6F7365000D0E0F04050C0B0A06F1
:10CF8000070809000000000008080800080A4A40D5
:10CF900000000A5FEA5FEA0ED92ED36E1932448987
:10CFA000330C924C924D08080000000488080804D5
:10CFB0000804848488000A448A4000048EC48000E7
:10CFC0000000048800000EC00000000008000122DC
:10CFD0004488100C9252524C048C84848E1C824CD7
:10CFE000901E1EC244924C06CA525FE21FF01EC140
:10CFF0003E02448ED12E1FE24488100ED12ED12E37
:10D000000ED12EC4880008000800000480048802A5
:10D0100044880482000EC00EC008048244880ED1E9
:10D0200026C0040ED135B36C0C925ED2521C925CB9
:10D03000925C0ED010100E1C9252525C1ED01C90AE
:10D040001E1ED01C90100ED013712E12525ED252A2
:10D050001C8808081C1FE242524C1254981492106B
:10D060001010101E113B75B131113935B3710C928E
:10D0700052524C1C925C90100C92524C861C925C4A
:10D0800092510ED00C825C1FE4848484125252525E
:10D090004C1131312A44113135BB7112524C92522C
:10D0A000112A4484841EC488101E0EC808080E105D
:10D0B000080482410EC242424E048A400000000031
:10D0C00000001F0804800000000ED2524F10101CF8
:10D0D000925C000ED0100E02424ED24E0C925C902A
:10D0E0000E06C81C88080ED24EC24C10101C92525C
:10D0F0000800080808024002424C101498149208D4
:10D1000008080806001B75B131001C925252000C31
:10D1100092524C001C925C90000ED24EC2000ED077
:10D1200010100006C8049808080EC80700125252D2
:10D130004F0011312A4400113135BB00124C8C9242
:10D1400000112A4498001EC4881E06C48C848608D8
:10D150000808080818080C881800000C83600000F4
:10D1600000000000010000000200000003000000B9
:10D170000400000005000000060000000700000099
:10D1800008000000090000000A0000000B00000079
:10D190000C0000000D0000000E0000000F00000059
:10D1A0001000000012000000140000001600000033
:10D1B000180000001A0000001C0000001E00000003
:10D1C00020000000230000002600000029000000CD
:10D1D0002C0000002F00000032000000360000008C
:10D1E0003A0000003E00000042000000460000003F
:10D1F0004B00000050000000550000005A000000E5
:10D2000061000000680000006F0000007600000070
:10D210007D000000840000008B00000092000000F0
:10D2200099000000A0000000A7000000AE00000070
:10D23000B5000000BC000000C3000000CA000000F0
:10D24000D1000000D8000000DF000000E600000070
:10D25000ED000000F4000000FB000000FF000000F3
:10D26000B0D20000C53B0000BBD200000D41000061
:10D27000C5D20000813D0000D2D200007D3F0000F9
:10D28000D9D20000CD3F0000E2D200001D400000D6
:10D29000EED20000153F0000FFD20000F13D00007B
:10D2A0000CD30000AD3E0000646973706C617900BE
:10D2B0006C696768744C6576656C006D624469736F
:10D2C000706C6179006D62446973706C61794F664E
:10D2D00066006D62506C6F74006D62556E706C6F9D
:10D2E00074006D62447261775368617065006D62AD
:10D2F0005368617065466F724C6574746572006E38
:10D30000656F506978656C53656E64006E656F502B
:10D310006978656C53657450696E004E6F74206552
:10D320006E6F75676820726F6F6D206576656E2011
:10D33000616674657220636F6D70616374696F6E8E
:10D3400000436F6D70616374656420466C6173683F
:10D3500020636F64652073746F72650A25642062B0
:10D3600079746573207573656420282564252529E3
:10D37000206F6620256400426164207265636F72CD
:10D380006420666F756E6420647572696E672069CB
:10D390006E697469616C697A6174696F6E00256485
:10D3A0002025642025642028256420776F7264730B
:10D3B00029002564207265636F7264732C202564D4
:10D3C00020776F7264732C206D6178494420256446
:10D3D0002C20636F6D70616374696F6E2063796375
:10D3E0006C657320256400526573746F72656420E8
:10D3F000256420736372697074730053746172746E
:10D40000656400726164696F000000009CD40000D4
:10D41000DD4A0000A9D40000794D0000B9D4000015
:10D42000F94C0000C7D400000D4F0000D2D400001A
:10D43000054B0000E2D400008D4B0000F6D4000044
:10D44000754B000005D50000EF50000011D500001D
:10D450006D5000001AD500001150000025D50000C5
:10D46000594F000030D50000954F000039D500001D
:10D47000C94F000042D50000154B000051D50000F7
:10D48000F54A00005AD50000254B00006E6F6E650E
:10D49000006F74686572007061697200646973611D
:10D4A000626C65526164696F006D65737361676575
:10D4B0005265636569766564007061636B6574527B
:10D4C000656365697665007061636B657453656E4D
:10D4D00064007265636569766564496E7465676545
:10D4E000720072656365697665644D657373616723
:10D4F0006554797065007265636569766564537417
:10D5000072696E670073656E64496E7465676572F3
:10D510000073656E64506169720073656E64537464
:10D5200072696E67007365744368616E6E656C0046
:10D5300073657447726F757000736574506F7765AB
:10D5400072007369676E616C537472656E6774689C
:10D55000006465766963654944006C6173744D6568
:10D5600073736167654944000000000096300777D7
:10D570002C610EEEBA51099919C46D078FF46A70C7
:10D5800035A563E9A395649E3288DB0EA4B8DC79E7
:10D590001EE9D5E088D9D2972B4CB609BD7CB17E67
:10D5A000072DB8E7911DBF906410B71DF220B06A37
:10D5B0004871B9F3DE41BE847DD4DA1AEBE4DD6D47
:10D5C00051B5D4F4C785D38356986C13C0A86B6447
:10D5D0007AF962FDECC9658A4F5C0114D96C066367
:10D5E000633D0FFAF50D088DC8206E3B5E10694C47
:10D5F000E44160D5727167A2D1E4033C47D4044B87
:10D60000FD850DD26BB50AA5FAA8B5356C98B24266
:10D61000D6C9BBDB40F9BCACE36CD832755CDF45E6
:10D62000CF0DD6DC593DD1ABAC30D9263A00DE5116
:10D630008051D7C81661D0BFB5F4B42123C4B35606
:10D640009995BACF0FA5BDB89EB802280888055F86
:10D65000B2D90CC624E90BB1877C6F2F114C6858E6
:10D66000AB1D61C13D2D66B69041DC760671DB01D4
:10D67000BC20D2982A10D5EF8985B1711FB5B606A6
:10D68000A5E4BF9F33D4B8E8A2C9077834F9000FE6
:10D690008EA8099618980EE1BB0D6A7F2D3D6D0886
:10D6A000976C6491015C63E6F4516B6B62616C1C76
:10D6B000D83065854E0062F2ED95066C7BA5011BA6
:10D6C000C1F4088257C40FF5C6D9B06550E9B71246
:10D6D000EAB8BE8B7C88B9FCDF1DDD62492DDA1506
:10D6E000F37CD38C654CD4FB5861B24DCE51B53A26
:10D6F0007400BCA3E230BBD441A5DF4AD795D83D26
:10D700006DC4D1A4FBF4D6D36AE96943FCD96E3465
:10D71000468867ADD0B860DA732D0444E51D033345
:10D720005F4C0AAAC97C0DDD3C710550AA41022755
:10D7300010100BBE86200CC925B56857B3856F2025
:10D7400009D466B99FE461CE0EF9DE5E98C9D92985
:10D750002298D0B0B4A8D7C7173DB359810DB42EC5
:10D760003B5CBDB7AD6CBAC02083B8EDB6B3BF9A11
:10D770000CE2B6039AD2B1743947D5EAAF77D29D9D
:10D780001526DB048316DC73120B63E3843B64947D
:10D790003E6A6D0DA85A6A7A0BCF0EE49DFF09937D
:10D7A00027AE000AB19E077D44930FF0D2A30887ED
:10D7B00068F2011EFEC206695D5762F7CB6765809D
:10D7C00071366C19E7066B6E761BD4FEE02BD3899D
:10D7D0005A7ADA10CC4ADD676FDFB9F9F9EFBE8EFD
:10D7E00043BEB717D58EB060E8A3D6D67E93D1A13D
:10D7F000C4C2D83852F2DF4FF167BBD16757BCA61D
:10D80000DD06B53F4B36B248DA2B0DD84C1B0AAFBC
:10D81000F64A0336607A0441C3EF60DF55DF67A83C
:10D82000EF8E6E3179BE69468CB361CB1A8366BCCC
:10D83000A0D26F2536E2685295770CCC03470BBB1C
:10D84000B91602222F260555BE3BBAC5280BBDB21C
:10D85000925AB42B046AB35CA7FFD7C231CFD0B5BC
:10D860008B9ED92C1DAEDE5BB0C2649B26F263ECAE
:10D870009CA36A750A936D02A906099C3F360EEBBC
:10D880008567077213570005824ABF95147AB8E27C
:10D89000AE2BB17B381BB60C9B8ED2920DBED5E55C
:10D8A000B7EFDC7C21DFDB0BD4D2D38642E2D4F1AC
:10D8B000F8B3DD686E83DA1FCD16BE815B26B9F63C
:10D8C000E177B06F7747B718E65A0888706A0FFF9C
:10D8D000CA3B06665C0B0111FF9E658F69AE62F85C
:10D8E000D3FF6B6145CF6C1678E20AA0EED20DD75C
:10D8F0005483044EC2B30339612667A7F71660D07C
:10D900004D476949DB776E3E4A6AD1AEDC5AD6D9BB
:10D91000660BDF40F03BD83753AEBCA9C59EBBDEDB
:10D920007FCFB247E9FFB5301CF2BDBD8AC2BACA8B
:10D930003093B353A6A3B4240536D0BA9306D7CDFB
:10D940002957DE54BF67D9232E7A66B3B84A61C41B
:10D95000021B685D942B6F2A37BE0BB4A18E0CC3DB
:10D960001BDF055A8DEF022D416C6C207461736BC7
:10D97000732073746F7070656400763038300020E7
:10D980002573202573004D656D6F727920636C657A
:10D9900061726564004E6F20667265652074617304
:10D9A0006B20656E7472696573000000F4D9000025
:10D9B0007163000001DA0000D76300000DDA000097
:10D9C000A763000013DA0000B763000019DA000053
:10D9D000C76300001FDA00009960000029DA000028
:10D9E000F563000031DA0000C561000073656E73F5
:10D9F0006F727300616363656C65726174696F6EE9
:10DA00000074656D70657261747572650074696C1F
:10DA100074580074696C74590074696C745A007499
:10DA20006F75636852656164006932635265616451
:10DA3000006932635772697465000000B0DA000053
:10DA40007D640000BEDA000081640000C7DA0000D7
:10DA50008D640000D1DA000091640000DADA000081
:10DA600095640000DFDA000099640000E4DA000049
:10DA70009D640000F0DA0000A1640000F7DA000005
:10DA8000A564000000DB0000A964000005DB0000C5
:10DA9000AD64000010DB0000B16400001ADB000080
:10DAA0008564000024DB0000896400007466740053
:10DAB000656E61626C65446973706C61790067655D
:10DAC0007457696474680067657448656967687449
:10DAD00000736574506978656C006C696E650072DE
:10DAE00065637400726F756E64656452656374007B
:10DAF000636972636C6500747269616E676C65005E
:10DB00007465787400746674546F75636865640036
:10DB1000746674546F7563685800746674546F75D6
:10DB200063685900746674546F75636850726573E6
:10DB30007375726500766172730000005CDB000033
:10DB40004169000066DB0000216900006FDB000016
:10DB5000FD6800007BDB000089680000766172458B
:10DB60007869737473007661724E616D65640073D9
:10DB700065745661724E616D6564007661724E61C6
:10DB80006D65466F72496E6465780057656C636FAA
:10DB90006D6520746F204D6963726F426C6F636BAB
:10DBA000732100705F73706920213D204E554C4CED
:10DBB000002F686F6D652F6769742F2E706C61740C
:10DBC000666F726D696F2F7061636B616765732F2C
:10DBD0006672616D65776F726B2D61726475696EC7
:10DBE0006F6E6F726469636E7266352F6C696272F4
:10DBF00061726965732F5350492F5350492E6370DA
:10DC00007000535049436C6173733A3A535049431F
:10DC10006C617373284E52465F5350495F5479705C
:10DC2000652A2C2075696E74385F742C2075696EB6
:10DC300074385F742C2075696E74385F7429000025
:10DC400000000000000000004D6B0000096B0000A8
:10DC50002F6B0000396B0000436B00002D6B000040
:10DC6000000000000100000002000000160000009B
:10DC7000040000000500000006000000070000008E
:10DC800008000000090000000A0000000B0000006E
:10DC90000C0000000D0000000E0000000F0000004E
:10DCA0001A0000001B000000140000001300000018
:10DCB0001100000003000000100000001C00000024
:10DCC0001D0000001E0000001200000015000000F2
:10DCD00017000000180000001900000000000000FC
:10DCE00000000000FD6F00002D7700007D70000037
:10DCF0009170000087700000F96F0000ED6F000068
:10DD00009D70000019700000E96F00000000000025
:10DD1000000000000000304300000000000030C39D
:10DD20007371727400000000FB21F93FFB21094070
:10DD30007CD91240FB2119407A6A1F407CD92240CD
:10DD4000BBFD2540FB2129403A462C407A6A2F40F2
:10DD50005C4731407CD932409C6B3440BBFD354040
:10DD6000DB8F3740FB2139401BB43A403A463C40F8
:10DD70005AD83D407A6A3F404C7E40405C47414023
:10DD80006C1042407CD942408CA243409C6B444082
:10DD9000AC344540BBFD4540CBC64640DB8F4740D9
:10DDA000EB584840FB21494083F9A200444E6E00E5
:10DDB000FC291500D1572700DD34F50062DBC000D7
:10DDC0003C999500419043006351FE00BBDEAB00DF
:10DDD000B761C5003A6E2400D24D42004906E0000A
:10DDE00009EA2E001C92D100EB1DFE0029B11C0097
:10DDF000E83EA700F535820044BB2E009CE9840074
:10DE0000B4267000417E5F00D691390053833900FB
:10DE10009CF439008B5F840028F9BD00F81F3B009B
:10DE2000DEFF97000F980500112FEF000A5A8B00B4
:10DE30006D1F6D00CF7E360009CB2700464FB7001F
:10DE40009E663F002DEA5F00BA277500E5EBC7002C
:10DE50003D7BF100F739070092528A00FB6BEA0024
:10DE60001FB15F00085D8D00300356007BFC46004B
:10DE7000F0AB6B0020BCCF0036F49A00E3A91D0084
:10DE80005E619100081BE60085996500A0145F00A3
:10DE90008D40680080D8FF0027734D0006063100D2
:10DEA000CA561500C9A873007BE260006B8CC000E5
:10DEB00000000040FB21F93F000000002D44743EAB
:10DEC000000000809846F83C0000006051CC783B90
:10DED00000000080831BF0390000004020257A38C4
:10DEE000000000802282E336000000001DF3693547
:10DEF0000200000003000000040000000600000013
:10DF000024940000CE930000CE930000FC94000007
:10DF1000CA930000CA930000F2940000FC94000031
:10DF2000CA930000F2940000CA930000FC94000021
:10DF30000095000000950000009500000895000085
:10DF4000009F0000729D0000B69D00001A9D000019
:10DF5000B69D0000A69E0000B69D00001A9D000020
:10DF6000729D0000729D0000A69E00001A9D000098
:10DF7000129D0000129D0000129D0000B49E000042
:10DF800028A600002AA500002AA5000048A8000035
:10DF900024A5000024A5000030A8000048A8000027
:10DFA00024A5000030A8000024A5000048A8000017
:10DFB0003EA800003EA800003EA800004CA80000BB
:10DFC0002C2066756E6374696F6E3A2000617373FE
:10DFD000657274696F6E2022257322206661696CF8
:10DFE00065643A2066696C6520222573222C206CBA
:10DFF000696E65202564257325730A008000002062
:10E00000232D302B2000686C4C0065666745464721
:10E0100000303132333435363738394142434445A4
:10E020004600303132333435363738396162636413
:10E030006566000000000000000000000000000015
:10E0400000000000000000000000000000000000D0
:10E0500000000000000000000000000000000000C0
:10E0600000000000000000000000000000000000B0
:10E0700000000000000000000000000000000000A0
:10E080000000000000000000000000000000000090
:10E09000000000004300504F53495800002020204A
:10E0A0002020202020202828282828202020202048
:10E0B0002020202020202020202020202088101018
:10E0C0001010101010101010101010101004040474
:10E0D0000404040404040410101010101010414132
:10E0E0004141414101010101010101010101010120
:10E0F0000101010101010101101010101010424234
:10E1000042424242020202020202020202020202EF
:10E11000020202020202020210101010200000008F
:10E1200000000000000000000000000000000000EF
:10E1300000000000000000000000000000000000DF
:10E1400000000000000000000000000000000000CF
:10E1500000000000000000000000000000000000BF
:10E1600000000000000000000000000000000000AF
:10E17000000000000000000000000000000000009F
:10E18000000000000000000000000000000000008F
:10E19000000000000000000000000000000000007F
:04E1A000000000007B
:08E1A400641FFF7F0100000071
:10E1AC00FFFFFFFF4006000001000000E803DC0554
:10E1BC00DC05DC05DC050000FFFFFFFFFFFFFFFFB8
:10E1CC001800000019FCFFFFFFFFFFFF020000001A
:10E1DC0003000000FFFFFFFF000000000100000033
:10E1EC000000020001000000FFFFFFFF0000000024
:10E1FC00020000000000040002000000FFFFFFFF0F
:10E20C0000000000030000000000080003000000F4
:10E21C000A0000000800000001000000800000203F
:10E22C000000000054E0000074E0000034E0000046
:10E23C0000000000000000000000000000000000D2
:10E24C0000000000000000000000000000000000C2
:10E25C0000000000000000000000000000000000B2
:10E26C0000000000000000000000000000000000A2
:10E27C000000000000000000000000000000000092
:10E28C00430000000000000000000000000000003F
:10E29C000000000000000000000000000000000072
:10E2AC00430000000000000000000000000000001F
:10E2BC000000000000000000000000000000000052
:10E2CC0043000000000000000000000000000000FF
:10E2DC000000000000000000000000000000000032
:10E2EC0043000000000000000000000000000000DF
:10E2FC000000000000000000000000000000000012
:10E30C0043000000000000000000000000000000BE
:10E31C0000000000000000000000000000000000F1
:10E32C00430000000000000000000000000000009E
:10E33C0000000000000000000000000000000000D1
:10E34C00430000000000000000000000000000007E
:10E35C0000000000000000000000000000000000B1
:10E36C0055C700006DC10000000000009CE00000DB
:10E37C009EC90000D6CD0000D6CD0000D6CD000041
:10E38C00D6CD0000D6CD0000D6CD0000D6CD0000F5
:10E39C00D6CD0000D6CD0000FFFFFFFFFFFFFFFF33
:10E3AC00FFFFFFFFFFFF00000100415343494900FD
:10E3BC000000000000000000000000000000000051
:10E3CC0000000000000000000000415343494900D8
:10E3DC000000000000000000000000000000000031
:10E3EC00000000000000000000000000E900000038
:10E3FC00D96A0000216E000049730000C1000000C2
:0400000300006EBDCE
:00000001FF
